:020000040000fa
:10000000f8ff032079490400a5d30300e5da0300d3
:100010003d0c04002d0e0400c51704000000000074
:10002000000000000000000000000000c3fe03000c
:100030002505040000000000c3fe0300c3fe03000a
:10004000c3fe0300c3fe0300c3fe0300c3fe0300a0
:10005000c3fe0300c3fe0300c3fe0300c3fe030090
:10006000c3fe0300c3fe0300c3fe0300c3fe030080
:10007000c3fe0300c3fe0300c3fe0300c3fe030070
:10008000c3fe0300c3fe0300c3fe0300c3fe030060
:10009000c3fe0300c3fe0300c3fe0300c3fe030050
:1000a000c3fe0300c3fe0300c3fe0300c3fe030040
:1000b000c3fe0300c3fe0300c3fe03005d7604001d
:1000c00065760400c3fe0300c3fe0300c3fe030005
:1000d000c3fe0300c3fe0300c3fe0300c3fe030010
:1000e000c3fe0300c3fe0300000000000000000088
:1000f00000000000c3fe0300c3fe0300c3fe0300b4
:10010000c3fe0300c3fe0300c3fe0300c3fe0300df
:10011000c3fe0300c3fe0300c3fe0300c3fe0300cf
:10012000c3fe0300c3fe0300c3fe0300c3fe0300bf
:10013000c3fe0300c3fe0300c3fe0300c3fe0300af
:10014000c3fe0300c3fe0300c3fe0300c3fe03009f
:10015000c3fe0300c3fe0300d9e40300d9e4030097
:10016000d9e40300d9e40300c3fe0300c3fe030087
:10017000c3fe0300c3fe0300c3fe0300c3fe03006f
:10018000c3fe0300c3fe0300c3fe0300c3fe03005f
:10019000c3fe0300c3fe0300c3fe0300c3fe03004f
:1001a000c3fe0300c3fe0300c3fe0300c3fe03003f
:1001b000c3fe0300c3fe0300c3fe0300c3fe03002f
:1001c000c3fe0300c3fe0300c3fe0300c3fe03001f
:1001d000c3fe0300c3fe0300c3fe0300c3fe03000f
:1001e000c3fe0300c3fe0300c3fe0300b9620400a4
:1001f000c3fe0300c3fe0300c3fe0300c3fe0300ef
:10020000c3fe0300c3fe0300c3fe0300c3fe0300de
:10021000c3fe0300c3fe0300c3fe0300c3fe0300ce
:10022000c3fe0300c3fe0300c3fe0300c3fe0300be
:10023000c3fe0300c3fe0300c3fe0300c3fe0300ae
:10024000c3fe0300c3fe0300c3fe0300c3fe03009e
:10025000c3fe0300c3fe0300c3fe0300c3fe03008e
:04026000c3fe0300d6
:020000040000fa
:1002640046696a6a50664500b86a04006402000080
:100274005046696a6a506645000000bf146704006e
:1002840074020000000000006c0200007600000010
:10029400186b040090020000c58103008408b101ba
:1002a400b0b0b000ff1019010c020608010c0410d4
:1002b400051c0a000001007f00007d000000000012
:1002c4000000000008b10181b0b00084000000000b
:1002d40008b10181b0b000840000000008b10181c0
:1002e400b0b000840000000008b10181b0b0008407
:1002f4000000000069810300b0af1000ff10190175
:10030400111ed0030000b40404b80401d2048a020c
:10031400000001000000000045810300b0af0400ac
:10032400ff101d011528222c0184010a8e0100965c
:1003340001040000ae01248e010001000000000051
:100344001d810300a908b100ffff010008b101816c
:10035400b0b000840000000008b10181b0b0008496
:100364000000000008b10181b0b00084000000006a
:10037400f8b500bff8bc08bc9e467047e97104009c
:10038400b9560400b523040049640400f8b500bf5d
:0c039400f8bc08bc9e467047955604005b
:020000040000fa
:1003a000c4cc020001000000cecc0200010000001d
:1003b0002ccd0200010000004ccd0200b0a902804b
:1003c000d8cd0200b0b0a8801ece0200010000000f
:1003d00020ce0200010000001cce0200010000003f
:1003e00016ce0200b0b0aa8048ce0200ae71b28034
:1003f000e8ce020001000000e4ce0200aa3f3780f0
:1004000028cf02000100000034cf0200b0b0aa8063
:100410006ccf02000100000072cf0200010000005a
:100420006ccf02000100000070cf0200010000004c
:1004300096cf020001000000a6cf020001000000dc
:10044000cccf020001000000decf0200aa0db28076
:100450003ad00200b0af068094d202000100000042
:1004600090d20200010000008cd2020001000000c6
:1004700088d20200ac3f0180e87f03007cfeff7f52
:1004800078960300010000009e960300008404801b
:10049000ae96030001000000a8960300b0ad0480f2
:1004a000da980300b0a80380fc980300b0feff7f39
:1004b000fe980300b4feff7f0899030001000000ce
:1004c0000699030001000000d49b03000100000016
:1004d000340c040048feff7f34150400b0ac0180ea
:1004e000321e040001000000f6210400010000009b
:1004f0004e27040001000000cc2c0400b0ab0280a9
:10050000f8360400b0b0aa806c3704000100000087
:10051000dc3c0400b0b0a880423d0400b0b0ac8028
:10052000e0420400b0aa018020480400010000005d
:100530006c48040010feff7f8c4d04000100000099
:10054000cc4d040001000000e44e0400a0fdff7f3c
:1005500078500400b0b0a880b4500400b0b0ac80b3
:10056000e8530400b0b0a880d0540400010000009b
:100570000255040001000000345504000100000091
:10058000665504000100000020570400010000002f
:1005900050570400010000008057040044fdff7f15
:1005a000ec580400b0aa0380b45904000100000014
:1005b000705a040001000000c85a04000100000045
:1005c000a05b040001000000485c04000100000082
:1005d0006a5c0400b0b0ac80705e040001000000f2
:1005e000305f0400b8fcff7f3e63040001000000a0
:1005f000a0640400b0b0aa80f86404000100000008
:10060000306504004cfdff7fc86504000100000058
:100610009468040001000000a468040000840480c1
:10062000d469040001000000e0690400010000003a
:10063000ec69040001000000f869040001000000fa
:10064000186a040001000000246a04000100000090
:10065000306a0400010000003c6a04000100000050
:10066000486a040001000000546a04000100000010
:10067000606a0400010000006c6a040001000000d0
:10068000a06a040001000000ac6a04000100000040
:10069000b86a040001000000c46a04000100000000
:1006a000d06a040001000000dc6a040001000000c0
:1006b000e86a040001000000bc6c040001000000b6
:1006c000c46c040001000000cc6c040001000000b8
:1006d000e26d0400010000006c6e040001000000e7
:1006e000546f040001000000566f04000100000078
:1006f000586f0400e0fbff7fbc6f0400ccfbff7f62
:10070000bc6f040001000000c46f04000100000081
:10071000c46f040001000000dc6f04000100000051
:10072000dc6f040001000000dc6f04000100000029
:1007300004700400010000002c700400010000009f
:100740002870040001000000247004000100000073
:1007500020700400010000001c7004000100000073
:100760001870040001000000147004000100000073
:1007700010700400010000000c7004000100000073
:020000040000fa
:100780000000000000000000000000000000000069
:100790000000000000000000000000000000000059
:1007a0000000000001000000120000000200000034
:1007b000000000000c0000004552523a20666169ba
:1007c0006c656420746f20616c6c6f63617465206c
:1007d00074656e736f72206172656e610000000057
:1007e0004552523a2074656e736f72206172656e65
:1007f0006120697320746f6f20736d616c6c2c20a5
:10080000646f6573206e6f7420666974206d6f6409
:10081000656c202d206576656e20776974686f752c
:1008200074207363726174636820627566666572b2
:1008300073000000ac070000a40700008007000060
:1008400000000000e00b0000d80b0000f00b0000df
:1008500001000000a80b0000a00b0000b40b00007a
:1008600000000000900b0000880b00009c0b0000b3
:1008700002000000580b0000500b0000640b000049
:1008800000000000200b0000180b0000280b0000e7
:1008900003000000e80a0000e00a0000f40a00007b
:1008a00000000000b80a0000b00a0000c80a0000fa
:1008b00001000000800a0000780a00008c0a000095
:1008c00000000000680a0000600a0000740a0000ce
:1008d00002000000300a0000280a00003c0a000064
:1008e00000000000f8090000f0090000000a000004
:1008f00003000000c0090000b8090000cc09000096
:1009000000000000a40900009c090000b4090000d8
:100910000400000088090000800900009809000018
:1009200004000000740900006c0900007c0900004c
:10093000050000004552523a204661696c6564200a
:10094000746f20616c6c6f63617465207065727385
:10095000697374656e7420627566666572206f6671
:100960002073697a652025640a00000001000000f8
:100970002100000001000000200000000000803f76
:100980000100000020000000030000001f00000024
:10099000070000000500000000000000010000004a
:1009a0001f000000030000001e0000000600000001
:1009b0000400000001000000010000001e00000013
:1009c000020000001d000000010000000000000007
:1009d0000000000000000000000000000000000017
:1009e0000000000000000000000000000000000007
:1009f000010000001d000000010000001c000000bc
:100a000001000000010000000200000001000000e1
:100a100002000000000000000000000000000000d4
:100a20000000000000000000010000001c000000a9
:100a3000020000001b000000110000000000000088
:100a400000000000000000000000000000000000a6
:100a50000000000000000000000000000000000096
:100a6000010000001b000000020000001a0000004e
:100a70000300000001000000010000001a00000057
:100a8000020000001900000010000000000000003b
:100a90000000000000000000000000000000000056
:100aa0000000000000000000000000000000000046
:100ab0000100000019000000030000001800000001
:100ac0000b0000000a00000001000000010000000f
:100ad0000100000000000000010000000100000013
:100ae00001000000180000000200000017000000d4
:100af0000f000000000000000000000000000000e7
:100b000000000000000000000000000000000000e5
:100b100000000000000000000100000017000000bd
:100b200001000000160000000100000001000000ac
:100b300002000000010000000200000000000000b0
:100b400000000000000000000000000000000000a5
:100b50000100000016000000020000001500000067
:100b60000e00000000000000000000000000000077
:100b70000000000000000000000000000000000075
:100b8000000000000000000001000000150000004f
:100b9000020000001400000002000000010000003c
:100ba000010000001400000002000000130000001b
:100bb0000d00000000000000000000000000000028
:100bc0000000000000000000000000000000000025
:100bd0000000000000000000010000001300000001
:100be00003000000120000000900000008000000df
:100bf00001000000010000000100000000000000f2
:100c000001000000010000001c0c0000140c00009a
:100c1000000000000100000080ffffff0100000055
:100c20000000803b02000000010000000400000002
:100c3000440c00003c0c000000000000010000001b
:100c4000f9ffffff01000000fcab2c3f0200000099
:100c500001000000040000006c0c0000640c0000a7
:100c6000000000000100000080ffffff0100000005
:100c70005f22b83d020000000100000040000000bb
:100c8000940c00008c0c000000000000010000002b
:100c900080ffffff010000008477133d0200000089
:100ca0000100000000020000bc0c0000b40c0000b9
:100cb000000000000100000080ffffff01000000b5
:100cc0008477133d040000000100000010000000c4
:100cd0000100000020000000ec0c0000e40c00000b
:100ce000000000000100000080ffffff0100000085
:100cf0008477133d04000000010000002000000084
:100d000001000000200000001c0d0000140d000078
:100d1000000000000100000080ffffff0100000054
:100d20008477133d03000000010000002000000054
:100d300020000000480d0000400d000000000000f1
:100d400001000000360000000100000029ef033e12
:100d5000030000000100000020000000200000004f
:100d6000740d00006c0d0000000000000100000088
:100d7000360000000100000029ef033e04000000df
:100d80000100000001000000200000002000000021
:100d9000a40d00009c0d00000000000001000000f8
:100da00080ffffff010000009e793f3d040000002e
:100db00001000000010000002000000014000000fd
:100dc000d40d0000cc0d0000000000000100000068
:100dd00080ffffff010000009e793f3d04000000fe
:100de00001000000200000000100000014000000cd
:100df000040e0000fc0d00000000000001000000d7
:100e000080ffffff010000009e793f3d04000000cd
:100e1000010000004000000001000000140000007c
:100e2000340e00002c0e0000000000000100000045
:100e300080ffffff010000009e793f3d030000009e
:100e4000010000004000000014000000600e0000df
:100e5000580e00000000000001000000ffffffff2f
:100e6000010000005107c23d030000000100000026
:100e700040000000140000008c0e0000840e0000f2
:100e80000000000001000000ffffffff0100000064
:100e90005107c23d040000000100000001000000f5
:100ea0004000000014000000bc0e0000b40e000062
:100eb000000000000100000001000000010000002f
:100ec00086355c3d040000000100000001000000c8
:100ed00040000000140000000100000004000000b9
:100ee00001000000200000000100000020000000c0
:100ef00001000000030000000100000020000000cd
:100f000020000000010000000400000000000000bc
:100f1000010000000100000020000000140000009b
:100f2000010000000400000001000000400000007b
:100f30000100000014000000010000000300000098
:100f4000010000004000000014000000010000004b
:100f5000040000000000000001000000010000008b
:100f60004000000014000000f80f0000740f0000a3
:100f70000000000020000000000000000000000051
:100f80000000000000000000000000000000000061
:100f90000000000000000000000000000000000051
:100fa0000000000000000000000000000000000041
:100fb0000000000000000000000000000000000031
:100fc0000000000000000000000000000000000021
:100fd0000000000000000000000000000000000011
:100fe0000000000000000000000000000000000001
:100ff000000000000000000020000000aed4873b8d
:101000003624a23bc7d6873b7c5a793bb0583c3b41
:101010008179583bf9f6583b17d2813b742d723bce
:10102000096b5a3be056ca3baefc643bf5474c3b70
:1010300095ccb53bb9f56e3be582803b45db873b04
:101040005d163e3b20c3983ba2796b3bd2a1713b1e
:10105000c9e06f3b5135843bc15c3b3b42e7543bad
:10106000586f723b69ffa43b20154c3b8cd6723bfa
:1010700024178c3bb5968c3b3f3e9c3b0400000004
:101080002000000001000000030000001400000028
:10109000d8d7ff1a0bd1eb074bd7de3cf69addd938
:1010a0001e33b7e8f6cb22dd02be0fee3f080fed90
:1010b000da81d312f71bc0d1f80c21a835b9eebce8
:1010c0001afd0d26bf96880010e2c7ebcad2e00bce
:1010d000d8b5b7eb16da1ed8f9d2fbdffa2618e935
:1010e000fe1fd01133f981cef0d3fdd0c3faee014b
:1010f000eb19f21537e9cb31f7f5e3eadfd80ae768
:101100000df3f206fd09ef1ffc81e8022bcbd0faac
:10111000e6d80a2342360d1b2108f7eb47f41dc21f
:101120001525db3014faf80f0a2ad508dcde15ceb7
:101130003aeec3e41a20bf22e90f06fe2dd0fbe5ec
:1011400027f2cf1bb10bcbe9c3f0b022d504bd060b
:10115000d0cff8d50e3ff43300e3efd681e9b80dd8
:10116000ff2aa92eb0b7e838fde5013128054fcf99
:101170008eca281139008ef1e9ec1159b9242709da
:10118000fa6e0b1b891530197f2c20f1b5bad39e4e
:1011900088083fc3e2d2a50a030fecab30c8ffd8e2
:1011a000b04616b8b7f71df8ed4ce333b73ef0c7bd
:1011b000b931d4e3d01fc889c64ecd10eef1fe116f
:1011c0009d8155d4371031be8311c1c0dfec1ffba8
:1011d000b512ea38dbf9109003fd43f3a412ff0cbb
:1011e000ae1024d6fdeca41fd9e6e3cc2bf105ba52
:1011f0002f172cb8be06c1d8564d0bbf10e5f1ed28
:10120000f0112ce10436aa510c9ac83ad300f7e445
:1012100017f517e9f5f7b2f4fad52c31b346c4b790
:1012200081ea0045fd4503e1bafd343406520ab6b1
:10123000a843bdbcf0e8e209c5ef1d01d5ad0eb273
:10124000e4dd5e23e911e30e28d11cfff52a35b653
:1012500006e4c6a5ed3d362603efd1dd0bbf22a186
:10126000edbe35d738b1eea89d08e23fd681bc8ce3
:10127000d00dd12cc4b0431b40ffc8f2d38121183c
:1012800028ed12e4c3d5012a02adf60113f6c8ca4f
:10129000c3a6c1ff2b0ce4f61b251a3637f1f83034
:1012a000cdb3d714cecf2da0dd3911e8e19f289022
:1012b00018ff192af2f0f65a1d084ac423e6ebfc7f
:1012c00008b11c81fd0bcc3eb5b117375b041a0d7c
:1012d000e9fad3a01cf1f0e60a02a515b3372cbe3b
:1012e0002d202f10ba9e0d0c09140bbb0e05ff0507
:1012f00004c5ea3118d204c9fc02b9a8faff08b53e
:10130000f2d7fde11fece00af6f9efee1a2a95f0ac
:10131000260906dbecf112ca22f3fafcf4d9bcfe72
:101320002a1f810abf16bf1dcc5aaa32ecf1330026
:10133000712bce0613051421f9f108e6f1c91b1f24
:10134000aae5e6ced52b031d35ba19ca112c2b817f
:10135000077f066438d6cf5647ecd6c416bc08b60d
:10136000678e3ebdf94a163b06d0b0550b0fea1802
:101370000fe1fdbf47bb1681d861bd1fd4f2d00a73
:101380002407c8de23d7bed007fc8a1aa6c183383b
:10139000a8ff34223d4e2d1b2ef94605d9eecdf285
:1013a000a12904e7c80807da14140e0b00f22cd5a3
:1013b0001205f30f18f3133400f018fad1092de9d0
:1013c00000df14cf05f724aee10648ff24e7f0f76d
:1013d000d8f7120a21e4f78121d2b9d821810bdd97
:1013e000f939e1eccbffef54ae4bb63119b9ddbca6
:1013f0003a82e8e10ffef1ccd80c311ea352a810be
:1014000007cb0e9644a7f3ac29f8ed0add09114984
:10141000ac6e8d1853e2bec1efcafc21161adbadcb
:101420001df69e1dced1c3283a0be3b507b0e9c423
:101430000232dcbd22dfce24f808da1eddeb0c0917
:1014400058b7c6ad9f00c9fd04f1f811c673810af3
:10145000b3119aefe6d181c5cc2123d5c009e7f6b7
:10146000ef28ffe405e4ff1102079ffc0ef1d3b65d
:10147000f1d7082a1934080ccfff181bc3ab98fe0c
:10148000eb16cfc1fce7d0101d2c2b034925eaf940
:10149000c914192a54f2aa28ca50d3c719ebc896fe
:1014a000e63fc938821101eb47c2910a1f2389e048
:1014b00007db14e73af28e46e2d68105f8dbdecd93
:1014c00043e313f0af3d01f80bc5248fee23f4fb8b
:1014d000b4ed06fc0b3b28c3cde1edaf0b0e00e2f3
:1014e000eeef2ffcf02713b60efdf526b6cd07c69e
:1014f0003cf6f9c4ad2a080e19140481df12341d1c
:10150000e4bfe8dfe0dc30f6ad16f193c60334f754
:10151000bae91fe30f1de809d70f0de88131e9d7bc
:10152000fc1b00ccfeb34e32ba3ed5a9de384ec20b
:101530000900cc4eac2d25e01c012c16e31fe4c0a5
:10154000d7edc217c00e9d33e8fc49354c04f1d6e7
:101550001fcb3d04ec1c17cc0e0a101a11dfcb3741
:10156000210af6d32aba17d735de1f812565d7366b
:10157000daccde346d24f6b71db403aaed3f322574
:10158000d1440db0e0b3eb0af414cdee07f1adadec
:101590005b24ee03a71735e147bf09170715eef0e7
:1015a0002c059bff3626b4acdfff14daf399d14348
:1015b000e6b081ea3422c90c1406170113c431ecd9
:1015c000ecc9d2ef1dd40ad2f5fb04e116de378355
:1015d000101a12260f03f43a2f0f082818d1ecfb2b
:1015e000ffd71bfec6108120b60d37da4e261fdf4f
:1015f000efd117dab3e149e8b02d27c79df51d0dee
:1016000031e8778b243ad2f78a11f5b00b10ca175c
:101610001a5604c3fe9a4318bbeecace88e90402e8
:10162000142481ff262b1be8ecc165b5d0e30ed650
:10163000e1e0c04bb806f74c8ec406deab99ccd1c6
:10164000e90c33ff2c03b0100024e4f824e4dbdac7
:10165000e2e4c1c1b5e30f1451dabb384b01e1e854
:101660002b16d18144f50715b523cc2d8a08deee63
:10167000b9cccfdcf1da230a291022d131da4412b5
:101680001af633ba061a2830e9e8d74ee4e91be522
:1016900024ad0c8155d2018a2d6cef39fafac7fec0
:1016a000452fbfc729faf2e1e7ea8729d4f1ece632
:1016b000dcbffed51e05dff5ed11061232f8d601ae
:1016c000f10df900f106e3ea1781ca06d90bdc1a1d
:1016d0002ec82aa81cd70115ff32e41b13cb212ddd
:1016e0009bdecbefc4f0aab155d92b1b1854cb13fa
:1016f000f4086cb5bcfcf0efd2c009b5d52116d703
:10170000f118d9f901052881e3bef8feeecfdfc656
:101710001a38ed2db73442d8bda77fecaf18fbc304
:10172000ccf00abde1429b2402fe173e671623da85
:1017300010a029f7d5f8c00ec716e158b0e2e7d5da
:101740004d08e0d412e51ec532fc54813c1f39f926
:1017500029cfc939391115c02be12e9ae408f1e0df
:10176000dff1ebb1b60b26cad20114f809e0211360
:101770009ada43f917cfedd7e4def7b9e2da242598
:10178000e02a011081faef0ed2cdde46daf215dc46
:10179000cf1519cdd6f8fc1be8072298042debbb1a
:1017a0003191ea1709afd3d7152781d92433bbd993
:1017b000e30ae7f946a80824e016f9e131409d085c
:1017c000d253dff8eae91eeb21b2ebeb05f7aff1fc
:1017d0002effd6f5f8dba82cd0b408fed6c10ded4f
:1017e00009add8f3f4150032f9d214ddeddd00e6d1
:1017f0001300d9caf5acff3dc003cd1746ea1cb9aa
:10180000209eeedc110681f1fdd61e58afbf94e09c
:10181000a01800001c1800000000000020000000bc
:1018200000000000000000000000000000000000b8
:1018300000000000000000000000000000000000a8
:101840000000000000000000000000000000000098
:101850000000000000000000000000000000000088
:101860000000000000000000000000000000000078
:101870000000000000000000000000000000000068
:101880000000000000000000000000000000000058
:101890000000000000000000000000000000000048
:1018a000200000006a304b39178c72398e334b3967
:1018b000f8803a39a5df0c397ee9213956472239bb
:1018c000d7324239f62235399f5d2339f15697399f
:1018d0004f452b39bcca183901fa8739dbba32397e
:1018e0006c3d4039463a4b39fd2c0e394f846439f2
:1018f0009e1f303986ba3439ab6a33392cc5453925
:1019000036230c39af3d1f393f543539e4d1763990
:10191000b7a4183970a13539a38f5139764e523991
:1019200056b96939010000002000000000000000e5
:1019300000000000000000000000000000000000a7
:101940000000000000000000000000000000000097
:101950000000000000000000000000000000000087
:101960000000000000000000000000000000000077
:101970000000000000000000000000000000000067
:101980000000000000000000000000000000000057
:101990000000000000000000000000000000000047
:1019a0000000000000000000000000000000000037
:1019b000101a0000bc190000000000001400000014
:1019c0000000000000000000000000000000000017
:1019d0000000000000000000000000000000000007
:1019e00000000000000000000000000000000000f7
:1019f00000000000000000000000000000000000e7
:101a000000000000000000000000000000000000d6
:101a10001400000053c7cb3b22576f3bcafab33bbd
:101a20001ba7a23b62286e3bf819ab3b8f44af3b30
:101a30009ce3b03b4b04783b24e7383be1f62f3b7b
:101a40004c539a3b4492c43b31158e3bd4e5933bb7
:101a5000afb3833b13cd653b07f8383bb76bac3b6b
:101a6000675b893b040000001400000001000000d7
:101a700003000000140000001ae706380cffeff91d
:101a8000f81a0dfef602ed112c050aea7fdc501360
:101a9000eafadd0efbd7eceffdf6fb0ded0f05efdf
:101aa000612b4a2fcb20e20b000e2812d8f4f8f954
:101ab00001fafdf008211e99d77f31df2d4d2ce969
:101ac000da080c04feb30d26f6111ccaff2056ecf2
:101ad000012b3551f806c728f1fb46e1f9404fe3e9
:101ae000fff15eeae0f25646d0e510ec03101ff776
:101af00059d7de020508e9f8d31506f9020700f800
:101b0000edf9e5057fdcddf7f011fbf3e2f8f131eb
:101b1000dc12e10006f8dfff55ebf607e60612f4eb
:101b20002afa18ff02cb1bf50622010381cbc10262
:101b30000801e3ed000405f1161813e5000e1e136d
:101b400084b51ff5eaffedf609d8013010ba001c84
:101b5000fbf003049de4f510edc505eb202525f50c
:101b60001e0005fde10119d27f561679ce2add341b
:101b7000051929e5e2c3edf2f717100c77e9bf3636
:101b8000d3d6504005ebffea0008fc231012d40f17
:101b900060a19216cbe27753e71d2ad71dd521e627
:101ba0000cc4f2037fbfc5e7f4070ffbf4de01dcd2
:101bb00019f4faf2f207ef1518a5eaeecaf8f7f0f1
:101bc0000305122b0326e5f5ee0210e9ca085f5063
:101bd000141cda12f70207f7d4edff12faf4fcf73f
:101be0001c3ef4e3c2f50802f13df5e508f723fcdd
:101bf000fff7fe0c57242bd5e812f71506f514e471
:101c00000700f9e907f313fe7f1bbdcef4210b0c8f
:101c1000ef0001e129ebcbf9e30515fadb7fec15c9
:101c2000062012b71ad7eddee7f2ddf1f6d7f401a0
:101c3000e9e39c03f3baf6071d30f92b00eaf1fd46
:101c4000f10e09061cc030091c0b1522fef0121af9
:101c5000010f0b0e121c09e9567f08913fe99ef017
:101c600040f80b4cf3e5e2e3dff03de44147ebbd28
:101c7000032d83ee4b0fec07e00b2719ed18d7f27d
:101c80005536e5fa05ebc5e41146f7f413fcd9f136
:101c9000dbf524f5650b2b69c55c06a9372008ee3a
:101ca00018d02e0ac520639965c522562c24f8f653
:101cb0002216b7cf22f6013de74df642fe81ff45e1
:101cc00034c05246e050ec031a5be4c0d1dc26017c
:101cd000a0b0e8af7c193ad92d3fbe640b19ffc301
:101ce000f14ce22b87aa1e8af251e50b2dcd04cdd3
:101cf000b9d17a071103d42196b12743f52b7f364a
:101d0000a8cfea8eebec398f1d1bbb4f4e44eae99e
:101d1000490006462e0901042303f12df00f152c6e
:101d200046fcde1a74b2f126f2fddd0eeae408cdbf
:101d3000032026eaebe881becbaac6f1dcecf71162
:101d400036fff1dd0c07fbfe7f06d2de31090721ed
:101d5000f3f3f401f6f51efd0ae8edf1c5f211f812
:101d6000d0e3c30bfcf31ce8fc0de9ebdce9fa075c
:101d7000b2082f5302022ee10915fee703f505080c
:101d80000a061a0bf90aee3fb8cb13d1ed5a3c1ee6
:101d900043f5f2f6b7f81821baf324ee813322f6b0
:101da00027f8003f2cfdf4dbf70631ccee231fcce7
:101db0009316f9fdfdf8dd0b0bf0070c061ee7d3bb
:101dc000f0b969c840db1a091e111ad9dd07fd1ade
:101dd0000ef023fb08ca1ceb11d1d5ec17f042e240
:101de000fe0416cc17fd12effe8146b6fdf913c4b2
:101df0006bfd29e7f9f0d800fd0920e4da50653ad7
:101e0000343d81f2000af835df0030b4f129f71fc4
:101e100010ed47ec21ece4161b0ae419f31a02eb6f
:101e2000eb38e01c3dc55df2c731c0fd18360b0f25
:101e3000262af5f7d034f3cfba7252d81e46c2f92b
:101e400043ebefb8d2cafe320808faffedcddc460c
:101e50006226ce244d08f808fe1b0516e6f2cee9f0
:101e60002d7293f17f093b3e12050f0be1ef1e042b
:101e70001211ebdcbec196014f960a6fb10326002a
:101e800011f207fd2206a03eb1b8fcb567ba843d49
:101e9000362017c7012e9aaa2e68abf781f698d67e
:101ea0006518b82c630b9528c65c2acffb1b3cc178
:101eb000810f373a2c0fe4d7dde3c3edf3fcde28c6
:101ec000f2e9e5efd4eee125f0e41a18072d161f2c
:101ed000071d1238f90c16f4e9ebded02f2fe72995
:101ee0001520f205cfe6f8f7fa12ed39a84328508d
:101ef0006424270033f9240cf60e073ed2e048fb99
:101f0000da5545194626ef16e7f0bfd322f2d9e796
:101f1000fbf717edd62d7f47172bd106018d062b2a
:101f2000e1fcf624ffe8f8fc881f0000341f0000e5
:101f3000000000001400000000000000000000008d
:101f40000000000000000000000000000000000091
:101f50000000000000000000000000000000000081
:101f60000000000000000000000000000000000071
:101f70000000000000000000000000000000000061
:101f8000000000000000000014000000e649af3926
:101f9000ece04d3927d19a399de98b397fdc4c39fa
:101fa000172e933990c39639962898398b575539ff
:101fb0004c0d1f39f45c1739d9bf8439cc16a939b7
:101fc000d66f7439dc707e39e793623948ac453995
:101fd000d21b1f399e509439894e6c390100000084
:101fe00014000000000000000000000000000000dd
:101ff00000000000000000000000000000000000e1
:1020000000000000000000000000000000000000d0
:1020100000000000000000000000000000000000c0
:1020200000000000000000000000000000000000b0
:1020300000000000000000004c20000044200000d0
:10204000000000000100000000000000010000008e
:1020500032bbcd3b02000000040000004000000045
:102060001f28a61608a82d194cc4b233152f3cbf43
:10207000bf06d4312be4bfbb2b07af2737c7ad2832
:10208000c7340151bc0a9d03fdf1ace5d8a51d1173
:10209000ffa4d5201a19adc6ebade30990b521b761
:1020a000b6b013ac84a4fe2ee53ccfdda1a4af2bcb
:1020b000492ec1cfc6b2cae4cf2e1e9fa6ebf6d3df
:1020c000e2d481b4b81007b8ca552360cb42a5c585
:1020d000bd294317b171cc3db407e4b803a6b814c9
:1020e000c8daccc60dd1bc00f8ca37d4f12be44114
:1020f000da05def7c5312f2338211017d0b948a9ea
:10210000ee28a2eb2a08e09fb2ca1ffb4af11a1080
:10211000fb2bd1171ed5072afb164c47faeec82712
:102120002a3926c01c3807c7d3b7e92cb6addbc5a2
:102130000ff557f132e9ca1dceb5d215f03ff800c0
:1021400056c615f429ad0d1a4fdbe1dde02220a2c1
:10215000aa2cd2a2b0f104e5ae18f6d8f84c34eeb1
:10216000742100006c21000000000000010000004c
:10217000000000000100000091de983b020000001a
:102180004000000000020000031a041c07e9f804e4
:102190000d07e7f407d7e3df04140af9e70af9efbc
:1021a000f7ff02fdf9f900de03f2e8fef208d7fbc3
:1021b00001f8daed38f20bff1c0fe80007e1f3f944
:1021c000f101df0b082ae5eed1f9f33efffff5f24e
:1021d000050edcf0260cfa090eeee71bf4effa11ff
:1021e00025c012fadb0cf32efa00ea160930ef0aca
:1021f0000dfeec0200f328e8e9fec503f7f2c2fb8e
:1022000025da2a12e801ea35e6f606213427e30941
:1022100024edea00f9ee2c2f141fc2fbe5d0dff00d
:102220000cd623d1e30bdd45da070f0de1e31d10da
:10223000dfded4f8e00e202ecff3eae5eadab0cf05
:10224000ffe424e9dcd4c41bb60c05ffea1c24051a
:10225000c4c7f3ded6e71c0fcf01d90bd7ecdb0eda
:1022600015d606e0c1f9d1021107080ee2f24427a3
:10227000e4ec09ecdc02091812d7faefe3ffe1fc09
:1022800037ee1010d5e7e62bff12f32b01c520180f
:10229000e9f51ceadc0a2d36e6def702e2e8f8137f
:1022a0004be54406e7e7f7270005fde936dd1c02ac
:1022b000d307feeeeffa18ffd5ee1608cf0a0d0b86
:1022c000efe80525db041c110e23e2f81604f91fc4
:1022d000f1180cc904fbeee9fa0e1c25d2fd031619
:1022e000fde9d810c617fdde07fbddee13e802cfcf
:1022f000f3fa13ea16cedbd2ea00ff26e00d08134c
:1023000025f1cc090d2d11d8ff11e52b0cdaebd0fe
:102310000e11f9f8f714c0d6ef0a062fe1050e1ad0
:1023200022f2f4050706e6ffe304d81def0026c8f5
:1023300006f1e9ebcfe4cacb26f5d40209e201109d
:102340001f04d11a0913ebf5ca09d74401f5e5ecce
:1023500019d8e21beee7d2dd0c08dceb17eae21e2f
:1023600002e1fb1e0b0af3d409f3d719fef3be19e1
:102370001f02e0fec8ede4d50ffafa1816cbe80804
:1023800015e4f3cbecf6dc2f0b06ea420f0316083c
:102390001710bf12e4f035f9013902eeeddee7e97e
:1023a000f5d92e180e0800221b23040afafb0c266e
:1023b00019ffe0f2ee050fed0f19e322f7eed40757
:1023c0001edb3211d908d529ed15e119182af411af
:1023d000e7c4e0e6d1f919130ecde4f1caddfaf84d
:1023e00033e83300cf0de143f7f90004040e390d53
:1023f000f5fd10e3eff6352904fb00f1dae60ef8ff
:1024000020dd35f8c1f8dd12e0f21e18132a181588
:10241000edf304f0e6f01e271d09ffefc2f0f6db36
:102420001dd214e5cbfddd21fafc13010bfdfe1bd3
:10243000e0e807eaf00012f7bdf9e8e1eceef60695
:102440001be81b11d7f1fb22ed33e93af000182508
:10245000eff01adee3e01b13f9f6fe0cd5dffb25e7
:1024600024e018fbd4052014e8e70a1ff2e01c144e
:10247000c804facdfb1afe04e9f80724e1f40124ac
:10248000f8f72eeecef4f219ebe1f6f2250b38fe5a
:102490000d0a00f6e7f6201efef4022cd8f3071111
:1024a00000df081cd70405030af8ffc91e1127f234
:1024b00000fbfef6e3f1f609fcec0d0fee090e0e43
:1024c00009e4bf1cf2ec04d2022eb11c100f0fcc99
:1024d000030917ece7e5c2c0140e051111eeff1752
:1024e00009f7d0ffe628f8ecff27d7141c00fdb44d
:1024f00018f81bf9e2e6dcbdef11f904f504f4125b
:1025000005cdeb151bf3f9c50b2bc11a011be5df3c
:10251000f30a1cf0fcf502e3fb19f01adeecf029db
:102520002ddfe705e3f409e7f6e6e2110cf8e3e74f
:102530000901000debf2d5ce0104d0f0efdb130959
:10254000eb04c7f9edfdeeeffefed424f1ecc90279
:1025500028f1f8dff2e3f81407fbd01400e6c7e631
:10256000f7f6ff0bf326e9f91efcff07ee06b3f8ba
:10257000eef8e2f5efd903dd00e2040b1cbdde0648
:10258000e5d903c2f319e91ff4eb30341acc133246
:10259000fd160e0916f50e1aeb2e38d0fb1a3bc9a4
:1025a00000232b0520c412380a02212808f7e7333c
:1025b000070dec0d45162c160507e2f008f411f492
:1025c000f40319d105d9cc33d605132aee0a23fc1e
:1025d000f807f10932cc20f207f6cabb09cf12ee98
:1025e0000006f9d8fcf1da27d0130a17f10535fdfa
:1025f0000c12db13050f050cf5f5d8d703d509fd33
:1026000014031d1902edbd20e30a0417000b15f792
:10261000da11d9f9060f150215ee06e7f5dd1d05ed
:102620002af115f8fce7d120bd1cf13a40de0bf889
:10263000faffdff30c1004f7f5d4f4dd0cd500f04d
:1026400008e51af1ece2bc1ab707fbf9ddcb0a1a70
:10265000d301d3f6021713fbdde70d17f5d007f210
:10266000fcf300f90cdade0fde0201f5fbd908fd00
:10267000ca04cd07eb190b09d6d0fa0812c80bfd16
:10268000fc041710f0d6c822e9e5ff25cdcc25fcc7
:10269000c218e218f2f801e4faefe70af2ef13f4d5
:1026a000eef2320a01f7ce0ec8140b0fdadceff3ac
:1026b000cc05e005f802f2d6fed70e090ae5f41eb5
:1026c00001ee2012fdf3d5f2c8e407ded7081be8bf
:1026d000d111d0e701fde3dff6e40b10f8ea1b0ca3
:1026e000fe1513120809cdf1b8dce8d3e70104e7c1
:1026f000e90bbd2cfff4b9cdfeedfc2524e1f71666
:10270000d70fe61033c9c5f3c80b0df6edd8f0eac4
:10271000f615cefd0e04bcd31d000f0e03bbfc1935
:10272000f303e11415d9d0ece0ec00f105e4e90e77
:10273000e418ba1b0f1de8d30907fb0705def701f4
:10274000fb030e382ce1d41aeef0e70df1f3093259
:102750001bf0f010da2ff9dcfaf709fa08f01ae6a4
:10276000ebfe141828f8e916f3ef0b09ebed114115
:102770000618e40a12fcf7eaea0a12172002f50426
:10278000000ef21e0306e114e91d0d082117fdc21b
:102790000801f5210be8f12c1b1cec0cfdd5d9240c
:1027a00028020debec1edce1f1102203ff061bef0b
:1027b000dffbc3f926ff2210fef5e2280fff12f619
:1027c0000df1261c141aeb00e91301fafb0603e6cf
:1027d000f21a08ed1c09091809ffca29f1eae306f3
:1027e00026f91ce0ed01e6190f091602f80b28d6b0
:1027f0000ad00bd4eba30bfff5dfd90404eaec17e6
:102800000c0534f3eef4200e12ff07d30801dcecc4
:102810001aaa09faeec30e15de06cbfaec10c302b3
:102820000ffa1beff7ee361c0912f9e4010f0fe166
:1028300008a72eefb3e0130d0a07b7e2dd17fdf688
:1028400025f71ee7d01b2215190bf7f504101cd431
:10285000ffc605f8c6d20111f41dc5d5120dde1450
:1028600013f6ffddf7fe23010b051bf626e524e03a
:10287000d1cb03f8eacf1700e406e0d8e413e4cba9
:102880000bf62af8e709151eff1f0505edf828ceff
:1028900000e6fcdce4a81317e903cbddd315edbd9e
:1028a00022d710efbcf3fc161308f0f82a1929c937
:1028b000fdd5fde8dfc11107cbf6c6e8db07f8b7a9
:1028c000dad602e1d1db150616eff704250ff7e3a0
:1028d000e2cff9e8d9ca18e9171cabccec0cf0b37d
:1028e00024e716dff7de050312f9e21111fc00ce32
:1028f00006d11e04dbc40f0ffe1dcbbfdf04dcbfff
:102900001ade14f1e3110f121204ed140b1dead9b3
:1029100010c200f5f7be0d0efd3ce0e7e10be1db78
:1029200023022fd0e80f0b161016e120f9fe0ece71
:1029300002b32116e7cd35f9e909a2dff317d3b9c0
:10294000e0e604b7fdfc29f33e00dd270b1704d0b9
:102950001ea91a17f5b5faf8dd0dcc150019fffc04
:1029600017f1f5f4091820fb0dedea1b380ff2ed15
:102970001ad13109edfa01f01c24d209f92c17e61d
:10298000170028d6ee191122f80ffb0f101beff9d4
:10299000140af80cece8f2ed12f0ddf8190c03eb78
:1029a000ff02f8df04260bf30cfffb23d8fbb9066c
:1029b000260518cc23dce7e80e17f4c1f9f0f6f38e
:1029c00005f7f0efcffd38f7edfef7140ed4002e2b
:1029d00009050aeed6ebfef41a0a12231de4c61608
:1029e000f1ed290de81618ffdb13cbf520f0d00927
:1029f0000aedead8daf30cef0303ee2006ecc21579
:102a000029e204f5e9ebf90cd514e205fd20f7fa0b
:102a10000efacbffe6ee030ce8d3d9f1faf4f1f5a8
:102a20001de439ecdf14ce14d410e3eed6f3e32a20
:102a3000fab6e4d4daef150f16fdf7f3d4d5dcfec1
:102a4000f5cbfbeee1f4f911011cd1fa280ce724d7
:102a500031bfbddfcf21191c16e80809b8ecf2cc54
:102a600025d717f5ea1ee415e32de9232b2122458e
:102a700021ca03edcb2329f9300ef9fdba0ae61479
:102a8000ebe024f9b720ed3d0644e1184144fc0495
:102a90005ae4d9fce70508fa26ecf7efe408e4ed80
:102aa00026f806ce0f08e8080b0ef72b03390f297e
:102ab00019080506e9f7000d0edd0a150405170ac9
:102ac00014fffd04eff5d719f23dfd16ea080028c2
:102ad000e8131eeafd16050b07e8021f12070a108d
:102ae0001914171906ffe04b00230b0c21ef0019f6
:102af000e2ff0fdc10f01af7fdfdf60be818fc18ea
:102b000015f30609fd100e1005080015ffede92765
:102b1000fd1a11f80e0bfb3302fe1f1f00060711f2
:102b2000da01102ff7fffc231a00f3dbf6db0314a6
:102b3000ff2718ede513fb0c06e4fe341711f81d12
:102b400010100028ef3c17e8ee1b0cf4fa030123e9
:102b50000e1a11d3fe02eb2526132816ec08f809ed
:102b6000f9e9eb1ff93c31f1f124001106f51a27c0
:102b7000220afbf9fb11ee230d0a1d14ff13fc259d
:102b800004e5140d12003a23eb19ef2b0ffa1e3750
:102b900038f0eafd180b121211fd2ff3f1ea1a0ab0
:102ba00019fb2c1738ec121edd1df20b0507151f43
:102bb00014fbf2ffe71216fc0604ffefdefefb0437
:102bc000f8dd05f0eef2fc1ee403ee2ef2192527e7
:102bd000f4fde804f1fa13fa23e1d1f7c2eafe1694
:102be00008ec040ad3efe20dd911fe2110101025d4
:102bf0002415dff5f90904fded10d3eddc1916fffe
:102c0000f3dbfc03ebfcdc30de1afc2d2000362667
:102c10000a0709ebe51516160c030208c3fa0cf1b6
:102c20000ecc211eddefd712c50fef3427f01a2787
:102c3000e81cd2f5ed02180bf9acf106cfccf20f7f
:102c4000edcefb12dc03b625d210f70a08de0a1d12
:102c5000e717d8eaec0c1de904d21704d1dd110204
:102c6000fee40715e8faca23fef0f434d4f4051e96
:102c7000bf1cefe0e632250008c90104f4e00e12a3
:102c8000d6fc1dfdf81edbfcdcf303f2f60d0e0294
:102c9000ea0ccccce814eef605d10e1df4f41afdc6
:102ca000b2e3041c072cc201ade003fe0f08f5e5fa
:102cb000c618cbea18eac7db15d11224eaaef70a28
:102cc000cef5fff9000ed0dac7f50af9e9fefddf0f
:102cd000d90fd1c2ecd9d3b4fec4190611e3f70f52
:102ce0001afcfe06091ccbe1c709f50dea08f1ec58
:102cf00001fdb7f3e900c4d11fc42607fec9ef0eda
:102d0000fa03d61424e9d0d3c701f52f06c5fdee8a
:102d1000e30bd20efcf4c00005fbf90408cbecf287
:102d20000b0bf70f0408f7f9ece9f713d803d4df1e
:102d3000f4dde42411d6ed1b1fefe6f31cd6ea09ff
:102d4000f5f80a2a1805fc11f709fa01f21fdddf70
:102d5000f907f4eadcf6e6f6e80d08f02de1d0f428
:102d6000f7e305edeffa120eef0af412d0d8ea00fd
:102d7000fde9ed06efd80be016df0febe7f2f8d533
:102d8000f5dfececd2030226beffe9fff9190ee5f0
:102d9000060cdff812cf1211f6effff8e5c01f2e78
:102da0001ff2240af6e5f002162af7f8f8fc2802ca
:102db000edf923090af8390bdd0812f90500fb1dae
:102dc0001f061513fe141915e2ef160efef8fd0b83
:102dd000ddf0ec111aff2e07e2ffe50c16fae30016
:102de00005fc25e718ea0f171deff9f5d1fc0b04d8
:102df000070803f12ce60d2eff140c010709fa1f3a
:102e0000f2df40d8ecdc180b24e4d5f70febeef83a
:102e1000c5d80b0fee07f611da16da0bfc200edf21
:102e2000f7d400ed02df14d307ddc2f307f72bf26e
:102e30003cb30121d7f6c9e31116fef5fa2c0ad5e9
:102e4000d50bd8cf04010ceb10feeff20df0f7fa22
:102e500019dfff17ece9f6d7f013ec0b1f1f15c1b4
:102e6000f216e3fa01faf3e8eaededf720eef617d1
:102e70000fe8e4c615e8e7cff521fed1ecfd1ef31f
:102e8000fef000edcf0100c3f903d80beeea0918fc
:102e9000eee6e102e7e4e7d71afaf7fdf2fae1f528
:102ea000fb18e8d2fe00f3e0011fe2f6fe0511e098
:102eb0001deb04080fd4f7e30704040321def7fd3c
:102ec0003703ece71505ee00e1071efa04f9f1d827
:102ed000ecffdde208c3043ad803d4c913d516deeb
:102ee000f1d826fbf0cdf91eedf52803fcffe6de58
:102ef000eee4d900f3ed202feee6bfd5fcc7ded31c
:102f0000f0f719cef8e4c91f040112ff0009f3db42
:102f1000d4f50813d5c71a20f1dff72003f6f5f62c
:102f20001406230814d6080f120403fa0ef443e51e
:102f3000091324e907d51719fd1bddf2030bfbff6d
:102f4000eb151713f6071f0c0d1001f111f8f5041e
:102f5000fcf3061fd317141eede5040817eae1334e
:102f6000f70b3f261bfd0a1813f5e3d2081407e7f9
:102f7000030e23e70d2101f403130628171713127c
:102f8000ed10d40104f928bf19fc2fe9130afee45f
:102f9000e20ce6fe2306f204e00120f31ae6351007
:102fa0001c310a3508e4ffd5fbeb220707f32befb2
:102fb000e810d8082df8001ce003f413fae701e547
:102fc000f91dfc1922ede910eb072b021804f5d8c6
:102fd000fced14002df9f818e9f3e41715dc09e607
:102fe0001918f8ec0ffb0300f1e22206fbe520d9eb
:102ff000c5f210f71dd8fd0ce300eee115f5eee982
:10300000fb1021fe1bfeff111ce3f00e1d120ac473
:103010001af40b251002ef05f641d30e10e6fee17f
:10302000f00ff3fe2a061feef3fd0cfa2318fdda6b
:10303000f4e0fa22ffdfdafced31e0e3211a18fabe
:1030400002ff07ee0de31212fef003ee1028f3de8e
:1030500003e6e90c12bcfa15f91da7ef19ea0dfaff
:10306000062903dd0ff81e000def18eedff50fe067
:103070000803f80517dffb11f61eedc404f9fdddaa
:103080001c070feb06d413ed1c092bfac9c202e68c
:10309000c0041c1215e1ece8d310d3ae2b05eeeb07
:1030a000120828ffffb819fb12e5ffe816e62acf41
:1030b000eb16000a1abef61aeb30dfae0f1bfdf35b
:1030c0000a0f1cf303c309f2f6e3070f32061fce03
:1030d000cd16f810f4ec1010cc2bd5d201f61ec58d
:1030e000f916f8f102e514f306e011fc120befe318
:1030f000e4e8fc1df4dd10edfc15c7b8ec0f0dd7ae
:103100000f06fe0406f7f6f803fe13fa2a2806e86f
:10311000fafb202717f905f3c925f4dafcf71de7b8
:10312000fd0e14f218fc0ef003effa1a1f0d13c473
:1031300007fb164010ebd7dfe7ffe7d3e9fc09f305
:10314000d81716e829e819f2fffd0af9fe2128f63a
:103150001ee2ed2008ea0ce2ef1dd3e61c0716bdc7
:10316000fc4221de0df61ef21ee808c32d0709e21f
:10317000ee094522040bfbe8f020e9f02c291edfc4
:103180000f0df1d40be80addfe1a3feee9c4befbd9
:10319000ecf0f31a0dfdcae2f00014f913e5010c8e
:1031a0000b19f6fcf1e408c6d20a1cddeff412ebb1
:1031b000d9ebcbee10fdee06f5f10dfaf10f21067d
:1031c000ec05f91f0a1ff9ffec110cf9171d31f07e
:1031d000de0defeef913e504ebfe0f08e5dbee1b69
:1031e000fd11effcdbe8c2fbdfff06fd2bf626ec52
:1031f000f9d9ebcc02f3edece9180517d700e3267b
:10320000fbfbfbfae82ce1e1eafd0af5131be5f50f
:103210000ce6f334db09e1c4142afffe08f20305cf
:1032200002f008fc12ecdc0fe2fe18ff0e0027eda6
:103230001bf200f4e4e11f1a053ecdfa02dddaeddf
:103240001bf717e9f402cd16f70909fd150c02dd8d
:10325000d9eef0ead5e01129f9f4f1f0eed5b0237a
:1032600002fa0dead621ea0d0ef51c0ef5ec0be480
:1032700004d40be8e8c9fe09d72cdcf11af9e902fd
:1032800000ed1ef2d6f42311022708f60d0318ca2a
:10329000f1d920bbdfaf061703e3d4cafcfed0f898
:1032a0002adb0718d5e107011b05f40622132adbe8
:1032b000e8e818d2e9c1fe0e0317bfd60615ece503
:1032c000f0f513f7e0062d082127ffe0f8fb04e8ee
:1032d000bd15f9d4e6ca0b22d800cad6fd0ee2de2f
:1032e0000eed1c0805db170a07c5000602f915d20a
:1032f000fcdb0cf604cbf1ffdc03baccdf01fbca2c
:1033000005cf20f6e9f50f1e10f2ec2f31ef03e2a6
:1033100001ed25f323c40f1a0c2cdcf1f61d0df181
:103320001e0b0ce2c5be090d211c0f1cd7ddf6d407
:103330001acc0825eab1152b1beedae0d808e7ce47
:103340000cf129cfea070df510f6fc042527fbd078
:103350001fb00e130c07140104e8e2a7e62011bd0c
:103360001ee6fdecf921120506dbf21c2614f0df47
:103370000dee22f9110ddeebf734bbc5fd3b1be171
:103380001efc04d5f11c390021ce3aebe6fc25f0f9
:10339000e2002ef42c1ffb17b91835f3250154c792
:1033a000073c091302cb29f6edc526f7e9e9fbe353
:1033b000e5f9e1252cfa0422ca0510f6201615dce1
:1033c000f12714d117dcebdaebe82af0faf812e077
:1033d000fa0ce9144600f30acd19ecdc08e306e91f
:1033e000d302010039ddfd0bddcf0606f4be0dcca6
:1033f000d019e00a4102f400b615f9fd20dc20f9ed
:10340000c1f0071602f2e413f7f00326f0e90ad040
:10341000d820d01e19fdcae30a01f4e228dc14fd0d
:10342000e92efdfe2ef1edf907e0f9ecfc1004dccd
:10343000e910df0d29ffd9eddbfc03f20df712efe8
:10344000e7ecda0829da11e2fbc3efed01f00fe651
:10345000d0f2f90a21faebfce502e4f119d90307ed
:10346000ed140b0407df0c0301d107f3d3c412e3ff
:10347000e9fdebff1105d500c3ebfbc7260b1eca08
:10348000ee0619e61aa0eddcecb1ffe4cfc711039c
:10349000c208d30f0607dfe0a80704d40efe16e02b
:1034a000e40d18e906aeec06ebf00bf6dabe07d633
:1034b0001813dd1826fedefde619fe001add0dea02
:1034c000f4091d1134d2f5f0f3cb08fbe4caeb0a82
:1034d000d90be2150bedffecc618fef313e80dea6d
:1034e000f521fbd902fd04eafdb9f5feeee0f10796
:1034f000f8f5eb241613f108e5ff08da01e2feea1d
:10350000e81e11f90afaeaf9e2dbfbf0f8021ef80c
:103510002910e42f04f7fec7070ef2eb32de07f2a4
:10352000f7fd101a25cf04f9d2e801fe08eb32fbb3
:10353000e70ce62e1c28bcf0dc07e9e31b0806e8d4
:10354000f52501013ccd04e405ed33e7fc08040654
:10355000e9ef054a182002d1020edeec25ff1cda45
:10356000002a26061bd0e7140ed83dcdfdf62d0807
:10357000d702fa2e2706f4f3f00a0f0e21e71719e7
:10358000b147ed0224daf0f1d7f2bde8edff01fd1d
:10359000e0d6cfc0cde8f10806f103fccfdabc0fce
:1035a000f7accb12d31ec7f7e60795e1f1fbd5d9ef
:1035b000ebeecfdbb708bbc3fd07e9f3e3d1d915c9
:1035c0000cdec4040f03f0c207f8b1e51206b0e840
:1035d00012d8e10ab119adc0031ffdee0cfec10007
:1035e000f800a5fc2412fab50cf7bdee0711d201c4
:1035f0002bd716f8cf2ddeb6141efefeef1ae2f220
:10360000fa07e7e900faf2d2eafcdde6dbdb01f7d4
:10361000fefa051ae11edfe21b050a36022c180924
:103620000a07c3f2faec07ca13cfd6cfd8fbe1ffe3
:103630001e080b0f2418e9e1f90c13101415ecf017
:10364000e708e41d2521fdd60bd502d8f0fee602e1
:10365000100b101afd35fccd00100dfb10080ffcef
:10366000e40aed10f81f0ada07e40a04d2eeee25a8
:10367000031c0002e80806eacbe717eb19031af46b
:10368000d717cbfc14edf8fd17cb0bdad6bad81b45
:10369000ed1c0cee24fff103daf90def180b01d647
:1036a000a720c7fd1cc5fbf4fed00b07f1b7eefb4e
:1036b000071305e31401fb03eb0ffa1313eafeed06
:1036c000c3f9df1eea0314f921d321c701e106e69d
:1036d000f5f8060a15ef0917d20de5d4d807fcdb7b
:1036e000de10f60104f407fb00f607f5f2f302f929
:1036f000edfee5cd13e01d340d0519d50afff701e8
:10370000f2f40d06fa031614ecd30401f7e01905e0
:1037100018f6f7c51bea031726d208fde5e8e7050a
:10372000eed2060fcf05f1f0e8fbefdc1500f40d4b
:10373000f9f9ffdce608f12606f01a1501f3fafba9
:1037400008d1dfffb9ffdaf31313e5db12f909c380
:10375000edc701cd1de9101608f6f6eae3d7dcfa4d
:103760000ee0ee0fc410eff5dc10c9f00af3cec581
:1037700015cad9faf1eb0007facae7e1e9b39efdf1
:1037800008bbf6110101cd1df70a13481bf1f41215
:103790002df6d61101c2511f061800fae3dae4042f
:1037a0002ecd4c10f800fd2f0812300f1007f1211c
:1037b00021d109fdead8520d182703f704ebd8fef2
:1037c00014e239e9f3eefb51040fee1207fc100e80
:1037d000f3eb1ce601dd53350ff3efe6de01fceb06
:1037e00027ec21f0b9f80a27081a0d261f160a0b34
:1037f000fee911d7f0cb1e3c10fcdbe6f10ffbf32a
:103800002ad62bfecdecfa5cef1f12041d1609f22e
:10381000fccd0be5dbcb10200406d3c5b917d609c8
:103820001cc206ffd6f70a1604240a0af0ef21fa92
:10383000eee2fd01d5fc2310f3f8cef5e5f8fafb36
:10384000e8222bf7cddb1218fcf7eb10f5bb22f6c4
:10385000f50809f204d9f705e90c1405c3000b1ba0
:10386000ebf30013dfc21426f5fbfae81aec3fff76
:10387000ca07e3ddeee10212ee170d22e5f31c1498
:10388000e6e60f0cd3021415fff2e8cf450c0de26b
:10389000e6030beceedcfdbc16091203f0f7fe1d8f
:1038a00010e0e50be6fb08e8f816e5e44b2f1fe611
:1038b000effcfadfebecd7ebe11b0f48d81c0a203a
:1038c00044e79cf6f2e005dc1115b9fe270feed6b1
:1038d0000df90dd3d5edced224fa0007e207dd0aab
:1038e0000902f213f60f10c1f8d7cd0902d3e9dab5
:1038f00002e411eb02e4d5fa1bc80b20baf0fa0c73
:10390000f0c7e3f70d16eceef30fc706fef4d3e7ae
:1039100016f3f924e619d5e704f908f2e9efdef722
:1039200019d0ece7c0f4060bf8ff1f1bf00719d6ff
:103930001de8d701fad201d30f0bbf001cd3ecea6c
:10394000d0fc34fff200f32ef30ae333fc27e1044a
:1039500012d4e9f202f82a1a121bf8f6f6e3d004a0
:10396000e9fc0fda11faf92cf8f4080204f4e7156f
:1039700007fcdb02f0152aff1415da0006f308e550
:1039800006f312f7ce16da370829ed2201c6e9cd83
:103990001ef80c020005d8cb19c6f51c20eef23338
:1039a0000b20ba081c30d3e4e909eae8f21308fa5c
:1039b000e2f2e1f215efe20211f4fc04e8ce0615a2
:1039c00001edc607f021ea10e804ed13f612000736
:1039d000c7f3f9dbf00a0be304f11f29ebe0da4946
:1039e0002b11090de100e1f8ce02e6001b191115bb
:1039f000f6d8ead5f9dcf4f2fbf7cc15e5d4cbe246
:103a0000ffdc16e8d810e406dbf203eb0d06faef54
:103a100002d4de0ff40be40cff1caa060cc2b91b87
:103a200010e503ed151aea06f71102fa0bf90cf48a
:103a30001ceeefe9e9e31824fc2adb0de9d6e31ad2
:103a400014e70a1203f9ff04260ee1f31211faef4c
:103a500015ca08dbf6e70f251b0ed408ee25d53472
:103a6000fbe404fec71d0e042410020107f813f93d
:103a70001eeffb0ecbe20110ee18e71e0d03d6077a
:103a800009e02428e3e82601101800f6e80d09f8fb
:103a9000ebfa1f0fec0af824ee04efee01fac5f57d
:103aa000290a131a0ce01af30e27fee909fc1dcdb2
:103ab000e6060bdcedc909fe1b03ebda011ddaf2a9
:103ac0002406fe00d9190a07250bebff02e500e8e2
:103ad000d3e72dfe0dca0315f712d8d8d717d1c8d2
:103ae00026e00dd9d00922fc03eef60c29f7eae511
:103af000ebec1ae812bf0719e814aba30124ecb4ed
:103b00000ed112befdf1140735f600fe183e06c6b2
:103b1000f5ef3ff009d70125ee22e2e1e91df8caf1
:103b2000170d04adf4f335ee342cf8f8fd240bbd7d
:103b300021f21ae00bbe281a0307a8ebe217fdc218
:103b400012db0eccdffd2cfc2c1df6e93411fdd070
:103b500001ba35f406f8122ef810bcdddd0defc405
:103b600003dd1aaae419121501e9000b2617e6dc99
:103b700000ba1bf811ed1e350f38d5e9f24120b718
:103b80002be5fdc1f50d2702da09f7f2c4e8ecddfb
:103b9000fa01d1f7f5ede0d104e109ec2abd0e12ee
:103ba0000d0df5efeb0bc5ccf207f3d9ec1c13e8c8
:103bb000daf6ddc90dd8b9c4f508fbf8fed202fd6e
:103bc00015fdde17c618dfe3defcee100707dbe8a5
:103bd000dcf3d5e2f1fdcaff02f60315cfcddd110e
:103be000fbd4e80ad934ddeccf07d2020e221de067
:103bf000f6c6d6dbc3e0d5f910ffd8f5cedbc51786
:103c000018b6fa0bd321f402d81ccdf31001fbe255
:103c100024f0cb14dbf0fbecff0ae802e6e1f5024e
:103c200025d3f304f122f3fbdce1f7f710f3faf309
:103c300005ded3f6f0f000091c18150bfcdedb10d6
:103c4000ef05f30ff902ba0cdef1e3f20526fb06ed
:103c500021e1bbe102eafb13280df3f7f7b4df140f
:103c600008e11100f420da0cf614f5040807221d0f
:103c700002f8d0ecdd100403ec2cf004f8c3f006dd
:103c800000fe172012e7eefd4011f6e5ee08120add
:103c9000f5f6f5fdd4dc0c1afad6f7fc0403d809c6
:103ca00014fb0f2614cdfe0239ff090ce40913dec4
:103cb0000a0249fcf6fcfafa0b02f2dd0d0df502e0
:103cc0000a09fd00131c04f823fb0fe5dee0f4f302
:103cd000d00938f1e2e20f11f5e9eff60bf8f7fa47
:103ce000f9f70910e80522082dde0001f1f0f0f8df
:103cf0000c18181903f5f102cc2fe7c8fd20fae5de
:103d0000f407f8d908d4330b47f515f9f80dea098b
:103d100003e82733150803160228fdcb062ef2bf51
:103d2000f727ffbd10e43cf72425000dd9e809ee84
:103d300024d734f006ebf41c0313f3e7d912fcc6c6
:103d4000e8e517c5c9151fec101306dd04dc06eb0a
:103d500021d71c150ad8fa0eec21ebc7f927e4b1dc
:103d60002905d7bfda0039fdf8fd08d82700f5d6b8
:103d700012d9200124d6fc210e2ec4bdd7371aaa91
:103d800029f808adcd154d04112112fa0a0fe2d021
:103d9000fd0dfdf0faeaf3fd0e06dd1a0bc9e91080
:103da0002ced00faf914f7fb060704071cfa14fcc3
:103db000f8d9f7e9fdd12b0b0c08c3f8f3e6e7fbc4
:103dc0000be41704f018eb23e5110de70df510e7f0
:103dd000f7e7210103e6081810e6e01606e7cbe94d
:103de000100229f9fbf8ec130f07060d2f080de759
:103df000e3fc23d1f1ad041ffefaee1ee2fbe4e882
:103e000000003409c41300141df40cf41a1634f520
:103e100013bff705e4ec1609f220bd0cf7feccfb4e
:103e20000cf71efa20ff1410ff1eff16c9f902f34b
:103e300003d8060ed6dd2022fcebc600f70afe0be7
:103e400011fd1e0ef7e42b100f00ef11f61623e103
:103e50000ce402cce5c7f909e601d5fbe107da1667
:103e600009e70be2dbd10501081908eeedec2df0b6
:103e70000bdc02eee8cd1014f12bccd2e900f2ec11
:103e80000afa26e3eeec0312f80bf6dff6e01cdc90
:103e900009cdfef5e6baeff5d419efd8ea08e5e169
:103ea0001eeb20f5e4e309ee0704e1080aef0aef50
:103eb000ead00b21eadeeb02f202bce2e30f15b717
:103ec00009f929c3e5c801fc1c0bd2120a1ffcdb4f
:103ed000e8dd10f7e9eff3fe000bd6c1d819f5d1f4
:103ee00014e7f5c1e7e918fd1de6f1f0f50305e576
:103ef00013ab1204fbc900ffef0bb5e4e906fbe3cb
:103f000015caebc7d410f405f6e7f8f2341804e14b
:103f100001c20e000612f3ea002bcce0dc09dabd88
:103f200009f2eeb9dc0a06daec1311210a0e27eacf
:103f30000fd6221be3f6dfb90702e4ea10f107e926
:103f4000ece4e6e5070615eef8120a1f0c1c160055
:103f50001cc6fbe506ecda0ffb0203070407dd01d4
:103f6000fe080bf4040216e30615fc1f3410f90cce
:103f700003d0f3f7d103f8eb200306081712dee2b3
:103f800022e307d8ecf82be104ffdee3e91de5c9e5
:103f9000110c030c0f19e702f0cd091af5eaeef83f
:103fa000c9e20bfc0010e3fcf6e4e7d8061affdddb
:103fb0001edcf3dff5ebf0f6eb0404f0fad5ed19b7
:103fc000eeee0707dbe3fefbd8e91ad80ce4c8ca1b
:103fd000fef305f2eae1e419082b07e300d10b0731
:103fe000df0ce9dcf7fbe2f2d50bf1f4eff5e0d5fd
:103ff000fbf1efdd07fdf2140df1cdf80a01ddfb59
:1040000015d1d6eae0fcded2ec08fefa0dfee2b0f5
:10401000f400da9f25d9f3f215dcebefe0fffcdbcf
:1040200012f1f3f7d804faf4f201e2f61427e9bf2b
:10403000f4eac0ebeaf7e00a16df122513d3e91b16
:10404000fae7de141524fedc15f5dff403f2ededde
:10405000131500e0ee18e2c611c81018f2d906f5e3
:10406000ff10e423310ef0e00807f4080320e40712
:104070000bef0b23ef1eead924f3f3100d2de1fe15
:10408000ea15f40e23061d052afdfaf5f618db01e4
:104090000a26090a1e13e8e1f323121a0e0216ff7c
:1040a000f00eeb0529040ee713f1f3d8def3f91354
:1040b0003415021d163bdfe0db0611182d0e2d0313
:1040c000f61fc9fa0f10ffbdfcdce1cdd5cbf7fc24
:1040d0001f03fe1b1f17c3c2b011090d1512350bac
:1040e0009a28affb18eefcb60ce607d1e7cbe5103b
:1040f0000d090f2c1731e8dcb1f80cfd1a1111f481
:10410000ba27e2f118fe09cd0f9f2fe9d2f2cd1e9a
:104110000ff0f418250400ffcbe308ec3cfeeaf3b3
:10412000c019d9f229f3050209dc29d507f31a11c0
:10413000000205ff2026f81bc50c1e071f1906f3f9
:10414000de07f70001d20bf1f1d12024dad8f0e834
:10415000f01108f4ef1ae812f60df1f5fb290be562
:10416000d50806ee27e1fe05090f0e0fe9f6dde59d
:104170000d1201f531f11c1de2f0e001fc0a07f619
:10418000ea242501f6e7f80412a52b12f6ac142850
:10419000ed2423fe4a091718aa3f49e4252d4aeccd
:1041a000f3220f2d1ab21621e8cd2322f4bc0f16ec
:1041b000cff9f2241f110624cef40bec1c0326e9e0
:1041c000e12425f72bb1dc1fe8ed1626e3cf1ada40
:1041d000ed00f31a38f70713da15f7e427f23be19d
:1041e000e7f60fdb0ad7f716c9e81f1ff1e518003d
:1041f000051fec1c2feaf2f7ea0013f51fe31b0b77
:10420000df201f160deee837daf02317d9e7f5faad
:10421000f105daf915f4df003a0212030ee5160b88
:10422000e9fefe0607e1ee15e00c030601f3f3dc00
:10423000ed0bf0281f1be3f9e7eb06ff0be6200a66
:1042400014de12f422dce821f3e8f8e4d9da0f03f3
:10425000dc04fa21072f0dfbed06fd040def050d23
:10426000cde9f2f018ddf60cfbe81704c7a7200132
:10427000ee03ec30fffdf403d3faf01a1cfd10d46a
:10428000e615fcda22ccef16d8d911feefdb02f1ed
:104290009e1ae91d0f11e0ebd8f109e90d071cff8b
:1042a0000615161310dff50dc7ef03c6e0aff2d405
:1042b000cd02e51a0b0affe6e9f3fcf8fdde171163
:1042c000ff12f5f220e001eae1d9facaf5da12fab2
:1042d000f209d514f607edebe30ff8f109e3fceb77
:1042e000d20f06f20ab9f10009f1ff05081c14c942
:1042f000060afa09fe03cfc9fc0ef6f6fde012f637
:10430000d01c14060604e819fef0f3f4e3e400e21e
:104310000df6e30bf90adaf6f5f9f21f19ea0702ce
:1043200006f915fc25dbe510eee1f0f3dee00821ef
:104330000904ce37151ecde3cbfd1ce912ec1defb1
:10434000e21b110126c2f40be7e3f4ee24f2130b97
:10435000080aee50f02df3dbf0240c0611f111f6f3
:10436000d33125fa3ed7fdf5fae3fdfae3dd371642
:10437000f516e804fbfddfe5f11c0b1522fc090a2c
:10438000bc25ece10be6eaf329fc02f905cef500c9
:1043900013fffcfc1efae6db1022e3f3031bf20a18
:1043a0000bf005ebfdf92cebe7062002dd04fd0d1b
:1043b000fd06f219f6feeb0b05f6f5262a040115ab
:1043c000fc11ecf5ddf8010b10d90ce7cfdcebfab2
:1043d000f909f71a0df2f303c1ea2821f9011bffcd
:1043e000e025fef420ebff10f4ea13f3d3bdea2f2f
:1043f000f811f50be2171cebf9f729fbe8f211f8bd
:10440000c6eb07db04dbfa0a00dcdfeffe040d1964
:10441000e10015fe121efe14e0f2f5f5ecfeec16be
:10442000ecfe0202fb15e8fa08d9f4eee9f00bf411
:104430000910f105fef2feeee72100f6f41fe4d5c7
:10444000ea1fe8f013dbfef9ee0603f9e006100bb5
:10445000f2ee06ec2405fb0ae3e6f1d81013e00bbc
:1044600007010fff00ea10f6f4d9fa07e8f4cfe4e9
:10447000ed03fdfbfafc02fe02e2eee001f904e9c5
:10448000fefe10e906061515edf301fdd50227f62f
:10449000f102df0725f1f0eafe00dffdfde409eda2
:1044a000f2f1f2fe03dedc07eff8ea1601d9f5dae5
:1044b000f11704ffffe9fee80ffaf4080ce3eaf154
:1044c00029070113f8eaf1f0edec0d0d08ef05e412
:1044d000efee12f4fefcdcefe1e5fe081be9defd89
:1044e000c5f3f1f923e6e2f6eeff02071c070eed35
:1044f00004faf9030200fbe9151319071ff6f80681
:104500000519fd10fce2e7fb19eefb10141a00fc84
:104510000cf71501ee08e7e808fcdf0d1c01e6e7e3
:10452000e6f90405141202e1d6e7f6e6f5fce80523
:1045300003091c061deb1201053dd9e909160aed18
:10454000e8ff16d106d50616050628e2d9e708eddc
:10455000ec03f508f111eff308fa01f40c03190e5e
:10456000e5ef0a0906f7fd1b14f9e2ef24dd11fc63
:10457000d81a00dafbe901d4f7f2f1160de8fb0cca
:10458000d208dbf2fde505f909f9e451eeedf92079
:104590000e1afbe9e8d7fcfe02100dd8f6d3f4c4de
:1045a000fddf00fa09f00933df16e31a1306ec0dfc
:1045b00026d5e6d8150418040d09d908c7f3ec0a66
:1045c00014d2ff00e300fc1def1aee2cf70cf02dc7
:1045d000e4c6f119eefa1cf90f07d411e4f5f5075a
:1045e00014e214e4bfdef228e809db1604ee02341c
:1045f00001e9030cfaf311ed0a01e1eee909fe12fb
:10460000f2e313f2e5dde520d2fd0817f6220d33c3
:10461000f71cdcfbe30d0cf600f106edc90c09ee0e
:10462000ffe01fead5d7e323c31ff618d4fd101e01
:10463000cdeed9caddfb090104c0f4fcc0f7f30cd0
:1046400009d907f7cfedd015c809faedfff9141c09
:10465000f506dc07ecfb080605c00318c1de1be20b
:1046600026e4081ebdefd706d003fc0a0fe61202af
:10467000e618e6eaebfdff101ec50f07fcee0e156f
:104680000fd4f80ef123d827db26d82611191b0ae0
:10469000e31bddf8eefdf70118d9f718e6ee0a0a7c
:1046a0001fe018f5ddf8d70ecb061032fa0608fc2d
:1046b000d016c7f711f40108e1ca05fecae30703e3
:1046c00007031902ebf6f329b61a02320de8f21ebf
:1046d000dcf7d6e3e3f911f0ecbc1114f0e7021ead
:1046e0001bfb1211ee25b424c7101bf411fa33f48e
:1046f0000313d7e7fae806f61ce5e709e3dfff0056
:1047000005e9bb19e3f7d7e6d326fd15fcce010c6e
:10471000e216e4e4f5d8e8f310d4f7f006c60a2070
:1047200002f71720d1fcde20c6fdfa26eae8df09f1
:10473000ee01e0e5effb030d06f8163106bfdd28bc
:1047400006e709320ae9da38d905dd13e901e4fda3
:10475000f5f0b5d709f61be70ee906160dc5f22fe1
:10476000f6cbf705f90dd1fbecf3e224c2de2620ef
:1047700007eec014e7eed9dbffec15f90fdeee1003
:10478000fd0cff11f203e5f8fef9ed061a04e9c687
:10479000f5d9d2f8dcec26150bfce1fc04daec2ca4
:1047a0000dee01cefcf0d6f42b0d05010408f5f258
:1047b0000b06eefaefdefe0af50ac1ddf7e900f3bb
:1047c00007f612d7eceafde7fef621fef30e0aee3d
:1047d00000e3ddd4eaeb0a2b13e814ede20ee3ff6d
:1047e00001030ec8e727e3f5c90b2a072bfe08ffd4
:1047f000e7db05d8f7ac1a4201d90efff5fdffe45f
:10480000dddc19f9cdf5cb0cc4e011cd0d1e31e97d
:1048100019e304e3efc70d26dde3c500e4cfc5f9d6
:10482000eed01cf6fafd03251b260bf1fd020dc58b
:10483000cbff18e7c1c71228ffd9abe3280be1f47f
:10484000f41c15f6f9ea36fe0204011e16e20bde30
:10485000bded00e71acc03fee1f8ecd4140ceaf04d
:10486000180527ded6fc20fd090b14eefbae24ea6a
:10487000d3b20e17fcc11d1ef531d7cff608dce60a
:10488000340534d6e4fa071dff21f7d415ec0ad21b
:1048900002b7fafbfaaa0df7d51bcde7e9fbe1d683
:1048a000f7e301c0f4dc10fe06f4deed300af0e9b7
:1048b00001d71bfbd7e5f8060d10d6e0eaf602e3b8
:1048c0001ee0e4bcd9d120e91deeb61b2e1ec6f1b8
:1048d0000bd80c1ae8fbdfc21020cecbdc24ddbaeb
:1048e000f6f2c098e6f709fafa17bb1e2408ece9bd
:1048f00027b006e2f3bbe4e6f80ab6d4f923dbe31b
:10490000d5d1f2d0ebfd0c02e5fbdbfd212ddef570
:1049100013daed19e41ce4dd033e09c6faf0d8d041
:10492000f5eac1c1f32b01d8e81ce2e9e10d30e161
:104930000ddbedd6feeed8d4000fcf0bd3f6f6e1ab
:1049400000baeceae1f6d7fbd8f81304182906fe02
:1049500024d8dcf700c7f7f40107eb19ede1e7e62f
:10496000020cf018ee08e6fcfef5fb1620f7d12b42
:1049700011f4c406b630f909dfebf102f5fdd907f1
:1049800025f92fd9ea0d02fcf21ee5353119f7d6cb
:104990000803da16f2f13105150bbeffeed4e1166d
:1049a00023b833030b08fa231b1b1b051711dd0863
:1049b00020efe8f7f100452a0c02de1af6e7c60cf4
:1049c00023f42ce0e1ffe34bf70c04081808270f51
:1049d000f4fd01eb0bf25d15fceaf310e70809f6b4
:1049e0002bed15e3c4f8043123fdf80311f323087c
:1049f000efff15e9dfcb2708edfc05ffd8f30df835
:104a00001fc02511e40d0726f9fafef22027161320
:104a1000d3f303fac7f01c1af3f8da0fce03de0063
:104a200004e10f20e2071121f010ee0cde04fbf888
:104a3000d60011cdc9fa37f7f6e4d502e2fd114fe1
:104a40000bf52c31f3010d39f7e9073009fa11fca8
:104a5000f30ef9edeadaf70ef50a0c02c4f823209a
:104a600011de1d19e9ea0807e801f6ec0005f60178
:104a7000e6fafcf7dddf09fc17010e0de9f4ff0e85
:104a8000f9e7f11cf90807161412e5e1200213e614
:104a900006ee0ceae600f5c123ed001ae0f4f0188a
:104aa0001ef4dff2cfef0ce80609e6d8201817eb6a
:104ab000f7daffe7e0edcbe4ff060d12fb00051689
:104ac00022f3da07e5d2fa121724ddf82126f8f7e7
:104ad00010e216ddf3f4d2e308f5f9fdfcfaf6e98d
:104ae00001ece70af4f210e7fa06d8fb06e4f8e86e
:104af00002aa14f0f1ead2e404f0ac06da06f3fb01
:104b000004e8d6ee0af5fbe3081fce25ef12fff00e
:104b100008eaf7e5daefc4ee1406e004d0fc061567
:104b20000dcbd3dfbc0414dadffe17f3ecee21f378
:104b300022f6f3ede7f4e2e31308cf0910ddffe41a
:104b4000110103d8f000f70bee13d2200c33e5155a
:104b500040fd0bedf80adbe613f1f7fb07f2fada9a
:104b6000fef501e21813f212def90ff21816d9154c
:104b700001f1e61ae426deee370df5ed20dadbe58d
:104b80000be9eef1e702da082516afe8dd07122897
:104b9000ebe20c0cba27d8cc0f05dd08f916ba0fda
:104ba000fc119e05fc3c0ce926ffb4e1f9171fff40
:104bb000f2f62f20b81ababbff040113fc1c0f0732
:104bc000060acf2605093ab807f904d4ecefef1a24
:104bd000e510fd14ce1cd4c801fb440108272710a2
:104be0000a1acd0b0e32fac620c51cdbd3fcea191b
:104bf0000d07ffe20226fbcd08fe3c13ff15eef881
:104c0000050ed4f10c0712e617ea069cbbc0f21b96
:104c100025fb251a121210ecd7290e39100f0af5b0
:104c2000bc08c7e214060ac426fd16e49dd9f13a71
:104c3000f52510060eebe8ebdcf62c15090507e66a
:104c4000e618f2fe1207fbe10c032af00106eb095d
:104c5000260009131d0cfa05e82217fc030508f2cb
:104c6000b10ef4f50fef01f9000713ed3625d2f977
:104c700019f501f71c01f723010e08f90108111bb2
:104c8000f201d6fb1e1a09ebf50f1beceb0cd01052
:104c9000160f0ce60d000b2af3fcea17e914f707d0
:104ca000cd0ad2f2eb301af7fe03f80be3e5e30f7f
:104cb0000afb0fc1f9fc15131de70208dee7ed0939
:104cc00004eafeebc4390a05fa120e0102edbffe3a
:104cd0000f05ebe2ede0101900d718ff070bd71e08
:104ce0001ce2102c0e02fa21f514f407f21000dd7c
:104cf0002d1ee6bdfec51e1705eb120dcae12112e1
:104d0000e2de2e1ec203f714cb10cb07f5f5fae155
:104d1000edf6e5beb7bae0f005d7f912c3e5df243a
:104d2000f1afbd0ae6f701f5f30cd5f70d12ddd3af
:104d300008ccf1f3c5dedfef08f3da0fc7e7b320e5
:104d400018d3b8f9dd0bd2e5f815d6dafffb09df89
:104d5000f2d1d9accb01e1dbf3ffd1cdd7d3c6ea99
:104d600007e1c1e2d400f0f4be0cdc1ad6f7a909c1
:104d70000fd3dbf4c608d4ebead7cec8f4bde6fe09
:104d8000fae7fcf3fa00c5f303fbc0f81007fac416
:104d9000dde7dbe2e308d6ec08e7e22fc1c1b600ad
:104da00001c9c4fce71cdedfe6f8a7f608ec01d376
:104db000ddfadcbeb5f3d0ba09f10afcddf2ed2d67
:104dc00001dfb71fe10ef1d7f0eea4ec0ffcdfe836
:104dd00032be0c01a617acd50c00e9f9f5f8e9eaea
:104de00003f9a631f41500ce1618c7f3f80ec5f274
:104df00023e7070ce812c4c111061207f112ded630
:104e0000020cc20516070fc22afbcce1ddc1f3eb91
:104e10001120231df117e1e712ffdf23f802e01153
:104e20000a31cb190005fde839ecc6ebdf13f211ae
:104e300011f70cfaef15c5ca1a1413ed141100fb83
:104e4000f90ed1012b240ddb0dfa05bfda13f70f94
:104e500013030f19fc25ead222ee0a1d0d142bfbb9
:104e60000021e41d0b0607de0bf0f1ebbdfbfe0994
:104e70000d0e140ced12f6d1cc0019fe291411f010
:104e8000b521dcf11cd1ece109c51da7c4dbe407a9
:104e9000061305e637200ff4cbfc20c3250513d7f6
:104ea0008f2ac4eee5caffd30bbb2108dfcfeff298
:104eb000090a0dd1310b01180508ffef1616fad7b4
:104ec000d50cf2080702fc0909dd15c91af405e43e
:104ed000f5da0e0604ed1320df0ef9d8210500cf18
:104ee000f70300fceeca00fefaed00e8eefe101a31
:104ef000f310dff50c041e38df0e09e002fe0b0094
:104f0000dbfff617dfe50b04d0ceedcbf50821ff74
:104f1000e6f9e2c0e900222e10ec2605fdf3ff14ad
:104f2000f3d3d42adb0602e7f301f1f31e04dbef2f
:104f30001101ecdcfc051b22fe120df2f601020d44
:104f40001ee1f40bb814efdff304fef90905e9df05
:104f5000d4decbdddce7e9f801edf424d0aabf1004
:104f600028ccefeec60becf6f10fbfda1213d9e442
:104f7000eebdb6e9d0f5dcf416cfc9c8edbea7f496
:104f80001dc512fef7e7d30d1810b8d9f5f519179e
:104f9000f5e0161bda1dd6def3fee203ef44cd0b7f
:104fa000e50fc4f60d0729f91bfcd4cf0f0a12191f
:104fb00005e12c12ae2dc1e9071715e1fa15040f12
:104fc000fd09d00efbf72cc7ff01ebcc16f50bf754
:104fd000080de719e612cdd21e0e3d1c061707f785
:104fe000eb00e3130f0803dffdf20ae4e713de171b
:104ff000021ffd082025dfd71d063afc081af10b19
:10500000d524f21306ec05e80b06fffbf4eaff1ac1
:105010001c000ae1fb320edffe264025fe0e1bebd4
:10502000ea02ea10ea01fc061d1e0419e200e52c62
:10503000001a0afc10130f0301f42417fef80af6f5
:10504000fb13090822e60c1202091f27e0f9de3bd8
:10505000d817fd072b1a0012f4f42a250e0f29fe8b
:10506000f301140bd8f7f620fded220af302c90173
:10507000110f07df0c080617080714f912f0f21acf
:10508000fd06f8021603f41808fc1bdacee2de0374
:10509000fb2601b815f5040eeafd070702e900f743
:1050a000c401e3fddd14fcf5c8f9f5efcecce30f48
:1050b000fb06d7f1fcf8080b22f1020d01ebfe19fb
:1050c000ddf3de1de63fd300c3171aede8e2c61696
:1050d0000f16e60ceb0734f10cd41e2309e1d81ba4
:1050e00003e81e22111df403d6210503daf4ea1e9b
:1050f0001305cee500e6071e29f70a27e8e7fa2997
:10510000e7d6ff1bd6faed1eeefdfc07fdfa1601f1
:10511000f8f6c9c612d1021122f00324b4dae94b21
:10512000e98b051bdafed608ea18efda01f2cdc6e4
:10513000efe6d8e4f7f4f021ffeee717edd2d11b4c
:105140000eb9e70fe715d9caebf6c2f9fafdf7da9f
:10515000e2eff1c5b4fce50c02e7eff9dfd5fbf3b4
:1051600008e5d803cdf8ecf4f203d3fde4f8d5f765
:10517000faf2ef16f40cd8e001d5e2e8dec0e20066
:1051800003e7cce627fabbfd0820c1ed070dec0bc9
:10519000f8baecfae006001407fcea19dc139d32b9
:1051a0000cead2eec943d5010e15d8eff01b3cf343
:1051b00007ee0e0bdd05eef814e5f2161230c4f41e
:1051c000faf1fafafb2310fc2ae605cbeff6fefe15
:1051d0000cfa2a07ba29ed05f4022019f82cf92750
:1051e000eceee220090d11eb18ec19dbe41803fae0
:1051f000fe0726031010f8fc08032b233128e30bcd
:10520000fd1cdb02ed0614e72fee01c601cb0f20db
:1052100018133b15f70c0703eb2b1e16202bf1067a
:10522000ff08d8f2f8050bcb1a000de0edd9f21407
:105230001f1e15ee04dee7ffd12e19fb0930f7f132
:10524000041df5f0011325e417ee1dc4f7f4000268
:105250000eff1a10161200fbca1622eb0d1ef2d812
:105260000d01f7f10eea18e724ea18e4f920fb0231
:105270000cef35f1fff42027f708e5feed140500eb
:10528000e4f4dff50a0b0af60516f8d1f718e8e89a
:1052900003ff1ae707f6202612e6f8fd192305f1a9
:1052a000c004e8eae3190cfb2904f3ed120ede0852
:1052b000e7eb29c0f2f10804f7fc00e7ee05e6fb96
:1052c00006eafc10db2a02e71c0efae40622c31fe2
:1052d00025e6fcf5dbff091201fcf1fff1fcfd0bfb
:1052e0000fe916070af20104fd34e5f107041af686
:1052f00027fee7f403c41118ff08f7faffe40202df
:10530000fcf6140be00d00030710d403012521f275
:10531000f4cc04c0dacaec1606f6e5fcdcebdbf9eb
:10532000fbc7ffebe8ff18f8f80bbc061128d4bb4d
:105330000ddcefe4a6dcef0c22f5ee18c1f1c6e9b6
:10534000f0dfefde022219eb1000cae4e1f811d918
:1053500003d2fbc8dcf0fe0d1bf4ea03e4f2d2e555
:105360000efec8f3d5fae3fcf505cf0ce3efbc0164
:105370001dc7f1f6d5faf9e803f7ced2c5e0c8d5d6
:10538000fadcf9e90d02d30f2fff1bb8eb020ee98f
:10539000f32234ff3302f534e5ea191afd26160f1d
:1053a000ca23ea0bf21812d025030ae7e6fb09ce5e
:1053b000111afa18f20ad0fdf5eeed0c3324122082
:1053c000fa26fa01280d11c4060422e5e9efff05cb
:1053d0002506fa0707f8bbd709f1000a171402fce3
:1053e000e601c6091c1020df1de508fafbf4d6f51e
:1053f000fcff1123192ce803edfd08f81df80fe65a
:10540000f328df00361105ef2af113fbfe14c3e386
:10541000111b0c182911fbf70a0210f0300015d3ec
:10542000da28da00412508e73c0409fffd00f2fd17
:10543000e51216251915ddfbdb2112033015fee7f9
:10544000e8050be431fa20e911ebfb0203f4eaf181
:10545000100f0b3b0c0af3feea22fde3171b13fbb4
:10546000d91a1aeb29f11b0512f40edaed1ae7012d
:10547000050e0e2243f2e805d2f702e22b0706d60c
:105480000200e9f51ce90ae31bf81afede10e5e06c
:105490001006f6001af0ee0202290cf841ed0305a1
:1054a000f130050534090be6fff913e2d7e0edfa18
:1054b000160dff3e1429e8fef92b07f13210f7090b
:1054c000e127e21e2f2f00d118e214d3e8daf3f21d
:1054d0001109ff35081400f9ef050c09240810fc28
:1054e000cf1ff5f4210622ee0b0707eada0e1ae6c3
:1054f00014ed06240811f10de2f913f61efffc0e5f
:10550000df35e702f30919f8f10903db101e19ef83
:10551000150c0ef5effdf0f3fe1318e3221effe36a
:10552000f12b10dd272a0def02f12cdd210d0f08e4
:1055300003e9141331feee14de01f7fd121314f427
:105540000b23f1e5180ef6d9eef130e5070719f453
:10555000e3171f301f00ce15f2fcf9f937f91aecea
:10556000063f04e50eec0bf719de07e924e8f3fd2e
:10557000060f2b061ff51201e50a13edf6140516aa
:105580000a1a1cfc10041ae102f70ed0052318d9e0
:10559000f50c27dc100bc9111b04f9342c1c081264
:1055a000e60bca03010709c707f9fff9e802f6f29b
:1055b000180bf421d109a1c808f1e7f32b13f21e4f
:1055c000f30fc80a3df5e7a71110f3e003f6c8f59d
:1055d0002eeb030f1713adcd2a11fefa100df903b0
:1055e000f320c9e841ed03c5fa0503f2da19dedb61
:1055f00010fafc22104dafb408ee12fbf80b05f5c3
:10560000f429ba01380404be04fb00f4e104e40404
:10561000fe1e09190e0ebfd60f1405022c0b00003a
:10562000e631f5f107f7fbd508eb0ce8e206ce080a
:10563000192e110b1411d8cceaf51f1024ea17f516
:10564000fb11d9ea4811fcbaf1e40df8d0e5e5f315
:10565000de34fe261c1ff0c5021213031f0d0ddfe2
:10566000dd23e2f527f50ce806e507f4f7ecdf07a4
:10567000d21717ff4806e9e3f8e21606310a20e1df
:10568000d4fcbd0c1bdcedc6fac1ebcef201e40b81
:10569000f512fe063625dce6b80011f62218fbf7f7
:1056a000ce19e7f134de06db0cc60702d4c4f00cd9
:1056b0001d0a11140831f3f7ed1c0cf714f604055c
:1056c000e427d003390807da28d90ed8e8cdfa1232
:1056d0002109ff37180beae00b11070d1c0d0ae931
:1056e000c722cd012bfd00d1f8f90ebfe00ee1215c
:1056f000080bfb25101df6ebf1f70417200be90250
:10570000eefc03f81ff00cddfeda14d508eaf42aeb
:10571000fd13f7271d22f5fc010202ee3d0af1e51b
:10572000f021f6e93704fafc0eed39c80909120236
:1057300003f40017123fd7f6fa1b0c0522fe1be4f8
:105740001b440ce6140006e7060035e4f4f30509f3
:10575000e3200c350c14dd2ff81109111a14130174
:105760001c36f7d5240ffc0a071e3b11def4e40fac
:10577000eed503e822db200df6f002e30df12af06e
:10578000050e0004e4e9fdddfb2de82d191507f7f2
:1057900004f2f212ca092e0517ebe71b05edd91822
:1057a0001df21bfa040fe1351517f3071a0800164e
:1057b000f40b2ddde8f014ef0ef61713e5f4f016f8
:1057c00029fd091efa3d06292009e6041c171705c4
:1057d000f5f93001ca15121225ed1419e6f5dc1a97
:1057e0000f07141ef021fc132bfdf8f51f290b16d3
:1057f00019f319f7bdeb1b192b10091eeb12f6f26a
:1058000023f6ef18fc210dff0826fddd1e1ffbdb34
:1058100010fbf1f0eb011c0830f8ff110009132711
:1058200024111c0ce1212911001c08f5e5f9eddf1c
:105830003506f0d2cbf62a1b102303faf617150211
:1058400024fff914ff2012f3f0360623f51a12266e
:105850001c12f4ccf6e71d0819171c16ee04fe16f0
:1058600014ee1029dc14130b070bf6eb0506ef0002
:1058700028ea15f207ea23012203030dd1f10c18df
:1058800000e30612ec30111e16150a172b2efe002f
:105890002af018f6ec0d071f18fc18edcb0df90acd
:1058a0000ad5fdf8e32919141417e01d3a43f6163a
:1058b00004e405f4ea08081efcf7fc14d80ee7021d
:1058c00014ed0a10c907fa271716f6f5041cf21c86
:1058d000f8f81cf70bf0171629f60015f01de1215a
:1058e00025dd2521e11e07350422e11b0d1ffbffed
:1058f000f20e2ac4e1e315082ef9fd03f804f1f4d1
:1059000028f6ffefe62cf6282e1e090c0c17fe03d6
:105910000be936d8f2ee15311b08e6fad108e1039f
:1059200022f50cdfd9122317101d16271808ecf4e6
:10593000f1e710efd8de2e2b22f8d414f10de5e3b9
:105940001ae51019d0340f090e2ce42c022fe109ae
:105950002cbc30e7ffe6091e1e02f11ce011d0024c
:105960002ccb021cf43011ff14100a3317fed90c93
:1059700011ddeff9e806140618faf40dca2e051722
:1059800018c008e5e3150319f01f0bf0241ed7ce4d
:1059900007efc916f4f3181a04f9c002f5d6b707d1
:1059a0000aba19e6fcf9cf000b092c1117fde4ee39
:1059b000f6f80fe2fffa2e21020ce7fffef2ebfdf4
:1059c00014df13fde5d50e0f00f10be402fdf1f538
:1059d000fcf218b514cd2f15f4fae906bd01f5d384
:1059e000f1fdf9f3e8011114190d07e9100ef8e5be
:1059f000f2d230e7e8bd130ff8f6e0effffde8e57f
:105a0000180220f6f1eb0e0d110df0081e0a13e33b
:105a10000ec602fef1cf1b0cfe14b202dd04d6f955
:105a200015d313f7f8052dfafe110efdf5ef05d588
:105a3000e7ba18eadeb1fb1f020eb0f1fc20fedd72
:105a400013051bced7ce231cfef0051fefec1dfd6a
:105a50000add07e602c70819d91cc2dedc07e2c866
:105a60001fe615bad4bc0c0c00ee04e9f7f619e8f1
:105a70000bc0fafbe9d30508e920ebd0c209fed937
:105a800018fa13eaf7f90c17fb010de7470b20c9c9
:105a9000f7e4f002eed0f20fd916f511ddfaedefd2
:105aa0002ef213ebe7f20d0ff503decd233515fbd8
:105ab00001c91311e1f7faeed700c4fadf1104d3dc
:105ac00028f2d9f5c7df11e124fac4021b1fceec7e
:105ad000cadc04fcdbfdd4cfff05e5f0e414e5c22d
:105ae00005ffdcd0de0d1ce712f6d2051ef1e5ca7b
:105af00018ac13f1ffb9d1f40d15aff2d217eed1f6
:105b0000e4fbeac7df2719f1fe1abef6fa41ebe41f
:105b100011c00001fffdf1e8e916dde6edfed1e57b
:105b2000f7ee08c9dd160efbe50dee150ff928efaf
:105b3000fdf8da0408ecd0ccfa15d7ef0cd9eadb83
:105b4000f7d4ebcdef20dfe7e712e72efb15d9ef17
:105b50001beae9dd1edcd810070306fe04daffdbd2
:105b6000fd08efef0e0cfcf6180aef0e0f01f52101
:105b70000107fcfcd622ddf914f4fc1c0508d6df75
:105b800017f714e90a0ef2050809ee2afe032011a0
:105b90001c08d8f0feea04f22032eedf0ae7130117
:105ba000ffe1e3de0a0a1deafe33ee07020fdb0a1d
:105bb0002000eaef02daf7f1262c1b0ef0070f1493
:105bc00024ed02fbe80bd3e9e7f2eb40d807dd0d4b
:105bd00011c0e4060e2418ef02f4eae607f9bde46a
:105be00037ec0fd80af1ef34fa0fd81709ec07e6b3
:105bf00021e3e7eaf426feff1822dbdde5f505b533
:105c00000fe618bedef1e012ea1b02171c00ff12bd
:105c100009fbecf5fb2613f6fce0f5c7e4eef4df38
:105c200010ef10c1d3e9cd24ceebfd1f08cd09093b
:105c3000bddcddf4e2051a00d1c4d4c3d1060dc029
:105c4000f6d919d2d2e4d5fdc4120d18d0ec1f2c10
:105c5000eef3d6fdf8fe110be9d3eafbcecd11da57
:105c60001fd9f208efc2cfedeaf3ff14e8e0012eee
:105c7000cc0acdd1fc250a02e4ce0910e6eefceafe
:105c8000fd0823f7e909d21ad7eef4de0df71b1849
:105c9000f905d4f2de11fe16dfd0f909dfee180c9b
:105ca00015cc0003e41af103d809ece822321627d8
:105cb000090ffcece3d606080bb71406e2d6f71d75
:105cc000f7d5d70bf3e8eaf8dbf8fe161c2a13d257
:105cd000d41ad8df0000daede4bc070ff6e80d1b9c
:105ce0003af9f30afa10c9f4caeb0e1be213e20305
:105cf000d20bbe1bfb07f9dde2a40e13f7b412149e
:105d0000ffee2618e4ebda2dd8fcee10bcbfe6f26d
:105d1000e50be3fe1c150b0ef9d30e2bedbff62e93
:105d200009acf118ffcddd1ddafcf713e5da0b1d28
:105d3000b2f1e712f0fae9e81ef0f62216e1da19fc
:105d4000ff28ef2b16f3ee09ddf9e81305d6c1f7ae
:105d5000e20a0c3bfcf3e7f5180608090815121ccb
:105d6000d7dcfd0f0a051513d917181cdbe5fd1c40
:105d7000ff0bed081eefe100e1ddfff114d9f0fbb0
:105d800001fe20ea0e12e312f8f1d3cefbfce8eaa2
:105d9000031204f2ef0702051cdf3425edfc06e7d1
:105da000dd1109fd281ce2e7f4cb09ecdd05dcf090
:105db000121316f6d6e5dfe005fe18f2d7cae1fcad
:105dc000e7cbe804dce506d6d1ee0bf7ef12b8d747
:105dd0002aef01b6ecc3e1f402dfe7daece4cddb55
:105de000d8be28ebca12fd18d0eee1ee18e2a9e603
:105df000f2c9ceb6ecf7e8250fe9fbefe5e6cbec10
:105e000004b8f8f0d90903f6d210e00ff42802d450
:105e100003e6e4c0e3eeebf2f5bfe6f6eef50703ca
:105e200012f1f8fdcc17f309de0bc5cf210702d91b
:105e300001c0e6d4c22afcf2f5dbd90ad1edc91db6
:105e40000dd3d629da0acdd50d22c6eb1cfd0cc523
:105e50001ef1f109de01bfd112ecf608e30a01c719
:105e60000500d61304fee9d5f418f617f927e2f277
:105e7000ec1b02fdbd13d1d4160af5f7f6fd24fd87
:105e80000a00c41e10090ad40c03d7f501f5fa0b59
:105e90002cf40b19da14e8cf14e50f110cfc131fc6
:105ea000dd18c40b3e20fbe2101be5ee0e1dfd1fae
:105eb00007140ee5df20e9d006f533120d071413a1
:105ec000ed2bbe1b29e704db011ae3e1dc17061307
:105ed000e8141705110ce2d00ffb1b14ff2200d2af
:105ee000e00fc3ddff320fb20ef5fa1ee8e5012721
:105ef00007e9090c0e2b0eeac2f30d110c1af61667
:105f0000fa08d6de15f813dcffcc21f3e707e10c25
:105f1000fc1b11052dfe0af6d2032cd10700f1fb64
:105f2000c510fc01f6ef0701f9e707f0e10ce30506
:105f3000f61c00cf0cff0d11ce0b0de62a04feed72
:105f4000d70ee8ec0ef701e1f6f609f60b04d7cb15
:105f5000c518f9e823e8fa20f0191624fc09ff1106
:105f6000ff12ea1af722fafdfbfb0c05f228e5d531
:105f7000ebfcf8e21217fb35f8d50509f3f2f70b45
:105f8000f7ea1b12e31ef918d1290cf7261f28dea9
:105f90001cf1cc050ee63d310a03f4fef1d2ee0e03
:105fa00025ed14f4f0f8f107022a33fff405fbeabb
:105fb00027f0fc10f0002f2612fad000e6fbcad121
:105fc00003dd1acf0208d418eaf70cfaf9f51d1907
:105fd000f4df36dd12ef1102e9d6f508fd01f10c10
:105fe0000ceb2210e30c1b1ef6f015f2f5e108f89d
:105ff000d8d905e302af293ed5eef9fcf2100bf437
:106000000ce81c0ee5df161d0df0fa06090d01f176
:10601000ebca16fbdae61e33f700e0f3f01dd8ee0c
:1060200026ee210c14e1160c04e2ecdd13f00ee177
:106030001dc90efeb8db03f0ff16ead6ed1e0acf2f
:106040000b07eac7efd61f1e050000f811043ae55a
:106050001fe811e2f7daf4e4eb1ddd0b061d01e0a9
:1060600005fed4deea0d0bef0ef0e30307ef12f1ad
:10607000fbf6020af9dbfbddff02dde5e60c15e1cc
:10608000f4e8d2dee1f509d102f5edf91d17dfdc08
:10609000f3c2f90dfbf1ceecfdfad3e9c20f1efeff
:1060a00016d4d0ece4fa16f108fbd2ed4b0911d36b
:1060b0002ad4ecfadbf2cbde0316cc1de5fce5e3db
:1060c0002f0cdfa3e4fe08e9fcece80e230e07f139
:1060d00013ead9eacaf30bfb130adde9faf3f1d3a9
:1060e000fbd00402d8cff711dc0a01e51220dff45f
:1060f000f8b5ec2debe21106121fe2de070cccef37
:1061000004dd11d3fc0ec5f2b20f17e5fdf0e9f77f
:10611000dde1f6fd10f72b10de0ffeeee7c8e6db43
:1061200016e514cecefcd7f1e00f04ef08144ae3d5
:106130001bf4d2f8dcee2c19f91ad6f406f4feddc5
:10614000d0d924ff0d06de23fe01fa34f5051de744
:1061500002fd01110901240606e6f8341edb1210c7
:10616000eafd1c060ce0f5243ffcded61310030408
:106170001b44411b0312e8da1114f02a0d1c0e1403
:10618000e815ec00dfef0cda0609ec20f0fc193d15
:106190000b09ddfb1e0519e1172810e3e30d1ae4d6
:1061a000030810f814ef142af62e0dfa02eeca3482
:1061b0001efceff90b1318e9fd0c01e6f2edf702f6
:1061c0000fdcfef4fb0f0326d8ee0c2600e1220aba
:1061d000f8f6ed190923231cf1e5edd7ebf016eee7
:1061e00011d609d909eb0213e60afc0e0ef10922b9
:1061f0000323f8efd6161ef7e102f301c5ee0f00f8
:10620000f6fa142004dae517f412ed2402df100f79
:10621000da01cfe6f123fe0412ca2afce2de0b0605
:1062200005ce1434d9e0c613b6fae92e08de1830cc
:10623000ec11d5ecec0909e80abaeb09c7e4040350
:106240000fd9081ccef4c70ac80de51f1002150aa5
:106250000104d9e9f9f505fb0bd71022c9e3071da5
:10626000fabc160ee7e8b804d1fd01142315f62098
:10627000f5fbe2fccc0a19fa1ebef305f8fd0b2f64
:10628000ecf01d02d321d921d60cd71af2e0071b5e
:10629000edfbf207d50afff326d41008e3f006055c
:1062a00000bd07fe1001d725cf0de724e71006310a
:1062b000db1adafdf8150201fdd3fc10d1f919162d
:1062c0000be2fd14c5e9cb38a1fb002ae8e8212147
:1062d000f60ff9c308e911f500e112f9dc061724fd
:1062e00018010f08fb19d819c51206231ed205067e
:1062f000e513d2f6ebd717f209e6f9340ff224ffd3
:106300000be90118fc15d5f1c9060c05d2e60e10f3
:10631000e21fe4d9f6f904100acbee1ad9c322150c
:106320001bdffb2affffb1f3b7f0ef26fdebe627fb
:10633000f10ab0efe60011f40eeaf92c0dd4f026c4
:106340001bdb2322ed00cd39eff4ea1706ebe80c56
:1063500003f9b6e2cc150df415e72a20ffbefa22a8
:10636000faded82b0007cb08dbff060fdcf30300b7
:10637000fe13cff5efe6fa0c0aca0d2607d7e5089b
:1063800009deec1e0406e12aeb07c203f60deec29d
:10639000e9f2f1fddfd8fe0424baf404b9cdc13d21
:1063a0001dcff5fba720a7f4d90feb07e2f1fee91b
:1063b000ffe8dcd6cfe4e8fb10d9fbfde2e0d20732
:1063c00004c9fe0a0119eaeff1fcdd07fa08e7d972
:1063d000e0f3f1f6c6c3fffb110decc5f006d3e602
:1063e000fb00fa10c509030b1013eefe0e0df0d2e0
:1063f0000ad20bede7ddee120cf1cff3f3f5d9e69f
:1064000001e2f4fdeaf5f9ed1eeeebe8ea100cf717
:106410001df229f5f0f30efbe7dfde20faffd11fb6
:10642000f7200c220e26e502eef50bee27060d08ee
:106430002411330ae10d0bef0de4f9f9072ae314f7
:10644000151dfa290d1307f212e206f81411110ea8
:10645000fff12af103fce70007111500182200fbe9
:10646000fb0f07ed140a15ec1b0814fee0f229f0ef
:10647000f20a1307fa0cf412f90c07dbfe15f6f614
:10648000f7fcf6ec0df928f81efc11e4fbeafff12d
:10649000f6fc21f50aee0417dd1f0ad6031b04e5fe
:1064a000fb07f5e7e7ea1cf11bfb0bda26faf9df3d
:1064b000ffec2dea0fdf04021735f1e8e91a02ecd0
:1064c000fd050ff9050d1de53efcf7e9e4eef4eee0
:1064d0001bf0300c0bd3fcfd070bf9f0ee18e8e4d1
:1064e000ee04f3d8dbe32d040810fdfe130f0be1df
:1064f00028eb2803eee6fc0efb0affe9060d03de9f
:10650000faf6f2f7fdf237e947f400e11234f4f459
:1065100013f442d4e4f5e0f4f81200ecfe20fbf1b1
:106520000afdf7e6d7172dec3bf821e7f815d41054
:106530001fff1ade04d1f3fdfc340b07e21dfeec55
:106540000ef7e2e8dd1a0de90900f603e40b03e7b4
:106550000ce922d91dcffcf403fbff05e309e1059b
:1065600006cfcaebe41a10f00b1cf209421edb0442
:1065700009aef7f3f715ec1f0e3af3fcc8f2ccf6b0
:1065800020b52906e1fc160bf713f32dd1f4eb0d22
:106590000ee3ead8f7d929eaeb35e4d2c60dea0cc6
:1065a00012f313fa0b032efdf803ed080f0c34e180
:1065b000efdfe1020a20e9fadf0f0cebf8f6022622
:1065c0000f2d1f2bfb1dfffadef5cb1b0c0ef62348
:1065d000181bc201dd180a20de0a193324d3183d26
:1065e00006f4f1072914f6e5e018d0060610e9e3f1
:1065f0002213dee5f2f7e6e20814e03014ecf211c3
:106600000b14fc0dd11b00feebf0dd0501fde7dafc
:106610000fdec8ef04dfe5fcef2be7e429d0d2154d
:106620001de6010200f1f13dfce8d444d6f4f6e4a5
:106630001ef9d0df03ddefecfc01d1f5c6e3d60c8b
:10664000f0e610e4dafff11ae212f5eefa15ebedde
:1066500021abd917f20c2a18f9f0d41eeef1b7f6d7
:106660001bf3f1d8fb06c830e803fdea37164d17d7
:1066700001d6dd07f70a041208e1f106c1e0ed1fbb
:1066800022d31f05c709c20eda22f4ff26124f02d9
:1066900009b9feefd3ef130efedbe9dacbf6cae55c
:1066a00028c84ad4d7edd3210e1901222725380551
:1066b00001f51dfadbc8271e26dacfc3dfeee0dfc7
:1066c00024db3deed61003540f2c193126ff351c68
:1066d000e2e312e9fbeb2334e7def1cce106f0f470
:1066e0004afc4c00eff31657f7e10b2225f7232263
:1066f000d1f81fd2eaec380d0903f6f7eff6fe13d6
:1067000014e11007d7241a210e09f1472ef6251699
:10671000e60e0fbfd2001200fe04012ccc03f61ec1
:10672000ffe33a29c7d820250c26ff17fbcd0c061e
:10673000e1fe07e9cc060defdf01031bdc0a140db7
:106740001aec1f0af902211406f1d32ffeddf233f1
:106750001efa00dbf712e5e0e2f52702e61b130a5a
:1067600004c2e707f40604ea0319ef3dddef12fd6a
:10677000faf2fee8e5ea03de08f71701ef1a040f64
:106780001efe1cfdf7270cdbe82727f61c25dee89c
:1067900013f2c7f120d0132c17dbcc1fefb6def8b5
:1067a0001bd21109f5f5cc18120a16f21ff61ffcc0
:1067b000130a2304efe8341003ece41e14e0ceefd8
:1067c00003ed2606f4df01fe273115fedd07150374
:1067d00004061fdaf1e713ff0af7fb00f314e3e8fe
:1067e00015e711f6f4e319162400170de8dee6fab2
:1067f000e6db08f1f0ad1e0e1219d7eaec1dd7e862
:10680000f7dd26e4e8e1150a1dee0c180deaf70a9b
:10681000d6de05e7efb1172cd709d9e7ef23d7f27a
:106820001bf0230fefec1a06f9f205e417e90fdf6e
:1068300013c506f1e3d705faed15f4d9d110e3d36a
:10684000e30604cae6c717e70f03db222b0d330b61
:106850001dd717faee01d7ed0409eae7ea24ffc5d0
:1068600018020cc3e0d825f0fefedd02200f110354
:1068700014d20beae8e8e3e6e327c2efd9fcf4cf51
:106880002909d3cfd1ef11cbff0ae6132214e6e397
:1068900001e20b19e8d6cccc2226d200ea0df3d4c3
:1068a000ffe2f0b1dbf709e2000fcada4534dadec5
:1068b00014c8d625e70cdefbfd0ad0f8e31f1df156
:1068c00003e100b5deef20e8d9f9de1c0e21f6f079
:1068d000f5dcfdeffc22d7f50416e9ede404edd676
:1068e000efd8c6d5e214dee0dffadaece208e4d64f
:1068f0000cb9f3f3fe01d8f0f40ad8e4cfebb708f3
:106900000fd40be4f609b0e1ee06dbf3f6f916e579
:1069100006cdd8f91b1acafaddf614f02acce4d257
:106920002502f2d8f5f5e5e4faf9fb02eb0e2ccee0
:1069300019f7e302f2fee7e2ef2a0f1d0dfb042434
:10694000e6d41714fc0fe4dc04f9ec0410f0f1edcc
:10695000180bc0eb090027050928231302d8dc0512
:1069600027f0071307fee204cbf9e3f209fefef479
:1069700023ffe116000bfff60505f22ce7dadbff3b
:10698000fbf5f9dfe81df0df101dc4f7fe021c3f28
:1069900008e2fc21d12407e029e6e301ec08d7074f
:1069a000e0f4d00211241d13fd1def00181c18295e
:1069b0000aed0b13c30ef9e917f90c0be8241908bb
:1069c000f20ae128edef24ed06040afb0dfe152383
:1069d000dc06f709da19f9e508de0308fa052813d9
:1069e000edf6030cf5fbee0802f116fcc2e90f29e7
:1069f000cb0c0b0bf613f7e9f217030bea0b0e1196
:106a0000dcfd0400f9da0df6feed23eeb7f3083aeb
:106a1000420c25e30f38f0f5d3061530f0071913b3
:106a2000b114d0fe03fd02df21f234f9d3dbde2402
:106a3000ec0cedc811f7051cdfe816011be9102668
:106a4000da180c1c1ee1f803d3ea2518e6eae3077e
:106a5000ca09e9c31b2d0909f7ef1f0cefeb120d53
:106a6000f0d4010cf302cef1df02261ce900c2fcd7
:106a7000f301ec0f30040a1313f0251fd0e3ee1cd2
:106a8000eaebf310fc26da04f3f2eff3e804ea2a67
:106a9000e2f6dad9f808fa02ec00180bcffe061e6f
:106aa000e9d8d61df20c0fff080ceaede7e3d0eab7
:106ab000fae8ebd3ec0afcc80101090fd2f6d0fecc
:106ac000dfceff14d14efaf9fff8ce15e6e6b81c7a
:106ad00021ebd7f5f1dad7d311e3f01be7ede4189a
:106ae00021f3e13603210012ed17eb2302fac9d797
:106af0000828d3ffe2cbcfeb10ee0d0ae1ee110e2a
:106b0000fcd8ebe6de0301f301ebef1d06fef3d14b
:106b1000edecddea07d8070117efd6f4bc03eaef86
:106b2000ecdbc0d8dbf102ebfcfb0c23dafeb2cbd2
:106b3000fcd9e202cdc710031128cdfadcead6e970
:106b400000f0d7d9040106e6e617c8e6f1ec0ae73b
:106b500017d3fce8d2cfe1f0f0f5e3dbf4d4ded6d6
:106b600006ddf9bdd709fbd7c525f309d00a9efb81
:106b7000e2dadc02ecf0d3ecffdbeb08b5b3d2c415
:106b8000fad404edf9f7db2513ff1ad60722ebd36d
:106b90000c2f19091705f01bf613fc2325fe300beb
:106ba000001e00fdeafaf8d5f00838eaedf83cebf3
:106bb000e92b102c1df1f821f1e016132227081ef5
:106bc000fe3115f41bf512f114fa46ec141203e32e
:106bd000ee0e1b091dedea1613f9011d1806ecde79
:106be0000c13ebf9fa0623fd140117ea0b0805d87c
:106bf000fafa10070e16fb14f8e105001419f3f267
:106c0000e33c0fe2101e2b0030e50b053518ef11a9
:106c1000160e272e290c13ffed34e1092ffcfcc1c1
:106c20000a11f8dd31173dec1af315ec19260cecbe
:106c3000000d1a200b05fe14c725fedd22260de2ed
:106c40000f0418e114ee21ff20f107f5f8fde8de4e
:106c500012fa060f0bfd0410be27e9f80b230cec0b
:106c6000042709ce31cd261b05e503fbf5f80eee12
:106c700007f91e0d10f7fd02c63808cc1d00fdc82f
:106c8000eb1e04bc0c0126e91af825e8d9f523d639
:106c9000ffec13f00ad2fb1dff2aefd4122300c52c
:106ca000002111f015031efa1deeececf7090ecfd2
:106cb000250416211100f603091fd9ce14f5e2e6ca
:106cc000e3330fd829f834f621f91eebfbdcf8eaa0
:106cd000f2ea201c050f0f052e36d7e31516ded776
:106ce00001f206cf08fd29f712fdf7e60104f6cb05
:106cf0000fdd141cf4c3f70a062ccac3fa28dcca39
:106d00002105fce81fff170937060ee52e2b19f2a7
:106d10002aef2024f0f6e1f80a16ddec36100fee2b
:106d20001d300bf31fdc45ed2916f1b6062a29d9d3
:106d300033fc3efd15fc0303f23af1f6fa3cecd0cd
:106d4000f9f707def2fa1ef2100725fdfffb2bc54f
:106d50001ed5212cfc12180a0324e5fa3611ebd7b4
:106d6000f31715f218f814ee2d0505de220f01f3c6
:106d700016054d05fd0bede8fb28d3e719311bfd8a
:106d8000073e06f926f234ad02f7194016e8274d02
:106d9000161a2bfa38f81cf5fb1722dd080c49e30c
:106da0001019220009e40d2ee101101921f0091734
:106db0000a19e01821ef120519f807e608f4f7d0d0
:106dc00011f10bc210f3d919e8f3033af5081117c2
:106dd000e80af41d330b0c1af3f7d6e200dd1301b9
:106de00017f71ffd05e1fe27dcf21401f91c37023d
:106df000fa0aea152e2d050409fc0fe41ec6151a21
:106e00000010faf611fff43bdc070c2ce1e61d380c
:106e1000f123bb00f60d090bfed81c0906cb07f8c1
:106e2000ebfced0d03d6e317e206ff10fdeb12ffbe
:106e3000da1dedf6f0e919fef0d7fae8fde90af7f8
:106e4000f2db080bf5e5f211ddf7f922dcf40a0bb1
:106e5000e90bd5000617f808e9e9e50e09d0092f76
:106e60000218160806f3d711ed090e2affdc03e518
:106e7000c608dc1b0f0f0509e9cfecfb13c311fba0
:106e800007100f0528f1c9fccdee091ed8be01116f
:106e9000aefcde16ee210ffcede204030bbf010e8b
:106ea000eb001900fcf3f008cfce0228d5e320d583
:106eb000b313d10bf7fef3ecddce131308d121f899
:106ec000f10e11181eecd322c7edfe11d8e31ef807
:106ed000db07bfe9e606edeef4d7ebee01c0140ddb
:106ee000ef13131bfa29d6e2d9000218f9ef0004b8
:106ef000db08e11108f7efe8f9f90d230bef112793
:106f0000f6f4ff01130eede8bc1e0423fac30de5f1
:106f1000e717cbf20115f4d2eb0c0d04f5aa0f1d07
:106f20000106db0f2000d510cef80501f3ed12fcb1
:106f3000e617ca180814dbcc1cf512fa0be9250b6e
:106f40000d121d2245e4df17e004ec2407f0f8538e
:106f5000e707d538ec1dffdc05df241211e70f0130
:106f6000e519ed0b26f1d1fbf4e41ef4d3d73ffd78
:106f7000ff18e4fe20d710e7ecf22a121e0ffe1bca
:106f8000d625f7040dd1f2f2f500f70f1a22ed0f16
:106f9000e0dff6dd1ef20d07fc27cff6d6040f1258
:106fa0001edaf8ecf6e51600ebfdf6f41af5fe191c
:106fb00003d6f10609021acf04f002ef06f90dea32
:106fc000fc1fed1105060816f6e1d01ff5ee0c1baf
:106fd000102ffff206180de5f0041aff0e0a09192a
:106fe000dce908011405ff00f712eefcf80afcdeec
:106ff00002f5c6f5e202dceef328fa2d041cfd2ea4
:107000000801f11a0700e4e6b1fbedf6d6c8fcd2a0
:107010001400e2f807caf8f707090dfb14fb091181
:1070200001ea1228ffdae216eafcf42ec7e1fcf7c7
:10703000fbf0d2020ed5f9e41ff3c7f7f6ecf0ef40
:10704000f6c1071ee1d703ede703f00ffde8dd1ef3
:1070500009c10607e1d601f0fbd5f1ffdefecefe49
:1070600017e40f29e01cf728c405faf520071c15c2
:1070700001d5e408ea17f0020ff2ec0bfed4d40db0
:107080000acf1cedc913ef1bd021ed0316062e25e8
:1070900019bfdaf4e2eb1d1732cee4fcba19f2e9bb
:1070a0003dc929cbc31eba1bcc390f23ee242afdc0
:1070b0000be3d1f1d8f5341818c7f6ecdcb5dad407
:1070c00018e524f6dde5cd31e2030a27171b2c0f66
:1070d000beeeffe304fb0c2e05d4e5e0d2fafaff86
:1070e00038fe3a18f1d3fb3ffe0f120719f50509d8
:1070f000dd050716edeb260de2f5e6e2e8fd0fe50e
:1071000039d12b49bc180734f503f7501cea2a2c57
:10711000d90122c2ea0921fec708f209d703fb12ee
:107120001ddd1121c7f516f2fcdded3815cdf32973
:10713000070b1ce9de11f10fd7f80604d902111b69
:107140001cf01331da2d053205eede1616f10417a8
:10715000de0c0df1dd0ff2d1d6020b0dce0d0e04bb
:1071600016d7ec15f8e7090cfa0de70606dc0e2039
:107170000710f9d1d0dfeff102133b1de90cf7fb4b
:1071800006cfdf13d1030fecf916f31c11ffda0061
:10719000d6e1d5fd1e00d900021bc8fadd0f0afb9f
:1071a0000bd90be108ffe710f610e92f1906ce0600
:1071b00009f6fff5ecfc241c1707bcef1adcf2f80b
:1071c00004ed20cdf1dfec2ef8e9f12007020529ce
:1071d0001e0ffd20f607300bfa10b5d008ea1ae4ae
:1071e000f0fb16ec33e90dffe9ee1609d5ebe1e90a
:1071f0001010ba0b0d20f9dc110919f6fef3f42f6b
:10720000e80fe02d00e7eafcf812d63febcdee02e6
:10721000092af9fee7ffee1002d90907d1fb0e2477
:107220000a030e22d6f3de1bf4ebe339f0eb1eed7e
:107230000200f0e2edea0afc1cb6080eeddfedf705
:10724000f8da1cf5d41202f0c810d720e50c1703a9
:107250000bd1e607fcf9e62f01100bf4faedcff1a4
:10726000f8e312f2e8e9d4f7d2f7f5133ef729d2a2
:10727000fcd9e20ddfc4d21207ede3e4f4d7f41435
:107280000ef6fbe4bc10d628ec0ed518f6fb0e1a51
:1072900007c8dc05e50b06e40ce6faf3e3f5dae7ec
:1072a00005d61ddaf0c9df17f1fa0f1527f402151c
:1072b000f700de00fb15150301c5f1f1fbe9c0ed98
:1072c00015d525d1d7bfea27d21e07351bfb192daf
:1072d000eedff9ffec15fc190afde7e8d1fcff072a
:1072e0001ce927d7eeeae616f91c0a2207f6001376
:1072f0000313f5041c05080715f3f5e4d6f228f688
:1073000020e31735cceef525d903122b1fd61e022c
:10731000f500f1dee51e1efedbdbf316d9f4093bba
:107320001ce70447010cd619b1d2d822f3fef12391
:10733000d214e7dffa06ff0ad3d31a25de0a2c128d
:107340001dd52f23f028ed34cff9ea1ee6d72519f5
:10735000e8f9dbbece0c090e11cb2a2ce4c0fb17da
:1073600014dcf921e20bcd3fd9050007d2ea27f85a
:10737000ea03e5d1ebececf6f9e7321dd4f2f81fa5
:10738000030ce4fbd3e59df30bad3be4f5c208e54c
:10739000fb1c16fd2e02ea02abfb33ef25233dd981
:1073a000063f25280c9c10e2f2d32e09f4c5f7fd08
:1073b000dc06fb1c44030913b7ee16f121f819eea5
:1073c000cc0617da0db8fd07fd0725eff7f6edf44b
:1073d000f40912112cedff0abb1303e724ef200080
:1073e000dd0df4f909e5f30ddcefffe9dfb62e0260
:1073f000f801f90029f8f102d2050cdf24e0341e6f
:10740000cc192e1809e8e80cd9ec061408e3fbcfd8
:10741000e313ee041403deeceff60ccf1ae41aeedd
:107420000c1de5ff18c7f7f402ff140c010229ec4c
:10743000ef010526170fd0e2fd0cfbe611f90be377
:10744000fa090d0c111618fefee70904dbe0f5e55c
:10745000b2ff01170003fe08dbee0ffc1dee111654
:107460000120faf20bf9ddf4e4c704e505e91bedb0
:10747000ee0ce70c0b0bfd04cbf8fdf205f10fcf82
:1074800006e706e81604f0f8dbdd1bf0dbbb01e9dc
:10749000b01cbe0c25f9e3dcf4fbf7d916e904e9ce
:1074a000f9091802f9eee30bdfd6fe10dfaeffd1cb
:1074b000020ccb2b0400f40ff314ffec17f3080fae
:1074c000fd0e16fa27ed03e9faef04f4e4f030f4c8
:1074d0000313e91e0109efd8e00701dc22f81eecd6
:1074e000da2108da25e2f8e6f8f9f50adffdfcf220
:1074f000f10ffb16030ceaf9daf7eff127fb00f2c4
:10750000ef1604f81b01e6fff5f510d00ffd18dcaf
:10751000ff04f429080cfdcff80fe7f031e9ded9bc
:10752000df21ffec2ef305fff5f608db27e623f558
:10753000f1fef9151bebcfdde6f8dde12604fbebf0
:10754000ec0a1c1433e109f7f2d312f9e2e713f362
:10755000e40beb2d0ff3f5e1e611ec183a1a31e2ea
:10756000fd1928e933d9ee1306d623dbddd810c781
:10757000e6031c04020af3e9d4010afd3bed1205ff
:10758000e026f7f22bdb01df1bf4fccbf8f11deb5f
:10759000161c5b090b0ec4f5dfe9f3001817f800a1
:1075a000db1cae21f8fc09bf07f5dbddf20ed8daf3
:1075b000f20afd12f018b7cc0afe0ef62411f61ce2
:1075c000e714d4f708ff17c01203f0ea0901d61d2b
:1075d0001d141b17f117b5d1f71123e8280f03dd90
:1075e000dd27ea0b2c1215c6fdf2f5f80af1e9facf
:1075f0000beee83a1148daee13140d040f0d02e811
:10760000e922dff946f904b40b0712eede0ae30eb5
:10761000de07fd0e2525d4df060d1d040f09f40637
:10762000e61dda000813f4d00ce310e2b3f7ebf137
:10763000f30c19102720defa060a0f2124162bf26c
:10764000d618cadf24e70dc8f6d800dbe7f8eb1040
:10765000f21ff5251c14eae0e3f50af931070becfb
:10766000da1aed000e03f5f2080b0ef6e10de2fc5e
:1076700005081f062c06e3ebf8ed1afa020c1e00b3
:10768000e805d80035df06c901dd0df3f110df167e
:10769000fa140227252deef1ce0315f3280903076e
:1076a000d623e7f333ddf5d2fde40bcfe4d8e010c9
:1076b0002508fc011b2bffdf0d1d0ce9240df9e64d
:1076c000f011d102340301ca14db12d9ebf0e3f755
:1076d0001c220a03170cdaf1030ff00b1ffd0c003c
:1076e000e925d7e405f513c8f6040afcefefe90e27
:1076f0001c27ff040826d707e9ef35ff1af707090b
:10770000022bedf811f80df7f8fe0bf60affea0967
:10771000f708fc2b0123d6fd13eaff0451fff8fa0a
:10772000e01feaf03e1900f50307fedb15ff0e131c
:1077300012f3f81f152ee2fc070a1c001f1331ed8f
:10774000e325f3f0070402f70d002aef0af507140a
:10775000d90f090e1e1b0803051410f90c0bf6e3d4
:107760002b2107de10fff901ea1234edfb14de03d2
:10777000000803052de3193af4eefaf02100f90fa1
:107780000af00d0a03f3fac20fd826eac3c6e1eee7
:10779000c63318061efee6eae51c37d92f2c38fa48
:1077a000db14f60918c91bd5dbd41df2ceadeed81b
:1077b000d3f3f505ff0df30cdcdf080d211c24ceff
:1077c000e916f3d736e0f2fbf8f41921d5d00be730
:1077d0000f0af9071af2e20ebc05e5d423f626edee
:1077e000db1107f21df0050cecde02e8f0cc18fd11
:1077f000f912f51e2515f1e7fcf00cef1eff110c38
:10780000ed1cef121cf007f4ddc10620e9f416ded2
:10781000ea14e81b1a04e9f5e51d25e632e1f8e66d
:10782000d1f7001112ccfde30fd50907fa0316efcb
:10783000d4fffc3e0921ea0cd41d021210dc16f222
:10784000fb20fbe72502f9e2f1c70bf700f1e4e6c4
:10785000bf0501110df1e0edf2fde3fa2a0b120b69
:10786000e800e1f208f206e5f5d6fa02f3cfeaf015
:10787000e714e1141b08e4edd4f50ac710e0fdd9c4
:107880000201eed723d7e8c4eed024fdd8d3ea0610
:10789000c40cce191af0dceddcf112eb2500fee38e
:1078a000050618ff22d5e404dac60afde7b0f9d0d0
:1078b000dd10e61e1df5dbe0e6f2fcd11cdd0df06f
:1078c0001f03e9db28cfffedfdc0f8f3e0b205fdb3
:1078d0000701032c0effe0dbd30beee50eecffee11
:1078e000ec0cecd637e201e2e6e0f6f7e1ebea0c6d
:1078f000eafb031e2700d70ef7171cd82bf6cde5a1
:10790000d9050de914f6e1ece6e1fce8eff5240415
:1079100005fcf046110300e9dd08ffea1ff801034a
:10792000ef3af0f045d9ee08d3e419d811fb10f284
:10793000ee07eb3f0707e4e9d90516e3150919ef50
:10794000d20519f935b7fceddbd805cdf8d8120210
:10795000f9f3ed3d031bf7e5dfe3f61143ef1ede20
:10796000bc1e13e849f4ea1113d424cae3d425fa5f
:10797000ea17220815130af3cef4050935060702a3
:10798000ad30db0a1bf104bf03f4df09fb1e03d992
:10799000061e0b12eaed00f102d30d08f5f1d3ea51
:1079a000e3ea0fde070ffff5ef00ccf2f7ffecf490
:1079b000fbf4ffece6ede5cef80a0cdef2d0f60ab9
:1079c00005dcf4faee13fff6e3f9efd21ef0d2da9b
:1079d0000ef803ebdafedeeb1b0be1d9f5ecebd492
:1079e000eae7dd10000c09edf203b6f70d2acc0d25
:1079f0000ccbec05d217dcbc15f2e108f409e1fd73
:107a000006b5d7e7f8e40dbd012beff2ddfee9097d
:107a1000f2d7fef2c2f2e0d21cf4c6ffed30c2e0b3
:107a200006e2f704f023f9f3f9f7bfccd6f0d5ef6f
:107a300007ddf009dc16ffe721e1130ced1be00f79
:107a4000fff8f1180929f4f51507a6f52923eff237
:107a500029fd0b0fcb1fc5ce0bdbf523090b1ff642
:107a6000fd0ae21ef314f5d81d15e9ef1cfee02413
:107a700005fb101ff32fdcc114edef07fa0907ee29
:107a8000f80aee11241b04d50df2efd0fa1d1cf0fc
:107a90003eeafb06d50ff9e0e0ee142e3002f513b6
:107aa000c715d10013250ece1fd5e1c9e513041566
:107ab0003a1c0d14fe13f4dbd804f3150c140cfd62
:107ac000e316d41f11ea02da28f30fd3edeed21237
:107ad000e6220ef4081dfb07dcffff0f161723f646
:107ae000c10bf1120cc906e921e630e2e1ded11545
:107af0000e1206e90beb053be81deb0704f809fb4a
:107b0000e6fadff20ce003e919c44508ddf7fa0be9
:107b1000ea17f1111c0b2412dbfb18e617e9f7f644
:107b2000d609d3f90f0dded7faf716fbd61001f6fa
:107b3000e00902df0ad30c24bdf10efbfef2d8f9f6
:107b4000e8f3f91bd4ece7f3090c01ddedeef3d912
:107b5000f00dfbcc0ad5ee04fb0d00ecebfddf0dc8
:107b6000f7c2d70bc41512f40a1e02f90aebe5dfbf
:107b70000612d7db03e4f312efe9cdf404dbe8e50a
:107b800016ea10d3fd48eaed13d1352534f2170a71
:107b9000f9281f18230d18f9d12cf8d31b2746de1e
:107ba0000d1d1e133aeb2e1808e4191612dc0e0deb
:107bb000231be01226010a06c81804fe081c1ac975
:107bc000001e10e733dee30cfef5f71508f41ae5a6
:107bd0001defe9fb0af401e6f601e3e008ef20e916
:107be0000e0534fa16ea0409dee90f00e201292045
:107bf000df39c5221c120ffad0f401011dc3230086
:107c0000f611090214e5caf7e2d7170cff050ee9d1
:107c1000d922da03221c1406dc0612f51fca130847
:107c2000d6f8f4250cf3de18e7c31218f8e92deaac
:107c3000d921d9252a02fee3cbe1fefa30c0121782
:107c4000a902fc07fdf9ec11d3df1424fab820e7f0
:107c5000b416d8290b1d0710ecf7e00e0be9062b24
:107c6000eb0d041f06d5eff5f1d40236e2e016d98c
:107c7000be03ee13f501f10ac1f0eaf020ef0dfab0
:107c800000fd180c22d7d8f9eed2f802c5d1e2efe8
:107c9000d41ddd0512fae1e8c806190216ec1efb38
:107ca000e10f0bfb0dd8e310d3d0fde1c5adf3e739
:107cb000e6faba252802d8ecf1fee00610d9120245
:107cc000db00f6ef13eeecfaeae500eeeadd0fe496
:107cd000eafbdc14031ae5e6daf001dc24db090d2b
:107ce000d5130e010c0ad5ef01e7f935fee8f1e8ee
:107cf000cffcf3230319d9d913090cf20be810fcbc
:107d00000026010135fee01fd4e6f2fc09d912ec91
:107d10000b08e8210503e9c9ff1de4f01df80e0476
:107d2000ec1af7ef3bcd05f413ece7f40cdb0b0793
:107d3000e8f1f72f1926cecbe301fec8fb0e1fe0ba
:107d400000210bf01efbf4fcf2e1fdfe07ddef1657
:107d50001409f52f0131f3f7eef6fdf71f1134c3c7
:107d6000f345feda0ff8df2512f42d06f0063aeca3
:107d7000fa17070f1eee06e1e605190127f30711b2
:107d8000e92aeb01260013f4f632ae1d0416ebf6d9
:107d900016cbf6e8c40bfaf525e7e007cbc2bf1512
:107da0000ac70cf2f611fc0f1c06bf0d13ff2a3494
:107db000fdfef000ae0feff8150edd0cd7f1f61852
:107dc0001ae60cfcf100f80af309e3e90a0e020bcb
:107dd000290fede0c7060b1945f42812ff02f21a2d
:107de0001de60feaf9190f0c0931db022b121d0dec
:107df00015e21cfdd4131611480f0607f6fde1fc31
:107e00001bfee11ff9101e112729f4df1113091cb5
:107e10002014f9e6c6fc29f40cff01fddff4fd286f
:107e200018e70016ec29fe00fc1df90e0e15ecfcff
:107e30001b07f7ebea050dfc17f40f200aeaf91d02
:107e400003ea1e0dfe170d0c111305261015110166
:107e5000241309da06f5090b20f90e16f404f0ffd5
:107e600026001820f9130108fa03070305e8001a91
:107e70000a0015e4eef2fefd40050407ee06d71fea
:107e8000e7f72d28f0222d040938e82f1a21fcf8f5
:107e9000270e1d0c010d13282200eb09f12ef6f11f
:107ea000fde6f6090c2925171b09f4262446e325cf
:107eb0001403fef3e60e162304e60d29e708011865
:107ec000fbf9160fe328091d11310726f844ed20b0
:107ed00012f20aec0fff3718050c1033f119e91ce8
:107ee0001bee2519fe2215091d0b0512edf41816bf
:107ef000f7fbfbd4e3102709f5ff2e29fb0b031c2e
:107f00001c09e80fd505290623fc0416f029072dc6
:107f1000f5ec26cdfbfb2e2b22ed0cfff2fff6102d
:107f200003f7e805c83a1fef0e11ffedd6feee1776
:107f300005021dd9fabd10212c091b1cea1ceb17e8
:107f40000dd7d90fa53921eb1739fd3aed18fbe410
:107f5000ec021ab4e7d4f60137030004f701ec1c75
:107f600020d8d5fdea3316e40f30d34e0625bcf2f7
:107f7000180013e2e806e10840e6f911e8eadaf948
:107f800037e4170ddd311240e728fbfdfb1de6d27b
:107f900004d122eef31009040ce6cd32d9ffb4452a
:107fa00018bf0203d02cc5f5140de5ebff1715ea39
:107fb0000d0f27f6f2f1f8fbf316fc0bf721dd2b82
:107fc00025f7fd48010dffec1ae902d7fe20e9ec88
:107fd0000b250afce2f80302141e1a272222f703db
:107fe0000006ef38121517ff190500f2070ddbfa2e
:107ff00017e80ddb08dd040909f912020917defa9a
:108000001110ff0839e425000fd407ff270004fcf6
:1080100018f8100c050b1304f6320f171b2fee0582
:10802000180f07fa001c27fb11f213edf10b160ec7
:108030000c0614f000f2050bd23104f5ed25100307
:108040000ffc20f900052ff031f71b002027fb0063
:10805000fceb2ef4f6d70cf817260feff63112cb07
:10806000061509d117d326f10d0510001b0c300e93
:10807000ebe02803fbdffd0ad43a03fe0a0efedc28
:108080000611dbc90ceb23fd1dfb08e4202cfaddf7
:1080900012df26caffddfe1f091efcbf121e08d01c
:1080a000fdeeeed705301ff625f0cede3422f5f8d2
:1080b00027c328f8fee5f5f41812fd03d5320504b0
:1080c00007fffdcfcc2e3ed63b1bf1201215c1fa87
:1080d000fcd136ea02eb11060022d8d8e808e0db32
:1080e0000be213def4f62ef2400bd4de0904f1ebc2
:1080f0001ec529ebf6c80929ed28d5dcdc0fcbf825
:108100000ce7e8dfdd003cd83729fcd92312fcc49a
:1081100002ddffc2ecc9e02aff32d7eeccfef8eb5d
:108120000ccf0adfcef518e0f2ded7f11e0bc0b49b
:1081300025e8f5eae1efebf2f515db24e6c7ea19ed
:1081400003bbd903e7f7e6e0fbe9e203091911ec09
:1081500009fef6e9cd09f5e808031702eff2b316b8
:1081600001e30907e1ffd1f6f107f8fc13fbe11782
:1081700025cbf212d20a05f205eeb9efe4d9d6e822
:108180000be7ef0f1125c1fdd5f8e3f1f808f3f186
:10819000ddddec03ea222a0f1fe8f51eeeeec22b0e
:1081a000fcdbf2fede2684e12fe706f7ed0c24f679
:1081b000e9f4f2e60c05f2f2f8e1f30f10effd0b33
:1081c000f9eeff2de114fff62ef20acb131f040582
:1081d000ff011de9b80d000e0d0c2c2423f0e3085f
:1081e000fa14dd0dec2315f1261afeed1d1bedf63c
:1081f0000dc211f305f0f9112b0c1df9171cdbe270
:108200003806fce51e2706e81cf607f2151b13f1dd
:108210001ae2240b0cf5fd0a202d0e04ec1ae9e5f8
:10822000f318e9fa002a36ef162112db0434ecfccd
:1082300029f12adeeed3fc0a1140fc05eb34fc15d3
:108240001c20f6f8e3f536ec20200ff01c08e706ba
:1082500017f81fdcf9e5f2030b3517ebd329f2ca47
:108260000dd5fdb7ef181dfc2b18fcf400261008e7
:108270000bf437f1f0fb091b0a3007f2e6fbfdb205
:10828000e7e7fedff12119fe3118f9f21914e101d7
:108290004df10ce00f09061e1614fddfe714f0f196
:1082a0000009edf3f00e1bf72f2cf6e50a3aff0656
:1082b00020ce19f5f414f9071b20f908e51ce8fd98
:1082c00015f4f017e2422ae655250ade21fae30406
:1082d000eeec2cf6eec60a0d1110fd130613fee2ad
:1082e00003f9f1e5e5090fee2620dee6fe2905eab1
:1082f000f8d210ebeafcfa30d21ddbe0fb3cd3ed08
:10830000f502e6c607e73ee7382cf6e31d2e14db40
:108310001ad15703f0d8ee25fc0dc5d9e422e5dfcc
:108320000000f9bffa0e50da520c0bfb1f24ddd50a
:1083300010f951dee0d4031d2316dcfdef0dd3054b
:108340000cf2fbefbe1729f438211cf21cfde5c02e
:108350000ef52ad719f22f25fe0bec12f72df50298
:108360000bf501e2cf141df108e416eb3912cee44f
:1083700021b917fe02f215311009b6d8ff29f8dd30
:1083800002f4fcde0c220f0d0be2c8ee1500ebf43c
:10839000021618e8e8efe1ff16f10e030712f701e5
:1083a000ea05d5f6f7082ce50f01ee180600bcd05b
:1083b00011e503fef5fadbd6f2ed14f906e7251315
:1083c00002c1d6fcedf709d515ddd7faf9e7d81ebd
:1083d0001beafee3f813cfed07fcfff80a0ce414e8
:1083e000f3d8cc040dfd17d1fe0fb2e7f70ce60869
:1083f00003fff7fff334d2b904020ce7dd061502e0
:1084000004ebb00cfd13fac9e30cbb06fefedb0a5d
:10841000f1e7efdbe4fdd0d3eef3f1e3cc20030191
:108420000c0ccd05f1110bf9f0fad0db0701eb07cd
:1084300010f4f40dea1df8d1fae30200f813f8fc89
:108440000efee6002010ecda0b06ebef1bee010a45
:10845000141c0406d71ef6c8f8e629f012003dd910
:10846000e428e30d2c27fed6fc03ff13faf7ed26d4
:10847000f41a081a040ceacdf1f5481621fd36e489
:10848000f01de31216fe08e305e6f81d0001f123d6
:108490000d1b01221f4fefdb0afc2932230f41fe87
:1084a000eb35def6331ff2f8fcd40b0bf8f7e905d9
:1084b0001305fe011735f7f10616470a180c24e9d3
:1084c000e029fde6131801da0bea0b00f310fa04b9
:1084d000072207201111e4f0ddef22f410f7251731
:1084e000e01fd6ee260d0e0e12f33007fcc3f84a3d
:1084f000ec29ee06ee510a09e9e75efc16041c00c1
:108500000a2207fd22f80602f8ab1ff601e80c3438
:10851000061cfe0809101e00cb0422f2131006fcf4
:10852000d517fffb2b08f511f4f217daf609f63828
:10853000f642f1e73b0dfaffeaec560821141d2242
:10854000ea25f6251d04fdfefdf617e5ecf0110405
:10855000ee31fc11eb0e0619edfe410efdeef81d9d
:10856000050dfc31f50f090adc0805deee080bed00
:10857000f51dd50ff808191e05f6f72bfdcbfe37b4
:10858000f7f72f31edf6cee1f8b012e1f2ec13017e
:108590000e23080b290bcfd7c81230c3041f2fe2bc
:1085a000ff23e20104bc23cbfecf1bfcedd71ffb56
:1085b000e817eb1108fe18fce60011f20afe05e1cf
:1085c000e41addf32dfcefe7fad51d15e2e6fde731
:1085d000f50f10141ef0060bd50607ff14f731eb4c
:1085e000fbfefc0810f7faebe3c320eed1ea06dc51
:1085f000d70dda1d2f0b05f8d9f7f30f1fde1e1468
:10860000dc0bfd1e1d07d302e2f3f60bfbf702f3b2
:10861000f028dc15f90bc9f0f2f0f70423ee13f3a0
:10862000de0af91825e9f702ffe4120c1c0404e045
:10863000e50dd0251c13d1fdf9fa03ec27de0df36f
:10864000fb0200e61ce6f005fdc30ae6f6e0d7e211
:10865000b80e092816fbe7f7ddf6fbff1f0b06dd5a
:10866000fa07f00017e209e8f7c9fe0edfd70adec5
:10867000cc02ee162705eb10cfe505f415ec0cdb6c
:10868000e6031e080dc501e701c518fbbcd207f7bc
:10869000c40ef42016e5e7d6f510f6c81d00150e39
:1086a000f90603f201b501fcedd703f6f4c912d6c1
:1086b000ff17f015f1fad6e7e708f1f40eeb0ce539
:1086c000e80a10ee19f3ffe0e8e8fcebe00110eb3c
:1086d000faf7e922011ed5e3e61905bcfedefdeb43
:1086e000e81004c41cebfcfdf9d60bfad0ed1af32c
:1086f000c3fdf8260408feeb041603e40ff810d4bb
:10870000f41426d209fef403ceeb0ef202f814dbc9
:10871000fa07ee3211fa08ece307f3d1faeb01e5c0
:1087200003080e0937e6ef08ebda09d91bfa2b012b
:10873000f1f7ee23142acbf2dd00fbe104fb19e490
:10874000e91d10082dcaff02d7bd1ef30adf02146f
:10875000e406e2391420f2ccf30a060b2a0725b806
:10876000c12726e01dd6ee04facf2ad4d3062bf576
:10877000e41e1812270109d0c6f40f032df81dfac4
:10878000bf3dfd1026dbffe614130aee0e1bfcd1e5
:10879000eaf40b04070fdffb08f7052022e1ea0cdf
:1087a000de38fa0df009e8d0f50109daf9063ae504
:1087b0000118291f02fae91eede2073824042b25cf
:1087c000ef1d04181a1106f717fc15e7f415150626
:1087d000de0e38e4e9eeeb00e7201401190f0a0c75
:1087e000f81bf9170e0406f8161107de1b1201f626
:1087f000d8e52af90410f8f815f8181b2dfffd022a
:10880000fe1af70d210a35de2b0108f3242a07f49e
:10881000fe01011719f4fc08e903050c101905db2a
:10882000f613eef00f1342e83d040df11e16eeefc5
:10883000f5f3302806e30f03e13806d31225fde6f1
:1088400025180ad113e335f32be1080a0020fb03b6
:10885000eeed251d16f61214e74bf9ea2222f5cfac
:10886000011b11ce1aeb47fe2df3030004e6f6f0d0
:108870002ef71c10fef50cfad262d1ff201006fb79
:10888000080202ecf1eb40e4250dfef8f7f0f9e206
:10889000090f0eeb08e7f4eb1a28fbfa330ff6008a
:1088a0000b29080bfbea31f633ef05eb10f4f1e38b
:1088b00025fd100eeb03f5022532fff31418e90d28
:1088c000fd170304fc001bed47ff20000fdcfbf548
:1088d0000d110c1ffefcff111023fe08f5fce1e753
:1088e000dffb00f409e13e011af307ed12110df26e
:1088f00003f4110005e3f306ff11e0de08ebe0ed01
:10890000f60c00d0e1e82ef854fcfce21e33fde347
:1089100008ff3710e7ecea0ff0fbf3dd1d3de9e05f
:108920000c0a05e3180556fe3ffb11d4eb232ae39e
:10893000f7f459090ce6f105f821f3f2f23500eaf3
:10894000fc0701e4f90525f8310b2501fa0119ddd1
:1089500014fe39271efa040ee415f2dc0a4822e55b
:108960000004fafd1ef527ec36fa1ee804090bd6c2
:10897000080e4ef726fa0e16ed38f1e0fd24fbce78
:10898000070403de170836d7121fe4edebeaf2d036
:108990000b02fceb0edaf3e416c1152e10effbf818
:1089a000de00ce09122bf0dcf9fbfa00d410faf04d
:1089b000ec3001d204ccc0c80ce6f9f1ede4ef1fb5
:1089c000ffced005d01104e8e5fdd6d20d10b3b22c
:1089d00000def4d8c9b0c9f51ef0c9d6d9b4ceefbf
:1089e000ecc3cff2d00fe0d3f120bff7240bf8cec9
:1089f000feb9dce7d6f7caff28e7c4fdb5dea4e37d
:108a0000f6a0d3ddb905f1dfdb2cbdf7f61e01d4ee
:108a10000bd9c7f2ebdfd1f0f7d5c41fc4e3ec22ca
:108a2000f9f6040cf407ccfbf30cf707fb0dfbe2a3
:108a3000f5f4f117e307f3fd02e4f425ecded721aa
:108a400007fc09090c09e6053e10f3f50802fe05ce
:108a50002d17f2fddaf7f3f30ff6fc10ffddee1041
:108a6000f40d0d0e1602f1061103f408fb2017f8a1
:108a70000d03fce3ee02eee21ee6fd0df303e3025e
:108a8000f8fefd0b07080efc180118eb051afffe97
:108a90002610150e000409081409131410ecebfc41
:108aa0000e1b021918200afc2dec1be4fb1907fe13
:108ab0000a0e2af7f5f1ffeb1e1509131c2703fd1b
:108ac000f40be3fe0417fdd82efc00c30ce31dfce1
:108ad000f2fc05e8ff04fdf0e4f40d08f7f8f5f208
:108ae000e70be90bfa1212db101105f60a090dfc6f
:108af000f9f32c04081a0107d60200e60014f5f871
:108b0000e50d04e70bcb3ceb3bf007d9da0aecfeb2
:108b10002efd1cfa10fdfa0d033c12d7010dfdc20b
:108b2000fb17f8d7faeb2ae83305280fdb06ea0132
:108b30003b04460912e0271a07081504f62607f237
:108b4000fa07fde1ce122bf2220e10f006fe09e527
:108b5000f41541f32ce21122fc1e0216f835e1ff58
:108b600011d10bf4f43f2609f413e6ef4f32f6ee81
:108b70002adf21c801ec20411a27eaf2d936fbf698
:108b800014f12404ca0e400529ba48f0f8e9c9e4f2
:108b9000da150f0433f3dae7a3f810cb191d43f10c
:108ba000e41ffcf30aab16dde0a623f0fddd05e6cd
:108bb000e80cf9052502f33cc2c7f6f615e928cd05
:108bc000b61bf0e510c5ff070ac40be7cdd7f2e4ea
:108bd0000bed021744e7031aa92300d90b0114da9d
:108be000dd0802f221f90000e7c41302d1ec05da36
:108bf000d627ee201eebfae0d01ce4f318ec2d0d86
:108c0000e7052f0d22def916dfc40721f0e70fe993
:108c1000d104e60e1c0acffbe915eadd1cd1f4e60f
:108c2000dc1a140236ced9fa09ea19080aff1fd94c
:108c3000e70401261e08d0e2d8e7140531f7090839
:108c4000e512000120f3fae111d4111bcfdffbd3b1
:108c5000de0917150e09e121f61600d917ea0419e5
:108c6000ea021aed16f5fc01eff3eef1e8e0dfdac7
:108c7000dbf9ec162e0dea00c60ff6dd0df710dd60
:108c80000b0b16dc12e8e9fcdede0fefc8cf130099
:108c9000c006e91b1bfad1c7c2fdfde81bf408f0b2
:108ca000f01402f4ffdadf18e6f406fb14cb09da5d
:108cb000f811db1311f8e00dd80ceaf62bf301f4f0
:108cc000df2300e1fdf1f6f6f8c7faf4fede13e06b
:108cd000ddff000e0f07e8e6e11be6df0afa1af4f3
:108ce000c819e1d912c00cfbf5d80205eff00ce36e
:108cf0000e11f827fafce001da1eebf02cee06bdaf
:108d00000b0c1cec10f7f6ecf1f00df40bd91bea90
:108d100014fee9f818fce5e1f81be4e409f1f3d2ec
:108d20000c260c1730e4271be40113e322f22ef586
:108d3000ddf3ee3bf507e7de01ecf7ea19d90ddece
:108d4000001836141ad9fcf8dee917fbc3fe28ef29
:108d5000fa00e7380ff1f1ecf1f8fdf53c0416e10b
:108d6000edfb351f3be2f90b1fd305b8e0f60fea28
:108d7000001cfc2c1ef3f7e6ddf7ed0c0eef011dd9
:108d8000cf52f80723ecf4e3fbfa9503f7f9ee2d45
:108d90000dda3c12b719d5e601fd0108eb0adbe755
:108da000fdc8cce5e60d22f11e13bdf30006f92e39
:108db00021b11f01b424e8ca0711f5d8ed15eff869
:108dc000f4f6c2fde51f31da02dcd1e4ece7f92c60
:108dd00010feea0dd90ccac60e190711e71702f4e6
:108de000f20ad31ffc02f901fe04bb0c0e19f513a5
:108df0000a071008db37ddeefe100c171433e52ae6
:108e0000ed18e41d06e206f91527fc01faeef01e46
:108e1000f11011ecdd010aee18f5240bf90711e54c
:108e2000f407cb1e14f708eb1821dded0316fa3416
:108e3000f90afcf7fd03f8f32be739ff0003090dee
:108e4000fde4ef231a34f1f6101e0a090408eafdc6
:108e5000ff16fc001112f6ec11fe18f508fa1b02c1
:108e600006f80518110cf10305110a1fd904d50adb
:108e7000eb0d0d10f418fe0f16e015170eea1e1f6d
:108e8000f2f108061a1dfc1008110c27cdf9e119a2
:108e90001e12030e142d0c0b0cf71a150afaf4040b
:108ea000ea22f717fd22f9f4f4fd0724edebf42292
:108eb000f01c01fa1022fd020dfd1b1eff021a36e6
:108ec000f6050dfdf81ade2bfef60bff13fff7116a
:108ed0002314def10a2cf70fefec30240ee8f34eea
:108ee000def7fa24ed0df1fdeee12506f0f0142a8f
:108ef0000818cabe0917142712e85735e3e11b2ae0
:108f00000dfc1068dd03d71fbe0b11e200f300302b
:108f1000e10dddb4ffd6171ff3d2430bb7f9e128fb
:108f2000f1bffc29cfeaaf27ddec1bfc1400e714ee
:108f3000dffadedc07f6121805d62629dee0ef1d83
:108f400006ccdc23d608d0c9f106c2d92515090400
:108f5000dbf9cc9eeae4faf910cafae6d5c9f51fa6
:108f6000fec2c61fbc05dcbbf3f6fcf4dcece8e992
:108f7000072ab3fbed11d6e7fea803fafdaae51b0d
:108f8000faeeeb311b16c80421e600efe4ff20eef9
:108f9000f12841112500f00cd61313fb2d4320f9c5
:108fa000d910df1cfc0f0dc5ecfd17d8e1edd7ceb5
:108fb000f827f50af5eadce0fdec10111c1a081799
:108fc000f120dc0219eb0dcf17f508fcfadff1ea0e
:108fd000f102f21ffd0dc5d4d112fe01f70e0d0beb
:108fe000d519f0fa23e807def2f91ed2bde2d3fd6f
:108ff000f726112b282edde5f019071e1c040501ac
:10900000df2ce90e38fb05e505e923dfd2dcd6f2db
:109010000923f226341debf5fc06140949ff1bee6b
:10902000da29d6eb0ff9e8c318cb22f0aff3eff74c
:10903000e52802362b04e8d8e0f22c03270218fcbe
:10904000ec1fd9e722f3e8c315b724c1f2d4eef33d
:10905000c40601fd1a03db06e7fe2f10fcfd0eeb34
:10906000b70db605200b01d3f8e10ae7dd10f0e4f7
:10907000fa010e141423fb0ce7e6f1e212020ee1f2
:10908000f713e2d919e80ae400df00efe9f102e0a2
:10909000e4d8fa3014ffe90aed170ef1121a10e3c2
:1090a000dc27f90619f5ffe216f7f407b6cae3e77d
:1090b000fa15070e2efde6fff203e6e218ed04f2c4
:1090c000da2adbf5131005e305db1710d9bbf2f73d
:1090d000111ef0150006f6f7f200eb2a17ed121735
:1090e000dc23d80e1cec06e9040ff1e5101af60b90
:1090f0001b2ced36fe21ded2030113162bf3021bcf
:109100000112f0e62e16f0f2e003faebf00fea039c
:109110001915ef3b0027dfd013f5ec0b2af40e01f5
:10912000ee2511df4201e4fffa05f1ea0a060eed31
:10913000f8ec0d202a1ed7eb09fff2041b063503bd
:10914000152efceb1c0efeef0a1610cef3e610fafd
:10915000e90c06400a16e1d6ec02f5e4261e0ede06
:1091600006491fd750fd12ffe9effceb050c16fb7b
:10917000fc0f0b0d0a03fe07f2fef6e7001909f9d2
:109180000322fcfb1b0903e215189a04cee4d7c2a4
:10919000f6e8d9f9c5f7bbfb33f9e438dfe590060b
:1091a000e401bbe6db18c2b4eef8a5ef071228fe17
:1091b000d5ee14fdb325bcb605f2ed07fbd2051aba
:1091c00017e4ca172a1bdea7fae5e4e83117f516fb
:1091d000f4fa200dc4129ed025f50e10f23be60bda
:1091e000e713aefa190d1bd8172fdffc05f9f004b1
:1091f00009002604e200c7dd32f92709100fdcfe62
:109200001f0bc602081512d0182af1d6dee0e0f8ce
:10921000150227fbf822d9c7351c12211523ff2b75
:109220000717ec13050f0fe3190d10e51115f804de
:109230003804151913f6fcf5060edbf622f50218b4
:10924000161eeaf72427fae50a1a02d9e41ce9f502
:1092500034fd0dfee308f3efff1d12fe0f20f30cab
:10926000dafcd8f804fd25d729fce9ee0ff8dffc7d
:10927000e71029f51917eafef70a18fe1907221454
:10928000d413e41a111326f229ed12c1de05ff06ec
:1092900033131a0608f209f717190a0f0a060e0403
:1092a000ce16cfd9e7111ce91210f91606deea082e
:1092b0000a060deffa20f8fd08f90c0fe620fb0571
:1092c000fdf0d9fdf12106c6111200eced12fcfff4
:1092d00014f20502eaf0f7faeaf7fa001815fbfbb8
:1092e000dc00f0e707f915f11b1701e0e20cfb00c9
:1092f000dcfcfaeafb19191315c30708e2edf7f8cd
:10930000e70afb02ea150e0215150df4f117fbea48
:10931000f0e8fdae0be427110c0719ffe317010479
:10932000f0e8eef9dee804e2ee0af7e3edf9d5ec59
:10933000ce08dcd610f12b2f23f91b04d104ec034b
:109340000cecf8e5da1107dcea0d02f3e41c0ecdb3
:10935000c3f229cee3d007170407130cc601e3209c
:1093600031bff0dd8105d0f7d518fd162a1fbbdf10
:10937000089ec207f119f1f920e3c8d4caaaaeefda
:10938000019aefe8e711d3f821e8f2f6f00436434a
:1093900005163805e30ae6ec02e40dfe083e08fc7b
:1093a000f2eefde7020d3724f302f01605f8fe1782
:1093b00029fae820da0e04fe1a02f1fcfaf3190a7f
:1093c000011206e9ddf8010201fde908dd12f625ca
:1093d000fb0cf02f0810eceb0a02ee080afa16f369
:1093e000e919f61bf507f2f400ffdbfaf209102089
:1093f0000b01fd11133e04e711033cfcfd220f1489
:10940000fb19e518250907100308020ef7ea0219ef
:109410001257eef306f105e10ee9251129e318f9db
:10942000ec1be3011ae9dedde724fbee0612dc1d8e
:109430000951dceafa23ede91ce14d2800fb05287f
:10944000fcf2ee2fd411c4fdf50511fcec00fc1f5d
:109450000a0bc9fefb2706fc0dd52c2a0cf61b09ae
:1094600008f4f830221adb06fa13ec2a0003e1189c
:10947000d10bd904083b0efe32dd342efc061a2334
:10948000f3f3f5fb0a0c0c09f4e7021704f0e82ae1
:10949000201cf10de75efaffe3f01c3109fb060e1c
:1094a000d6efef2a0308fffbfa080e18eee9f22dbb
:1094b0000b39e5f00029f3f4000245142efb1f0bd5
:1094c000e923071c0a07ef0ee6e41116e5e0e50eb6
:1094d0000a24e7f923f001f5030c2a211b04135396
:1094e00001280710282bd9f5d6231025f7f7f02ce3
:1094f000fe18e30111410cfc24e7511411da0b436f
:1095000004dbe1311ce8c6fcf101f0f5dff5ed3cd0
:10951000f70bd014f64018fe1fec4c321cfc041a5a
:10952000eceee729f109ddf9f70f0a20f5fcd62862
:10953000050bd7ed07fef5e513f4382a15e4362ab6
:109540000413e32bf517e90c0a132cd800fce70ce5
:10955000f035f4d500e5e6f907eaf904f0e9150974
:10956000141cfb0feef4f400f0fc0f0bdde9cefc55
:10957000e91ff50f14020de7e6d82a12f9d90c21dc
:10958000f60025311ff4d61d33fa9dddf3ef0508f3
:10959000f6eff8e7bb0caa120df2fb20ced8c20bf7
:1095a000dfd2a00ad10f0acc3b10a5f10321fb0c9e
:1095b000d8022208aa13aab810011d06021ce5e869
:1095c000e00ac412fc0407c909f8fccc0bfdf51f26
:1095d000030b1418d824bfbc0bfe2d1e152f21041d
:1095e000eb1bdd32150e19dc20e8f3f8ed1ce80169
:1095f0000e1cfd0ffd2ee8d80c06431101fa0c23ba
:10960000e21ccf04f2190bc306e6e5cab3ce020290
:109610002210240f1233e4d4dc0014f928110c18a2
:10962000f21bd70d102303c221cf1bd6b2cbfa1bde
:10963000002506f22f1cfbe2c0e435042a1dfceadb
:10964000e218cd1927f6fcce04c020d3e7e3fffed5
:10965000032408e92cff050bb8fa3cf3141a0eefab
:10966000adfdf9fbfff20ff5f0ef0debe8eddf0fcd
:10967000010c06fb17ea110ccdef20f20b062415a6
:10968000b1efed0130ef12f8120e1bc9d703ecf465
:109690000b0909d20d0727250707daf01cfaf3fc9e
:1096a000a208e3d6f82500ef0bf7f438ceea0d0f49
:1096b000f4ed1ab9f3fb262a2ce2e3efca08ea0814
:1096c000f509ef08fe560c0f24fe0ef2e012d7f358
:1096d000170403ffe8091f22e7e21509e1efe4f6aa
:1096e0000a03fd1202131700011503eadeedee0b6b
:1096f000251400e7f4e9f8060b07060c11f0111b1e
:1097000000fb0016c7f20a11fdfbeee4f2020bfab1
:10971000faf5e8a3e6c4ea181913f502b2cd06007b
:10972000e8b1e919d1f302f1fef8d2e4f905e2e17a
:10973000fefde6dfc9f4f7120be81ef4c3eee5f612
:10974000f6decfe1ef17e3e7c807d2c8f80209de7b
:1097500003dacdd6d9e3e700f9ff08eedbc2eeea83
:10976000f4c6c4fbcef9e2d1f70ee8f3e907a0098d
:1097700008a9ef08e305d8f91ad5f1c4e0afa1d4e0
:1097800015b5ece8ea15cfeefcf0cbc0e840e0c53b
:10979000f9fdedf8fb0511f804dd241e04d0e40505
:1097a000e2fe01e60418cfcc04e3fdf5fb0805eb6f
:1097b000f9ec04e915dce0e8020815d2ebe5eff678
:1097c00017d3e3f0b6eb16dcef16edde1214b1c5dd
:1097d0000eecedd0d8b0f4e40301dbebd8cee0cc56
:1097e000e9d6e0d2cc04f3d9e0f8dff31318c6c30e
:1097f00000d5d0d4c90bdd26f9dade06ea03b4d4ed
:109800001ca8f60ddafbfce3e61ecff9010ba9b9a3
:10981000c5e0c6b7e5d7f7f1089be7e6e2e9da105d
:1098200009e114ecc51bca01d802dbef2421b7d82b
:10983000f6ead1f8f91e0cfb0bc4f92fcceed009d7
:1098400003cfe512101cd9ee0affe100f414ebf58a
:1098500011f4fc06be22c5c729c006170f0100dfa0
:109860001f10f701240806e422feedfbf110f6f7c5
:10987000f3190df8c524d3c24cf0170a02f703ff01
:109880000101fb08fb0c0aec2bfdfb04fc21ff157e
:109890002a0f0d10dc19f5e01c030b0e000cf9f07b
:1098a000f105d5161a1d08e20aefebd1b2f4010c4e
:1098b00002221bfc140ce0d321111b0c180a1bf113
:1098c000bb0ab601fe0510b505110bccd922dbfb96
:1098d000f91e1a132406d6f0031c0415132006fde6
:1098e000cf10b2f5022900bc11ff14d818220a0ebd
:1098f0001c02f8e5172ef13306fb182bf32d031588
:10990000f6fdde1cef0705f217ce03d9f607c819de
:10991000070624090f1c161af10710df0e0601f1c5
:10992000e11515f70b171fe801e024e8e1e7da1766
:10993000130607d2141f1921d71a08e6111dfe06b7
:10994000dafad820dc02eadf0be417db030fe7d1f9
:10995000e30aefdd1dcde72ed71b04f9ff15e82c38
:10996000e8fcdd25e80e0eedffecf0fe2112f0ed37
:109970001ce903c4fd0f11330504f40edce8e60c0a
:1099800001f51410e40aec1d1dcc05fefe09455737
:10999000160b2f12111ee9fae80e15fe09543fd1dd
:1099a000ec24f72e0cff440ff0f50d0e03fcff1412
:1099b0002d20ec02f909e5f713fef606f7090ee98a
:1099c000f613f3fa08ec0aee0afd140ee4faf710a7
:1099d0000b11ef2f0522e708220612f10be6010317
:1099e000df1608f40c0404f2120f00f20df2071a4d
:1099f000053df2122e25efdf0b0b13fa3efd050796
:109a0000ea43e70d3b0308e8f40c060df3f2df260a
:109a1000fd22e0da222cf3e3f1f547ea15fe21f30b
:109a2000e122e31207fcdeedede4000cfaeeea19a8
:109a3000d01fda052e1d07f8fbbe450f14ea08f704
:109a4000e9f1dd211714e4f9f6de10faeae4000981
:109a5000f112d5211b38fb0016d7111619df0eecb9
:109a6000e00ff8143202defafaf2f9e6e910e1f852
:109a7000092607fc2814e0f7e6fa2af527fc26f168
:109a8000d2f6dc0f11fc00c8ffd6f0f81202e0138a
:109a9000f623e7270243eee1f2e6430a15fc360e11
:109aa000d60bf2202803020e000c0de8c5e4f007e7
:109ab000f121fefeee4bfed508d41f2618f8174afa
:109ac000fd0ee50f3619e9fd150b1505e3f103173a
:109ad0002c0afc0b2224f2ebf1f82b2f25f5244461
:109ae000f5fdc7002f2101ed080601f1f706bd1fa6
:109af0002024e320145acedc37032e241405323bf5
:109b00001f37cb033c05fddbfa1af9eff7020c3bdc
:109b10000a1df619ec36dde320ef48233b04202c28
:109b2000e612ec394a0600f30c170af9eefafa4f7e
:109b3000f3380013321de5e404dc671e13052e1113
:109b4000f83604033c0109e2f6080efa1ef4ff178a
:109b5000f626fb222816e0f4fb0022ee0d0617097c
:109b6000092aef0d1de2050c13fb0cf60101042d73
:109b7000f412fd0d3504262b100633fb00f70d13f0
:109b80000426f4180d03fb181a0cee2b27fff2f72e
:109b900010f4f1f313e5e3f9fc25e1caf3f9f0de83
:109ba000160ee60e0711191e0015e4260009c8243a
:109bb00015e703fb00f708f20214cf06c902d8fc30
:109bc0000a03f2cad7fdff06fbebde200dfefa1eec
:109bd000e5d8eb0af0f91ffbf32206e6e00ec7d743
:109be00012d712ffebe6121bf00be50f0604121e54
:109bf0000af8e3fae3fa140e0302e6ece0fdece007
:109c000003f520fbddf3fe1ee323001201fd1832f5
:109c1000eef0dbeed61f1101fad300ddb3e7ebc7a0
:109c20000ae212f5c9d9e50fcf090a24f3f3181790
:109c300015f9d3e9e5f0050425cdf2d7b6e105d84d
:109c4000e6da04d5c0ecc60ed91e231df0041b09ac
:109c50000ef3e508e71817f301ce1edff5c1ff0884
:109c600010ee0d11e7fbce10de0f02101331fb27b3
:109c7000f60dd2d7f90a020a28d30e09fcea0a1b0c
:109c80001b0406f8cafed01ac319d82f1e05f50dfd
:109c90000d03e200dd0508f40ae10412e9f410f80e
:109ca00018ed10f90302ef22cf07fa1619150b1e53
:109cb000d107d5d705110d0505b4fff703e6f42745
:109cc0001f010a10ee07c331ab02100c1b081f1056
:109cd000d200e7e2dcfb1a0301db1a18f8e40111f9
:109ce00018fd17110a0fa719bdf80f16f5ef080494
:109cf000b51bc60af7140adee2e61525edcd240fe2
:109d00000a06022514f2ac21d5fdf21df6c30d2b77
:109d1000ea17d3f4f835fef008eb0b32e9c81f322e
:109d2000dbdce01ce5d9c82ba015da25cfd0e9ff94
:109d3000f906bd08fa090f0a0efd101c01d3110e19
:109d4000fedb1226e60ec5d8c912c523daccef1dfc
:109d50000b19c2e412ee00d512dd1412fccd2c0951
:109d6000ffc5e824fb0fe8e1e12aea27e1e00d2a3c
:109d7000100eb41bdadb0acf18b71a330cd2e9f98c
:109d80000df9e807fbf6cb38f626fe3a06f90c0a81
:109d900012e7ecf9dce90fe01b25e5e6ead2dc0688
:109da00011f03bfb13eb0c27ff16e61f0c12d81625
:109db00013d2e6c517ea22051724e2f4f2f7d7df3b
:109dc000f0de2adcef07fb41e80aee20ff0725164c
:109dd000f8cfc80fe81c200819e9dee4ded2dd0266
:109de0002cba32f3def4e124e5040a28de0e2c421c
:109df0000afff3ebe3ff311def1ce50af5ec010769
:109e000000e220f0daede835f7040d15fef7f41b5b
:109e1000f0f0e5f9f5f7171ef1eafee2d0dd03ec0c
:109e200005d845f3b105dd33e2ef023804fbf01845
:109e30000c0509e2f9ed1203051a02dde5dcf2f387
:109e4000faddffe8cae3f030d1f2fa0c35103e1922
:109e50002708d9dae8ec140624fffcfee2f6f70145
:109e600008e80df9ceff1707c415f1152e2a171aa9
:109e7000fd0b03c6f3fffa041cf10118c6f5e23b23
:109e8000feed1f03b61fe30ae911e80921102c1c9f
:109e90000206e0eadcf2060600ccf402defbf5186e
:109ea00040c21a11e908001bdd190c03020729e75b
:109eb000e201dad8d6e7120700d606f1eceb09008a
:109ec0000ff63120bef3e62efe2ff92ef8000bf12f
:109ed000e01eeb1d04ff2ef5fac8fcfbfbe8ef1ead
:109ee0003be73b29f60bf83b02fef506f7fa0a15ad
:109ef000e50717ea05fc29e1050a11fafd10f41837
:109f0000f9fcd014f9fe111b0406ec1a11d020e85c
:109f1000e90d06e8f5fcf6da0b00fe18da190d0972
:109f2000fdf6cc0efdfbe8d7ee0de615f0d7e1d23d
:109f30000a1217ecd906dfeb13fdf008f2050c0e40
:109f40000307d31bd9f8f40de413c72100d3f0fea7
:109f50001fedd3f4d107f1df2518ff15e102f5035a
:109f600014cde4fb0f03f1d8e515ed21e7fffff079
:109f7000faf3d1f0b3c8dbd90fee071215ddda0f13
:109f8000e8efe7eae212ee0b27f7aad3eef410d6d9
:109f9000df03f1f5ca10e9fc04fce50af50fda0d60
:109fa000efcce20df3ff19e20216aa030306d2df9b
:109fb000fc2419f0b202aeb410f3e7e9d006023582
:109fc00007ebd4fcdf0832ec00f195f31300cae094
:109fd00015b8f1f7a825aba90b17fa04fd06cb0bb2
:109fe000ead0cdf5eb1519d3e70aba121800e00450
:109ff00004d20310c025d8b01613feffe832e2f8f1
:10a000000809d3fa0cecfcdd0a26ba02f5e8c4ec28
:10a010000712f4fadd06e0cd02f4200bfc28e71469
:10a02000effec20e1318f6d20ce9e5002ef9cd0ea4
:10a030001e161d08e92ff8c60bda0f0318feff03e2
:10a04000f6feeb161c18e8db24eb0deb1deaec0c1e
:10a0500000320a05fc06f5d00cd314fb18fd0000f5
:10a06000ef21051025eafae710f1fdfbd3e4e20c3d
:10a07000f9210cfef31aeee8e1eb12fb1b170efac6
:10a08000e303edfb34de0bee0cd514e7c3dff5156f
:10a090000325000d303ef1e4e1041fdb22020ebe79
:10a0a000cb22cff513f5f9cbfdbf1f27d9efe9fd83
:10a0b0000517f70e2b21f6eee81d0d1d1305efcc4d
:10a0c000c815cefb1427fbe504dc19cdffdcf50d2c
:10a0d000f51af5061e0afe0be106130f2605080405
:10a0e000d812f8edfde101ec13e71cc4e7f2082af1
:10a0f000101f0015f5390119efee29f8190d0405a7
:10a10000d816d9061bc305f710dadacceaff1126f8
:10a11000082005ca0ce8f600f404220013000ed64d
:10a12000e1eafa10f80405f400ea2fee1107e51a47
:10a13000110205fc1df90716fff725f22bfb08f5a8
:10a1400009160a19080e0beeff072bd611f81ebfd1
:10a15000e7260cb426e91a36e610e9fbfcee1513e7
:10a160002406e3fbeffef10ad13111e21107f0f30f
:10a170000bfacffa32fe2617f8c3ecfad69dedf4af
:10a1800004c73d301216dd199ca1000094a1000007
:10a1900000000000010000000000000001000000bd
:10a1a0002bfa133a01000000040000000000000038
:10a1b00025000000a2ffffffcaffffff5e000000b6
:10a1c000d4a10000cca100000000000001000000ac
:10a1d0000000000001000000571e3039010000009f
:10a1e0004000000000000000b201000084010000f7
:10a1f0005d0000001301000076010000bb000000bc
:10a2000074ffffffe9ffffffe8ffffff31feffffe5
:10a2100092fdffffe2010000b1000000e8feffff39
:10a220007300000026feffffbcfefffff2fdfffff4
:10a2300078000000c90100005d01000000feffff82
:10a24000fcfcffffb7fcffff93fefffff1feffffeb
:10a25000a0ffffff4603000080000000c1000000d7
:10a260006bfeffffff00000020000000aefeffffbe
:10a27000df00000073010000abfdffff4cffffff9c
:10a2800082ffffff9200000047ffffff52feffff2b
:10a29000e1feffffcbfdffff44ffffff1dffffffc0
:10a2a0001f020000a3fffffff9000000d9ffffff1e
:10a2b0005bfeffff55ffffff43ffffff8afdffff30
:10a2c000c3fdffff43feffff00010000cbffffffc8
:10a2d0005afdffff43feffffd0feffffec00000032
:10a2e0000801000056fefffffca20000f4a20000df
:10a2f000000000000100000000000000010000005c
:10a30000cf132f3b010000002000000000000000e0
:10a31000be6c02091b43d4ab0c0ac4e2eccc9ed643
:10a320007ffef41ffaf304403cfef530e77de4bd08
:10a3300044a300003ca30000000000000100000056
:10a3400000000000010000003682813b0100000097
:10a350001400000000000000c2b80f30d0ffbefaa9
:10a36000c1f12cdde6e7e881d809500801000000c2
:10a370000200000000000000ffffffff00020000dd
:10a3800094a300008ca30000000000000100000066
:10a39000010000000100000086355c3d0200000065
:08a3a0000100000000050000af
:020000040000fa
:10a3a8000000803f00000000ecff7f3fd40fc93a57
:10a3b800b1ff7f3fc70f493b4eff7f3fc1cb963b65
:10a3c800c4fe7f3f890fc93b13fe7f3f3053fb3be1
:10a3d80039fd7f3f59cb163c39fc7f3f02ed2f3cbe
:10a3e80011fb7f3f900e493cc1f97f3f0030623c32
:10a3f8004af87f3f4b517b3cacf67f3f38398a3c6b
:10a40800e6f47f3fb6c9963cf8f27f3f1c5aa33c5e
:10a41800e3f07f3f69eaaf3ca7ee7f3f9b7abc3c05
:10a4280043ec7f3fb00ac93cb8e97f3fa69ad53cc8
:10a4380005e77f3f7b2ae23c2be47f3f2dbaee3cc9
:10a4480029e17f3fb949fb3c00de7f3f90ec033dab
:10a45800afda7f3f2f340a3d37d77f3fb87b103db7
:10a4680098d37f3f2cc3163dd1cf7f3f880a1d3d2f
:10a47800e2cb7f3fcc51233dccc77f3ff698293da7
:10a488008fc37f3f07e02f3d2abf7f3ffc26363d25
:10a498009eba7f3fd56d3c3deab57f3f91b4423dc2
:10a4a8000fb17f3f2ffb483d0dac7f3faf414f3d84
:10a4b800e3a67f3f0e88553d91a17f3f4cce5b3d83
:10a4c800189c7f3f6814623d78967f3f625a683dca
:10a4d800b1907f3f38a06e3dc28a7f3fe9e5743d69
:10a4e800ab847f3f742b7b3d6d7e7f3f6cb8803d96
:10a4f80008787f3f0adb833d7b717f3f94fd863d73
:10a50800c76a7f3f0a208a3dec637f3f6a428d3de0
:10a51800e95c7f3fb464903dbf557f3fe786933d3c
:10a528006d4e7f3f05a9963df4467f3f0acb993d86
:10a53800543f7f3ff9ec9c3d8d377f3fcf0ea03dc8
:10a548009d2f7f3f8c30a33d87277f3f3052a63d0c
:10a55800491f7f3fba73a93de4167f3f2b95ac3d59
:10a56800580e7f3f80b6af3da4057f3fbbd7b23db5
:10a57800c9fc7e3fdaf8b53dc7f37e3fdd19b93d2a
:10a588009dea7e3fc33abc3d4ce17e3f8d5bbf3dbb
:10a59800d4d77e3f397cc23d34ce7e3fc69cc53d74
:10a5a8006dc47e3f36bdc83d7fba7e3f86ddcb3d5c
:10a5b80069b07e3fb7fdce3d2da67e3fc81dd23d7a
:10a5c800c99b7e3fb93dd53d3d917e3f895dd83dd4
:10a5d8008b867e3f377ddb3db17b7e3fc49cde3d75
:10a5e800b0707e3f2ebce13d88657e3f76dbe43d62
:10a5f800385a7e3f9afae73dc14e7e3f9a19eb3da5
:10a6080023437e3f7638ee3d5e377e3f2e57f13d41
:10a61800722b7e3fc075f43d5e1f7e3f2c94f73d44
:10a6280024137e3f73b2fa3dc2067e3f92d0fd3db1
:10a6380038fa7d3f4577003e88ed7d3f2e06023e85
:10a64800b1e07d3f0295033eb2d37d3fc223053e74
:10a658008cc67d3f6eb2063e40b97d3f0541083e3f
:10a66800ccab7d3f86cf093e309e7d3ff35d0b3ef0
:10a678006e907d3f4aec0c3e85827d3f8b7a0e3e84
:10a6880074747d3fb708103e3d667d3fcc96113e01
:10a69800de577d3fca24133e59497d3fb2b2143e6e
:10a6a800ac3a7d3f8340163ed82b7d3f3dce173eca
:10a6b800dd1c7d3fe05b193ebc0d7d3f6be91a3e1a
:10a6c80073fe7c3fde761c3e03ef7c3f38041e3e63
:10a6d8006cdf7c3f7b911f3eaecf7c3fa51e213ea9
:10a6e800c9bf7c3fb6ab223ebdaf7c3fad38243ef0
:10a6f8008a9f7c3f8cc5253e318f7c3f5152273e37
:10a70800b07e7c3ffcde283e086e7c3f8d6b2a3e87
:10a718003a5d7c3f04f82b3e444c7c3f61842d3edf
:10a72800283b7c3fa2102f3ee5297c3fc99c303e48
:10a738007a187c3fd428323ee9067c3fc4b4333ec5
:10a7480031f57b3f9840353e53e37b3f50cc363e56
:10a758004dd17b3fec57383e20bf7b3f6ce3393e01
:10a76800cdac7b3fcf6e3b3e539a7b3f15fa3c3ec8
:10a77800b2877b3f3e853e3eea747b3f4910403eb0
:10a78800fc617b3f379b413ee74e7b3f0726433ebc
:10a79800ab3b7b3fb9b0443e48287b3f4d3b463ef0
:10a7a800be147b3fc2c5473e0e017b3f1850493e51
:10a7b80037ed7a3f4fda4a3e3ad97a3f67644c3ee2
:10a7c80016c57a3f60ee4d3ecbb07a3f38784f3ea3
:10a7d800599c7a3ff101513ec1877a3f898b523e9d
:10a7e80002737a3f0115543e1c5e7a3f589e553ecf
:10a7f80010497a3f8f27573edd337a3fa4b0583e41
:10a80800841e7a3f97395a3e04097a3f6ac25b3ef2
:10a818005ef3793f1a4b5d3e91dd793fa8d35e3eea
:10a828009dc7793f135c603e83b1793f5ce4613e2c
:10a83800439b793f836c633edc84793f86f4643eb6
:10a848004e6e793f667c663e9a57793f2204683e91
:10a85800c040793fba8b693ebf29793f2f136b3ec1
:10a868009812793f7f9a6c3e4afb783fab216e3e47
:10a87800d6e3783fb2a86f3e3bcc783f942f713e29
:10a888007bb4783f51b6723e939c783fe83c743e67
:10a898008684783f5ac3753e526c783fa649773e06
:10a8a800f853783fcccf783e773b783fcb557a3e0c
:10a8b800d122783fa4db7b3e040a783f56617d3e77
:10a8c80010f1773fe1e67e3ef7d7773f2236803eac
:10a8d800b7be773fc0f8803e51a5773f4abb813e5f
:10a8e800c58b773fc07d823e1372773f2240833eff
:10a8f8003a58773f7002843e3c3e773faac4843e74
:10a908001724773fce86853ecc09773fdf48863ec1
:10a918005bef763fda0a873ec4d4763fc1cc873ee8
:10a9280007ba763f938e883e249f763f5050893ee3
:10a938001b84763ff8118a3eec68763f8ad38a3ebc
:10a94800974d763f07958b3e1b32763f6e568c3e71
:10a958007a16763fc0178d3eb3fa753ffcd88d3e08
:10a96800c6de753f229a8e3eb3c2753f325b8f3e7c
:10a978007ba6753f2c1c903e1c8a753f10dd903ecf
:10a98800976d753fdd9d913eed50753f945e923e0b
:10a998001d34753f351f933e2717753fbfdf933e24
:10a9a8000bfa743f31a0943ec9dc743f8d60953e2c
:10a9b80062bf743fd220963ed5a1743f00e1963e17
:10a9c8002284743f17a1973e4966743f1661983eea
:10a9d8004b48743ffe20993e272a743fcee0993eab
:10a9e800dd0b743f86a09a3e6eed733f27609b3e59
:10a9f800d9ce733faf1f9c3e1fb0733f20df9c3ef4
:10aa08003f91733f789e9d3e3972733fb85d9e3e7d
:10aa18000e53733fdf1c9f3ebe33733feedb9f3efa
:10aa28004714733fe59aa03eacf4723fc259a13e69
:10aa3800ebd4723f8718a23e04b5723f33d7a23ecb
:10aa4800f894723fc595a33ec774723f3f54a43e25
:10aa58007054723f9f12a53ef433723fe5d0a53e75
:10aa68005213723f128fa63e8cf2713f254da73ebe
:10aa78009fd1713f1f0ba83e8eb0713ffec8a83e04
:10aa8800578f713fc486a93efb6d713f6f44aa3e44
:10aa98007a4c713f0102ab3ed42a713f77bfab3e7f
:10aaa8000809713fd47cac3e17e7703f153aad3ebc
:10aab80002c5703f3cf7ad3ec6a2703f49b4ae3efa
:10aac8006680703f3a71af3ee15d703f102eb03e38
:10aad800373b703fcbeab03e6718703f6ba7b13e7b
:10aae80073f56f3fef63b23e5ad26f3f5820b33ec3
:10aaf8001baf6f3fa5dcb33eb88b6f3fd698b43e13
:10ab080030686f3fec54b53e83446f3fe610b63e65
:10ab1800b0206f3fc3ccb63ebafc6e3f8488b73ec8
:10ab28009ed86e3f2a44b83e5db46e3fb2ffb83e31
:10ab3800f88f6e3f1ebbb93e6d6b6e3f6e76ba3ea8
:10ab4800be466e3fa031bb3eeb216e3fb6ecbb3e2e
:10ab5800f2fc6d3fafa7bc3ed5d76d3f8b62bd3ec3
:10ab680093b26d3f4a1dbe3e2d8d6d3febd7be3e65
:10ab7800a1676d3f6f92bf3ef2416d3fd54cc03e1d
:10ab88001d1c6d3f1e07c13e24f66c3f48c1c13ee7
:10ab980007d06c3f557bc23ec5a96c3f4435c33ec8
:10aba8005e836c3f15efc33ed45c6c3fc8a8c43ebf
:10abb80024366c3f5c62c53e500f6c3fd21bc63ecc
:10abc80058e86b3f29d5c63e3bc16b3f628ec73ef6
:10abd800fb996b3f7c47c83e95726b3f7700c93e37
:10abe8000c4b6b3f53b9c93e5e236b3f1072ca3e94
:10abf8008cfb6a3fae2acb3e95d36a3f2ce3cb3e13
:10ac08007bab6a3f8b9bcc3e3c836a3fca53cd3ead
:10ac1800d95a6a3fea0bce3e52326a3feac3ce3e69
:10ac2800a7096a3fca7bcf3ed7e0693f8a33d03e47
:10ac3800e4b7693f2aebd03ecc8e693faaa2d13e49
:10ac48009165693f095ad23e323c693f4811d33e6b
:10ac5800ae12693f67c8d33e07e9683f647fd43eb8
:10ac68003cbf683f4136d53e4c95683ffdecd53e2c
:10ac7800396b683f99a3d63e0341683f135ad73ec4
:10ac8800a816683f6b10d83e2aec673fa3c6d83e8b
:10ac980087c1673fb97cd93ec196673fad32da3e7e
:10aca800d86b673f80e8da3eca40673f319edb3e9b
:10acb8009915673fc153dc3e45ea663f2e09dd3ee4
:10acc800ccbe663f79bedd3e3093663fa273de3e62
:10acd8007167663fa928df3e8e3b663f8ddddf3e0c
:10ace800880f663f4f92e03e5ee3653fee46e13ee9
:10acf80010b7653f6afbe13ea08a653fc4afe23efc
:10ad08000b5e653ffa63e33e5431653f0e18e43e3f
:10ad18007904653ffecbe43e7bd7643fcb7fe53ebd
:10ad280059aa643f7533e63e147d643ffbe6e63e70
:10ad3800ac4f643f5d9ae73e2122643f9c4de83e5c
:10ad480073f4633fb700e93ea1c6633faeb3e93e83
:10ad5800ac98633f8166ea3e956a633f3019eb3ee3
:10ad68005a3c633fbbcbeb3efc0d633f217eec3e80
:10ad78007bdf623f6330ed3ed7b0623f80e2ed3e5d
:10ad88001082623f7994ee3e2653623f4c46ef3e76
:10ad98001a24623ffbf7ef3eeaf4613f85a9f03ed3
:10ada80098c5613fea5af13e2296613f290cf23e6e
:10adb8008a66613f43bdf23ed036613f386ef33e4e
:10adc800f206613f071ff43ef2d6603fb1cff43e72
:10add800cfa6603f3580f53e8976603f9330f63eda
:10ade8002146603fcbe0f63e9615603fdc90f73e8b
:10adf800e9e45f3fc840f83e19b45f3f8ef0f83e83
:10ae080027835f3f2da0f93e12525f3fa54ffa3ec0
:10ae1800db205f3ff7fefa3e81ef5e3f22aefb3e4e
:10ae280005be5e3f275dfc3e678c5e3f040cfd3e21
:10ae3800a65a5e3fbbbafd3ec3285e3f4a69fe3e46
:10ae4800bef65d3fb217ff3e97c45d3ff3c5ff3eb8
:10ae58004d925d3f063a003fe15f5d3fff90003f46
:10ae6800532d5d3fe4e7003fa3fa5c3fb53e013f49
:10ae7800d1c75c3f7395013fdd945c3f1cec013ffb
:10ae8800c7615c3fb142023f8e2e5c3f3299023f60
:10ae980034fb5b3f9fef023fb8c75b3ff845033f7a
:10aea8001a945b3f3d9c033f5a605b3f6df2033f42
:10aeb800792c5b3f8948043f75f85a3f919e043fbf
:10aec80050c45a3f84f4043f09905a3f624a053ff0
:10aed800a05b5a3f2ca0053f16275a3fe2f5053fd5
:10aee8006af2593f824b063f9cbd593f0ea1063f6f
:10aef800ad88593f86f6063f9c53593fe84b073fbc
:10af08006a1e593f36a1073f17e9583f6ff6073fba
:10af1800a1b3583f924b083f0b7e583fa1a0083f72
:10af28005348583f9bf5083f7912583f7f4a093fdd
:10af38007fdc573f4e9f093f63a6573f09f4093fff
:10af48002670573fad480a3fc739573f3d9d0a3fd6
:10af58004803573fb7f10a3fa7cc563f1c460b3f63
:10af6800e595563f6b9a0b3f025f563fa5ee0b3fa8
:10af7800fe27563fc9420c3fd9f0553fd7960c3fa4
:10af880093b9553fd0ea0c3f2c82553fb33e0d3f55
:10af9800a44a553f81920d3ffb12553f38e60d3fbd
:10afa80031db543fda390e3f47a3543f658d0e3fde
:10afb8003b6b543fdbe00e3f0f33543f3b340f3fb6
:10afc800c3fa533f84870f3f55c2533fb8da0f3f48
:10afd800c789533fd52d103f1851533fdc80103f90
:10afe8004918533fcdd3103f59df523fa726113f91
:10aff80049a6523f6b79113f186d523f19cc113f4a
:10b00800c633523fb01e123f54fa513f3071123fbf
:10b01800c2c0513f9ac3123f1087513fee15133fec
:10b028003d4d513f2a68133f4a13513f50ba133fd1
:10b0380037d9503f5f0c143f039f503f585e143f71
:10b04800af64503f39b0143f3b2a503f0402153fcc
:10b05800a8ef4f3fb753153ff4b44f3f54a5153fe2
:10b068001f7a4f3fd9f6153f2b3f4f3f4748163fb2
:10b0780017044f3f9f99163fe4c84e3fdfea163f3b
:10b08800908d4e3f073c173f1c524e3f188d173f7f
:10b0980089164e3f12de173fd5da4d3ff52e183f81
:10b0a800029f4d3fc07f183f10634d3f73d0183f3c
:10b0b800fd264d3f0f21193fcbea4c3f9471193fb4
:10b0c80079ae4c3f00c2193f08724c3f55121a3fe7
:10b0d80078354c3f93621a3fc7f84b3fb8b21a3fd6
:10b0e800f8bb4b3fc6021b3f097f4b3fbb521b3f80
:10b0f800fa414b3f99a21b3fcc044b3f5ff21b3fe9
:10b108007fc74a3f0c421c3f138a4a3fa2911c3f0b
:10b11800874c4a3f1fe11c3fdc0e4a3f84301d3fed
:10b1280012d1493fd17f1d3f2993493f06cf1d3f8b
:10b138002155493f221e1e3ffa16493f266d1e3fe4
:10b14800b3d8483f12bc1e3f4e9a483fe50a1f3ffe
:10b15800ca5b483f9f591f3f271d483f41a81f3fd3
:10b1680065de473fcbf61f3f849f473f3b45203f67
:10b178008560473f9393203f6721473fd2e1203fb7
:10b188002ae2463ff92f213fcea2463f067e213fc5
:10b198005463463ffbcb213fbb23463fd719223f91
:10b1a80003e4453f9967223f2da4453f43b5223f1d
:10b1b8003964453fd302233f2624453f4b50233f64
:10b1c800f5e3443fa99d233fa5a3443feeea233f6f
:10b1d8003763443f1a38243fab22443f2c85243f31
:10b1e80000e2433f25d2243f38a1433f041f253fb7
:10b1f8005160433fcb6b253f4c1f433f77b8253ffa
:10b2080029de423f0a05263fe89c423f8451263ffb
:10b21800895b423fe39d263f0b1a423f2aea263fbd
:10b2280070d8413f5636273fb796413f6882273f3f
:10b23800e154413f61ce273fec12413f401a283f7d
:10b24800dad0403f0566283fa98e403fb0b1283f7d
:10b258005c4c403f41fd283ff009403fb848293f3a
:10b2680067c73f3f1594293fc0843f3f57df293fb9
:10b27800fc413f3f802a2a3f1bff3e3f8e752a3ff5
:10b288001bbc3e3f82c02a3fff783e3f5b0b2b3ff3
:10b29800c5353e3f1b562b3f6ef23d3fbfa02b3faf
:10b2a800f9ae3d3f4aeb2b3f676b3d3fb9352c3f2d
:10b2b800b8273d3f0f802c3fece33c3f49ca2c3f69
:10b2c80003a03c3f69142d3ffc5b3c3f6f5e2d3f64
:10b2d800d9173c3f59a82d3f98d33b3f29f22d3f22
:10b2e8003b8f3b3fde3b2e3fc14a3b3f78852e3f9d
:10b2f80029063b3ff7ce2e3f75c13a3f5b182f3fdb
:10b30800a47c3a3fa5612f3fb7373a3fd3aa2f3fd6
:10b31800acf2393fe6f32f3f85ad393fde3c303f95
:10b328004268393fbb85303fe122393f7cce303f10
:10b3380065dd383f2217313fcb97383fad5f313f4e
:10b348001652383f1da8313f430c383f71f0313f4a
:10b3580055c6373faa38323f4a80373fc780323f09
:10b36800233a373fc9c8323fdff3363faf10333f88
:10b378007fad363f7a58333f0467363f29a0333fc5
:10b388006c20363fbce7333fb8d9353f342f343fc4
:10b39800e792353f8f76343ffb4b353fcfbd343f87
:10b3a800f304353ff304353fcfbd343ffb4b353f06
:10b3b8008f76343fe792353f342f343fb8d9353f45
:10b3c800bce7333f6c20363f29a0333f0467363f44
:10b3d8007a58333f7fad363faf10333fdff3363f08
:10b3e800c9c8323f233a373fc780323f4a80373f88
:10b3f800aa38323f55c6373f71f0313f430c383fca
:10b408001da8313f1652383fad5f313fcb97383fcb
:10b418002217313f65dd383f7cce303fe122393f8e
:10b42800bb85303f4268393fde3c303f85ad393f10
:10b43800e6f32f3facf2393fd3aa2f3fb7373a3f55
:10b44800a5612f3fa47c3a3f5b182f3f75c13a3f57
:10b45800f7ce2e3f29063b3f78852e3fc14a3b3f1a
:10b46800de3b2e3f3b8f3b3f29f22d3f98d33b3f9e
:10b4780059a82d3fd9173c3f6f5e2d3ffc5b3c3fe1
:10b4880069142d3f03a03c3f49ca2c3fece33c3fe5
:10b498000f802c3fb8273d3fb9352c3f676b3d3fa8
:10b4a8004aeb2b3ff9ae3d3fbfa02b3f6ef23d3f2d
:10b4b8001b562b3fc5353e3f5b0b2b3fff783e3f6e
:10b4c80082c02a3f1bbc3e3f8e752a3f1bff3e3f72
:10b4d800802a2a3ffc413f3f57df293fc0843f3f36
:10b4e8001594293f67c73f3fb848293ff009403fb7
:10b4f80041fd283f5c4c403fb0b1283fa98e403ffa
:10b508000566283fdad0403f401a283fec12413ff9
:10b5180061ce273fe154413f6882273fb796413fbc
:10b528005636273f70d8413f2aea263f0b1a423f3a
:10b53800e39d263f895b423f8451263fe89c423f7a
:10b548000a05263f29de423f77b8253f4c1f433f77
:10b55800cb6b253f5160433f041f253f38a1433f34
:10b5680025d2243f00e2433f2c85243fab22443fb1
:10b578001a38243f3763443feeea233fa5a3443fec
:10b58800a99d233ff5e3443f4b50233f2624453fe5
:10b59800d302233f3964453f43b5223f2da4453f9d
:10b5a8009967223f03e4453fd719223fbb23463f13
:10b5b800fbcb213f5463463f067e213fcea2463f48
:10b5c800f92f213f2ae2463fd2e1203f6721473f3a
:10b5d8009393203f8560473f3b45203f849f473feb
:10b5e800cbf61f3f65de473f41a81f3f271d483f59
:10b5f8009f591f3fca5b483fe50a1f3f4e9a483f85
:10b6080012bc1e3fb3d8483f266d1e3ffa16493f6d
:10b61800221e1e3f2155493f06cf1d3f2993493f12
:10b62800d17f1d3f12d1493f84301d3fdc0e4a3f78
:10b638001fe11c3f874c4a3fa2911c3f138a4a3f97
:10b648000c421c3f7fc74a3f5ff21b3fcc044b3f75
:10b6580099a21b3ffa414b3fbb521b3f097f4b3f0f
:10b66800c6021b3ff8bb4b3fb8b21a3fc7f84b3f67
:10b6780093621a3f78354c3f55121a3f08724c3f77
:10b6880000c2193f79ae4c3f9471193fcbea4c3f49
:10b698000f21193ffd264d3f73d0183f10634d3fd2
:10b6a800c07f183f029f4d3ff52e183fd5da4d3f1a
:10b6b80012de173f89164e3f188d173f1c524e3f1a
:10b6c800073c173f908d4e3fdfea163fe4c84e3fd8
:10b6d8009f99163f17044f3f4748163f2b3f4f3f50
:10b6e800d9f6153f1f7a4f3f54a5153ff4b44f3f85
:10b6f800b753153fa8ef4f3f0402153f3b2a503f71
:10b7080039b0143faf64503f585e143f039f503f19
:10b718005f0c143f37d9503f50ba133f4a13513f7b
:10b728002a68133f3d4d513fee15133f1087513f97
:10b738009ac3123fc2c0513f3071123f54fa513f71
:10b74800b01e123fc633523f19cc113f186d523ffd
:10b758006b79113f49a6523fa726113f59df523f47
:10b76800cdd3103f4918533fdc80103f1851533f49
:10b77800d52d103fc789533fb8da0f3f55c2533f05
:10b7880084870f3fc3fa533f3b340f3f0f33543f77
:10b79800dbe00e3f3b6b543f658d0e3f47a3543fa4
:10b7a800da390e3f31db543f38e60d3ffb12553f87
:10b7b80081920d3fa44a553fb33e0d3f2c82553f21
:10b7c800d0ea0c3f93b9553fd7960c3fd9f0553f77
:10b7d800c9420c3ffe27563fa5ee0b3f025f563f7e
:10b7e8006b9a0b3fe595563f1c460b3fa7cc563f3f
:10b7f800b7f10a3f4803573f3d9d0a3fc739573fb6
:10b80800ad480a3f2670573f09f4093f63a6573fe2
:10b818004e9f093f7fdc573f7f4a093f7912583fc7
:10b828009bf5083f5348583fa1a0083f0b7e583f5f
:10b83800924b083fa1b3583f6ff6073f17e9583faf
:10b8480036a1073f6a1e593fe84b073f9c53593fb3
:10b8580086f6063fad88593f0ea1063f9cbd593f6d
:10b86800824b063f6af2593fe2f5053f16275a3fd9
:10b878002ca0053fa05b5a3f624a053f09905a3ffa
:10b8880084f4043f50c45a3f919e043f75f85a3fd0
:10b898008948043f792c5b3f6df2033f5a605b3f58
:10b8a8003d9c033f1a945b3ff845033fb8c75b3f95
:10b8b8009fef023f34fb5b3f3299023f8e2e5c3f85
:10b8c800b142023fc7615c3f1cec013fdd945c3f25
:10b8d8007395013fd1c75c3fb53e013fa3fa5c3f7a
:10b8e800e4e7003f532d5d3fff90003fe15f5d3f80
:10b8f800063a003f4d925d3ff3c5ff3e97c45d3f5a
:10b90800b217ff3ebef65d3f4a69fe3ec3285e3f62
:10b91800bbbafd3ea65a5e3f040cfd3e678c5e3ff7
:10b92800275dfc3e05be5e3f22aefb3e81ef5e3fdb
:10b93800f7fefa3edb205f3fa54ffa3e12525f3f0b
:10b948002da0f93e27835f3f8ef0f83e19b45f3f84
:10b95800c840f83ee9e45f3fdc90f73e9615603f4b
:10b96800cbe0f63e2146603f9330f63e8976603f55
:10b978003580f53ecfa6603fb1cff43ef2d6603faa
:10b98800071ff43ef206613f386ef33ed036613f42
:10b9980043bdf23e8a66613f290cf23e2296613f22
:10b9a800ea5af13e98c5613f85a9f03eeaf4613f45
:10b9b800fbf7ef3e1a24623f4c46ef3e2653623fa8
:10b9c8007994ee3e1082623f80e2ed3ed7b0623f4e
:10b9d8006330ed3e7bdf623f217eec3efc0d633f32
:10b9e800bbcbeb3e5a3c633f3019eb3e956a633f55
:10b9f8008166ea3eac98633faeb3e93ea1c6633fb9
:10ba0800b700e93e73f4633f9c4de83e2122643f52
:10ba18005d9ae73eac4f643ffbe6e63e147d643f2b
:10ba28007533e63e59aa643fcb7fe53e7bd7643f3a
:10ba3800fecbe43e7904653f0e18e43e5431653f81
:10ba4800fa63e33e0b5e653fc4afe23ea08a653f02
:10ba58006afbe13e10b7653fee46e13e5ee3653fb7
:10ba68004f92e03e880f663f8ddddf3e8e3b663f9e
:10ba7800a928df3e7167663fa273de3e3093663fba
:10ba880079bedd3eccbe663f2e09dd3e45ea663f07
:10ba9800c153dc3e9915673f319edb3eca40673f84
:10baa80080e8da3ed86b673fad32da3ec196673f31
:10bab800b97cd93e87c1673fa3c6d83e2aec673f09
:10bac8006b10d83ea816683f135ad73e0341683f0b
:10bad80099a3d63e396b683ffdecd53e4c95683f3f
:10bae8004136d53e3cbf683f647fd43e07e9683f96
:10baf80067c8d33eae12693f4811d33e323c693f16
:10bb0800095ad23e9165693faaa2d13ecc8e693fbf
:10bb18002aebd03ee4b7693f8a33d03ed7e0693f8d
:10bb2800ca7bcf3ea7096a3feac3ce3e52326a3f7c
:10bb3800ea0bce3ed95a6a3fca53cd3e3c836a3f90
:10bb48008b9bcc3e7bab6a3f2ce3cb3e95d36a3fc5
:10bb5800ae2acb3e8cfb6a3f1072ca3e5e236b3f17
:10bb680053b9c93e0c4b6b3f7700c93e95726b3f8a
:10bb78007c47c83efb996b3f628ec73e3bc16b3f1b
:10bb880029d5c63e58e86b3fd21bc63e500f6c3fc6
:10bb98005c62c53e24366c3fc8a8c43ed45c6c3f8a
:10bba80015efc33e5e836c3f4435c33ec5a96c3f69
:10bbb800557bc23e07d06c3f48c1c13e24f66c3f5e
:10bbc8001e07c13e1d1c6d3fd54cc03ef2416d3f66
:10bbd8006f92bf3ea1676d3febd7be3e2d8d6d3f87
:10bbe8004a1dbe3e93b26d3f8b62bd3ed5d76d3fb9
:10bbf800afa7bc3ef2fc6d3fb6ecbb3eeb216e3fff
:10bc0800a031bb3ebe466e3f6e76ba3e6d6b6e3f50
:10bc18001ebbb93ef88f6e3fb2ffb83e5db46e3fb3
:10bc28002a44b83e9ed86e3f8488b73ebafc6e3f21
:10bc3800c3ccb63eb0206f3fe610b63e83446f3f9c
:10bc4800ec54b53e30686f3fd698b43eb88b6f3f22
:10bc5800a5dcb33e1baf6f3f5820b33e5ad26f3faf
:10bc6800ef63b23e73f56f3f6ba7b13e6718703f45
:10bc7800cbeab03e373b703f102eb03ee15d703fdf
:10bc88003a71af3e6680703f49b4ae3ec6a2703f7f
:10bc98003cf7ad3e02c5703f153aad3e17e7703f21
:10bca800d47cac3e0809713f77bfab3ed42a713fc4
:10bcb8000102ab3e7a4c713f6f44aa3efb6d713f67
:10bcc800c486a93e578f713ffec8a83e8eb0713f0b
:10bcd8001f0ba83e9fd1713f254da73e8cf2713fa7
:10bce800128fa63e5213723fe5d0a53ef433723f41
:10bcf8009f12a53e7054723f3f54a43ec774723fd2
:10bd0800c595a33ef894723f33d7a23e04b5723f5f
:10bd18008718a23eebd4723fc259a13eacf4723fe1
:10bd2800e59aa03e4714733feedb9f3ebe33733f58
:10bd3800df1c9f3e0e53733fb85d9e3e3972733fc2
:10bd4800789e9d3e3f91733f20df9c3e1fb0733f1e
:10bd5800af1f9c3ed9ce733f27609b3e6eed733f6d
:10bd680086a09a3edd0b743fcee0993e272a743fa9
:10bd7800fe20993e4b48743f1661983e4966743fd1
:10bd880017a1973e2284743f00e1963ed5a1743fe7
:10bd9800d220963e62bf743f8d60953ec9dc743fe9
:10bda80031a0943e0bfa743fbfdf933e2717753fcf
:10bdb800351f933e1d34753f945e923eed50753f9e
:10bdc800dd9d913e976d753f10dd903e1c8a753f55
:10bdd8002c1c903e7ba6753f325b8f3eb3c2753fed
:10bde800229a8e3ec6de753ffcd88d3eb3fa753f6b
:10bdf800c0178d3e7a16763f6e568c3e1b32763fc4
:10be080007958b3e974d763f8ad38a3eec68763ffe
:10be1800f8118a3e1b84763f5050893e249f763f16
:10be2800938e883e07ba763fc1cc873ec4d4763f0e
:10be3800da0a873e5bef763fdf48863ecc09773fdc
:10be4800ce86853e1724773faac4843e3c3e773f82
:10be58007002843e3a58773f2240833e1372773f00
:10be6800c07d823ec58b773f4abb813e51a5773f57
:10be7800c0f8803eb7be773f2236803ef7d7773f7f
:10be8800e1e67e3e10f1773f56617d3e040a783f39
:10be9800a4db7b3ed122783fcb557a3e773b783f77
:10bea800cccf783ef853783fa649773e526c783f1e
:10beb8005ac3753e8684783fe83c743e939c783f2d
:10bec80051b6723e7bb4783f942f713e3bcc783f9d
:10bed800b2a86f3ed6e3783fab216e3e4afb783f6f
:10bee8007f9a6c3e9812793f2f136b3ebf29793f9a
:10bef800ba8b693ec040793f2204683e9a57793f21
:10bf0800667c663e4e6e793f86f4643edc84793ffb
:10bf1800836c633e439b793f5ce4613e83b1793f28
:10bf2800135c603e9dc7793fa8d35e3e91dd793fa3
:10bf38001a4b5d3e5ef3793f6ac25b3e04097a3f65
:10bf480097395a3e841e7a3fa4b0583edd337a3f73
:10bf58008f27573e10497a3f589e553e1c5e7a3fc0
:10bf68000115543e02737a3f898b523ec1877a3f4e
:10bf7800f101513e599c7a3f38784f3ecbb07a3f19
:10bf880060ee4d3e16c57a3f67644c3e3ad97a3f1b
:10bf98004fda4a3e37ed7a3f1850493e0e017b3f53
:10bfa800c2c5473ebe147b3f4d3b463e48287b3fbb
:10bfb800b9b0443eab3b7b3f0726433ee74e7b3f51
:10bfc800379b413efc617b3f4910403eea747b3f12
:10bfd8003e853e3eb2877b3f15fa3c3e539a7b3ff7
:10bfe800cf6e3b3ecdac7b3f6ce3393e20bf7b3f01
:10bff800ec57383e4dd17b3f50cc363e53e37b3f28
:10c008009840353e31f57b3fc4b4333ee9067c3f6a
:10c01800d428323e7a187c3fc99c303ee5297c3fc3
:10c02800a2102f3e283b7c3f61842d3e444c7c3f30
:10c0380004f82b3e3a5d7c3f8d6b2a3e086e7c3fb0
:10c04800fcde283eb07e7c3f5152273e318f7c3f3c
:10c058008cc5253e8a9f7c3fad38243ebdaf7c3fd2
:10c06800b6ab223ec9bf7c3fa51e213eaecf7c3f6a
:10c078007b911f3e6cdf7c3f38041e3e03ef7c3f04
:10c08800de761c3e73fe7c3f6be91a3ebc0d7d3f9d
:10c09800e05b193edd1c7d3f3dce173ed82b7d3f32
:10c0a8008340163eac3a7d3fb2b2143e59497d3fbb
:10c0b800ca24133ede577d3fcc96113e3d667d3f38
:10c0c800b708103e74747d3f8b7a0e3e85827d3fa3
:10c0d8004aec0c3e6e907d3ff35d0b3e309e7d3ffb
:10c0e80086cf093eccab7d3f0541083e40b97d3f38
:10c0f8006eb2063e8cc67d3fc223053eb2d37d3f5d
:10c108000295033eb1e07d3f2e06023e88ed7d3f5d
:10c118004577003e38fa7d3f92d0fd3dc2067e3f0e
:10c1280073b2fa3d24137e3f2c94f73d5e1f7e3f89
:10c13800c075f43d722b7e3f2e57f13d5e377e3f32
:10c148007638ee3d23437e3f9a19eb3dc14e7e3f44
:10c158009afae73d385a7e3f76dbe43d88657e3fb4
:10c168002ebce13db0707e3fc49cde3db17b7e3f7e
:10c17800377ddb3d8b867e3f895dd83d3d917e3f97
:10c18800b93dd53dc99b7e3fc81dd23d2da67e3ffa
:10c19800b7fdce3d69b07e3f86ddcb3d7fba7e3fa1
:10c1a80036bdc83d6dc47e3fc69cc53d34ce7e3f7e
:10c1b800397cc23dd4d77e3f8d5bbf3d4ce17e3f8d
:10c1c800c33abc3d9dea7e3fdd19b93dc7f37e3fca
:10c1d800daf8b53dc9fc7e3fbbd7b23da4057f3f29
:10c1e80080b6af3d580e7f3f2b95ac3de4167f3fa0
:10c1f800ba73a93d491f7f3f3052a63d87277f3f2d
:10c208008c30a33d9d2f7f3fcf0ea03d8d377f3fc4
:10c21800f9ec9c3d543f7f3f0acb993df4467f3f64
:10c2280005a9963d6d4e7f3fe786933dbf557f3ffd
:10c23800b464903de95c7f3f6a428d3dec637f3f8b
:10c248000a208a3dc76a7f3f94fd863d7b717f3f08
:10c258000adb833d08787f3f6cb8803d6d7e7f3f69
:10c26800742b7b3dab847f3fe9e5743dc28a7f3ff9
:10c2780038a06e3db1907f3f625a683d78967f3f07
:10c288006814623d189c7f3f4cce5b3d91a17f3f77
:10c298000e88553de3a67f3faf414f3d0dac7f3f34
:10c2a8002ffb483d0fb17f3f91b4423deab57f3f38
:10c2b800d56d3c3d9eba7f3ffc26363d2abf7f3f69
:10c2c80007e02f3d8fc37f3ff698293dccc77f3fbe
:10c2d800cc51233de2cb7f3f880a1d3dd1cf7f3f24
:10c2e8002cc3163d98d37f3fb87b103d37d77f3f8f
:10c2f8002f340a3dafda7f3f90ec033d00de7f3fed
:10c30800b949fb3c29e17f3f2dbaee3c2be47f3f46
:10c318007b2ae23c05e77f3fa69ad53cb8e97f3ff8
:10c32800b00ac93c43ec7f3f9b7abc3ca7ee7f3ff9
:10c3380069eaaf3ce3f07f3f1c5aa33cf8f27f3f29
:10c34800b6c9963ce6f47f3f38398a3cacf67f3f65
:10c358004b517b3c4af87f3f0030623cc1f97f3f3c
:10c36800900e493c11fb7f3f02ed2f3c39fc7f3f8b
:10c3780059cb163c39fd7f3f3053fb3b13fe7f3fc3
:10c38800890fc93bc4fe7f3fc1cb963b4eff7f3f21
:10c39800c70f493bb1ff7f3fd40fc93aecff7f3f3e
:10c3a800000000000000803fd40fc9baecff7f3fb7
:10c3b800c70f49bbb1ff7f3fc1cb96bb4eff7f3f45
:10c3c800890fc9bbc4fe7f3f3053fbbb13fe7f3fc1
:10c3d80059cb16bc39fd7f3f02ed2fbc39fc7f3f9e
:10c3e800900e49bc11fb7f3f003062bcc1f97f3f12
:10c3f8004b517bbc4af87f3f38398abcacf67f3f4b
:10c40800b6c996bce6f47f3f1c5aa3bcf8f27f3f3e
:10c4180069eaafbce3f07f3f9b7abcbca7ee7f3fe5
:10c42800b00ac9bc43ec7f3fa69ad5bcb8e97f3fa8
:10c438007b2ae2bc05e77f3f2dbaeebc2be47f3fa9
:10c44800b949fbbc29e17f3f90ec03bd00de7f3f8b
:10c458002f340abdafda7f3fb87b10bd37d77f3f97
:10c468002cc316bd98d37f3f880a1dbdd1cf7f3f0f
:10c47800cc5123bde2cb7f3ff69829bdccc77f3f87
:10c4880007e02fbd8fc37f3ffc2636bd2abf7f3f05
:10c49800d56d3cbd9eba7f3f91b442bdeab57f3fa2
:10c4a8002ffb48bd0fb17f3faf414fbd0dac7f3f64
:10c4b8000e8855bde3a67f3f4cce5bbd91a17f3f63
:10c4c800681462bd189c7f3f625a68bd78967f3faa
:10c4d80038a06ebdb1907f3fe9e574bdc28a7f3f49
:10c4e800742b7bbdab847f3f6cb880bd6d7e7f3f76
:10c4f8000adb83bd08787f3f94fd86bd7b717f3f53
:10c508000a208abdc76a7f3f6a428dbdec637f3fc0
:10c51800b46490bde95c7f3fe78693bdbf557f3f1c
:10c5280005a996bd6d4e7f3f0acb99bdf4467f3f66
:10c53800f9ec9cbd543f7f3fcf0ea0bd8d377f3fa8
:10c548008c30a3bd9d2f7f3f3052a6bd87277f3fec
:10c55800ba73a9bd491f7f3f2b95acbde4167f3f39
:10c5680080b6afbd580e7f3fbbd7b2bda4057f3f95
:10c57800daf8b5bdc9fc7e3fdd19b9bdc7f37e3f0a
:10c58800c33abcbd9dea7e3f8d5bbfbd4ce17e3f9b
:10c59800397cc2bdd4d77e3fc69cc5bd34ce7e3f54
:10c5a80036bdc8bd6dc47e3f86ddcbbd7fba7e3f3c
:10c5b800b7fdcebd69b07e3fc81dd2bd2da67e3f5a
:10c5c800b93dd5bdc99b7e3f895dd8bd3d917e3fb4
:10c5d800377ddbbd8b867e3fc49cdebdb17b7e3f55
:10c5e8002ebce1bdb0707e3f76dbe4bd88657e3f42
:10c5f8009afae7bd385a7e3f9a19ebbdc14e7e3f85
:10c608007638eebd23437e3f2e57f1bd5e377e3f21
:10c61800c075f4bd722b7e3f2c94f7bd5e1f7e3f24
:10c6280073b2fabd24137e3f92d0fdbdc2067e3f91
:10c63800457700be38fa7d3f2e0602be88ed7d3f65
:10c64800029503beb1e07d3fc22305beb2d37d3f54
:10c658006eb206be8cc67d3f054108be40b97d3f1f
:10c6680086cf09beccab7d3ff35d0bbe309e7d3fd0
:10c678004aec0cbe6e907d3f8b7a0ebe85827d3f64
:10c68800b70810be74747d3fcc9611be3d667d3fe1
:10c69800ca2413bede577d3fb2b214be59497d3f4e
:10c6a800834016beac3a7d3f3dce17bed82b7d3faa
:10c6b800e05b19bedd1c7d3f6be91abebc0d7d3ffa
:10c6c800de761cbe73fe7c3f38041ebe03ef7c3f43
:10c6d8007b911fbe6cdf7c3fa51e21beaecf7c3f89
:10c6e800b6ab22bec9bf7c3fad3824bebdaf7c3fd0
:10c6f8008cc525be8a9f7c3f515227be318f7c3f17
:10c70800fcde28beb07e7c3f8d6b2abe086e7c3f67
:10c7180004f82bbe3a5d7c3f61842dbe444c7c3fbf
:10c72800a2102fbe283b7c3fc99c30bee5297c3f28
:10c73800d42832be7a187c3fc4b433bee9067c3fa5
:10c74800984035be31f57b3f50cc36be53e37b3f36
:10c75800ec5738be4dd17b3f6ce339be20bf7b3fe1
:10c76800cf6e3bbecdac7b3f15fa3cbe539a7b3fa8
:10c778003e853ebeb2877b3f491040beea747b3f90
:10c78800379b41befc617b3f072643bee74e7b3f9c
:10c79800b9b044beab3b7b3f4d3b46be48287b3fd0
:10c7a800c2c547bebe147b3f185049be0e017b3f31
:10c7b8004fda4abe37ed7a3f67644cbe3ad97a3fc2
:10c7c80060ee4dbe16c57a3f38784fbecbb07a3f83
:10c7d800f10151be599c7a3f898b52bec1877a3f7d
:10c7e800011554be02737a3f589e55be1c5e7a3faf
:10c7f8008f2757be10497a3fa4b058bedd337a3f21
:10c8080097395abe841e7a3f6ac25bbe04097a3fd2
:10c818001a4b5dbe5ef3793fa8d35ebe91dd793fca
:10c82800135c60be9dc7793f5ce461be83b1793f0c
:10c83800836c63be439b793f86f464bedc84793f96
:10c84800667c66be4e6e793f220468be9a57793f71
:10c85800ba8b69bec040793f2f136bbebf29793fa1
:10c868007f9a6cbe9812793fab216ebe4afb783f27
:10c87800b2a86fbed6e3783f942f71be3bcc783f09
:10c8880051b672be7bb4783fe83c74be939c783f47
:10c898005ac375be8684783fa64977be526c783fe6
:10c8a800cccf78bef853783fcb557abe773b783fec
:10c8b800a4db7bbed122783f56617dbe040a783f57
:10c8c800e1e67ebe10f1773f223680bef7d7773f8c
:10c8d800c0f880beb7be773f4abb81be51a5773f3f
:10c8e800c07d82bec58b773f224083be1372773fdf
:10c8f800700284be3a58773faac484be3c3e773f54
:10c90800ce8685be1724773fdf4886becc09773fa1
:10c91800da0a87be5bef763fc1cc87bec4d4763fc8
:10c92800938e88be07ba763f505089be249f763fc3
:10c93800f8118abe1b84763f8ad38abeec68763f9c
:10c9480007958bbe974d763f6e568cbe1b32763f51
:10c95800c0178dbe7a16763ffcd88dbeb3fa753fe8
:10c96800229a8ebec6de753f325b8fbeb3c2753f5c
:10c978002c1c90be7ba6753f10dd90be1c8a753faf
:10c98800dd9d91be976d753f945e92beed50753feb
:10c99800351f93be1d34753fbfdf93be2717753f04
:10c9a80031a094be0bfa743f8d6095bec9dc743f0c
:10c9b800d22096be62bf743f00e196bed5a1743ff7
:10c9c80017a197be2284743f166198be4966743fca
:10c9d800fe2099be4b48743fcee099be272a743f8b
:10c9e80086a09abedd0b743f27609bbe6eed733f39
:10c9f800af1f9cbed9ce733f20df9cbe1fb0733fd4
:10ca0800789e9dbe3f91733fb85d9ebe3972733f5d
:10ca1800df1c9fbe0e53733feedb9fbebe33733fda
:10ca2800e59aa0be4714733fc259a1beacf4723f49
:10ca38008718a2beebd4723f33d7a2be04b5723fab
:10ca4800c595a3bef894723f3f54a4bec774723f05
:10ca58009f12a5be7054723fe5d0a5bef433723f55
:10ca6800128fa6be5213723f254da7be8cf2713f9e
:10ca78001f0ba8be9fd1713ffec8a8be8eb0713fe4
:10ca8800c486a9be578f713f6f44aabefb6d713f24
:10ca98000102abbe7a4c713f77bfabbed42a713f5f
:10caa800d47cacbe0809713f153aadbe17e7703f9c
:10cab8003cf7adbe02c5703f49b4aebec6a2703fda
:10cac8003a71afbe6680703f102eb0bee15d703f18
:10cad800cbeab0be373b703f6ba7b1be6718703f5b
:10cae800ef63b2be73f56f3f5820b3be5ad26f3fa3
:10caf800a5dcb3be1baf6f3fd698b4beb88b6f3ff3
:10cb0800ec54b5be30686f3fe610b6be83446f3f45
:10cb1800c3ccb6beb0206f3f8488b7bebafc6e3fa8
:10cb28002a44b8be9ed86e3fb2ffb8be5db46e3f11
:10cb38001ebbb9bef88f6e3f6e76babe6d6b6e3f88
:10cb4800a031bbbebe466e3fb6ecbbbeeb216e3f0e
:10cb5800afa7bcbef2fc6d3f8b62bdbed5d76d3fa3
:10cb68004a1dbebe93b26d3febd7bebe2d8d6d3f45
:10cb78006f92bfbea1676d3fd54cc0bef2416d3ffd
:10cb88001e07c1be1d1c6d3f48c1c1be24f66c3fc7
:10cb9800557bc2be07d06c3f4435c3bec5a96c3fa8
:10cba80015efc3be5e836c3fc8a8c4bed45c6c3f9f
:10cbb8005c62c5be24366c3fd21bc6be500f6c3fac
:10cbc80029d5c6be58e86b3f628ec7be3bc16b3fd6
:10cbd8007c47c8befb996b3f7700c9be95726b3f17
:10cbe80053b9c9be0c4b6b3f1072cabe5e236b3f74
:10cbf800ae2acbbe8cfb6a3f2ce3cbbe95d36a3ff3
:10cc08008b9bccbe7bab6a3fca53cdbe3c836a3f8d
:10cc1800ea0bcebed95a6a3feac3cebe52326a3f49
:10cc2800ca7bcfbea7096a3f8a33d0bed7e0693f27
:10cc38002aebd0bee4b7693faaa2d1becc8e693f29
:10cc4800095ad2be9165693f4811d3be323c693f4b
:10cc580067c8d3beae12693f647fd4be07e9683f98
:10cc68004136d5be3cbf683ffdecd5be4c95683f0c
:10cc780099a3d6be396b683f135ad7be0341683fa4
:10cc88006b10d8bea816683fa3c6d8be2aec673f6b
:10cc9800b97cd9be87c1673fad32dabec196673f5e
:10cca80080e8dabed86b673f319edbbeca40673f7b
:10ccb800c153dcbe9915673f2e09ddbe45ea663fc4
:10ccc80079beddbeccbe663fa273debe3093663f42
:10ccd800a928dfbe7167663f8ddddfbe8e3b663fec
:10cce8004f92e0be880f663fee46e1be5ee3653fc9
:10ccf8006afbe1be10b7653fc4afe2bea08a653fdc
:10cd0800fa63e3be0b5e653f0e18e4be5431653f1f
:10cd1800fecbe4be7904653fcb7fe5be7bd7643f9d
:10cd28007533e6be59aa643ffbe6e6be147d643f50
:10cd38005d9ae7beac4f643f9c4de8be2122643f3c
:10cd4800b700e9be73f4633faeb3e9bea1c6633f63
:10cd58008166eabeac98633f3019ebbe956a633fc3
:10cd6800bbcbebbe5a3c633f217eecbefc0d633f60
:10cd78006330edbe7bdf623f80e2edbed7b0623f3d
:10cd88007994eebe1082623f4c46efbe2653623f56
:10cd9800fbf7efbe1a24623f85a9f0beeaf4613fb3
:10cda800ea5af1be98c5613f290cf2be2296613f4e
:10cdb80043bdf2be8a66613f386ef3bed036613f2e
:10cdc800071ff4bef206613fb1cff4bef2d6603f52
:10cdd8003580f5becfa6603f9330f6be8976603fba
:10cde800cbe0f6be2146603fdc90f7be9615603f6b
:10cdf800c840f8bee9e45f3f8ef0f8be19b45f3f63
:10ce08002da0f9be27835f3fa54ffabe12525f3fa0
:10ce1800f7fefabedb205f3f22aefbbe81ef5e3f2e
:10ce2800275dfcbe05be5e3f040cfdbe678c5e3f01
:10ce3800bbbafdbea65a5e3f4a69febec3285e3f26
:10ce4800b217ffbebef65d3ff3c5ffbe97c45d3f98
:10ce5800063a00bf4d925d3fff9000bfe15f5d3f26
:10ce6800e4e700bf532d5d3fb53e01bfa3fa5c3f29
:10ce7800739501bfd1c75c3f1cec01bfdd945c3fdb
:10ce8800b14202bfc7615c3f329902bf8e2e5c3f40
:10ce98009fef02bf34fb5b3ff84503bfb8c75b3f5a
:10cea8003d9c03bf1a945b3f6df203bf5a605b3f22
:10ceb800894804bf792c5b3f919e04bf75f85a3f9f
:10cec80084f404bf50c45a3f624a05bf09905a3fd0
:10ced8002ca005bfa05b5a3fe2f505bf16275a3fb5
:10cee800824b06bf6af2593f0ea106bf9cbd593f4f
:10cef80086f606bfad88593fe84b07bf9c53593f9c
:10cf080036a107bf6a1e593f6ff607bf17e9583f9a
:10cf1800924b08bfa1b3583fa1a008bf0b7e583f52
:10cf28009bf508bf5348583f7f4a09bf7912583fbd
:10cf38004e9f09bf7fdc573f09f409bf63a6573fdf
:10cf4800ad480abf2670573f3d9d0abfc739573fb6
:10cf5800b7f10abf4803573f1c460bbfa7cc563f43
:10cf68006b9a0bbfe595563fa5ee0bbf025f563f88
:10cf7800c9420cbffe27563fd7960cbfd9f0553f84
:10cf8800d0ea0cbf93b9553fb33e0dbf2c82553f35
:10cf980081920dbfa44a553f38e60dbffb12553f9d
:10cfa800da390ebf31db543f658d0ebf47a3543fbe
:10cfb800dbe00ebf3b6b543f3b340fbf0f33543f96
:10cfc80084870fbfc3fa533fb8da0fbf55c2533f28
:10cfd800d52d10bfc789533fdc8010bf1851533f70
:10cfe800cdd310bf4918533fa72611bf59df523f71
:10cff8006b7911bf49a6523f19cc11bf186d523f2a
:10d00800b01e12bfc633523f307112bf54fa513f9f
:10d018009ac312bfc2c0513fee1513bf1087513fcc
:10d028002a6813bf3d4d513f50ba13bf4a13513fb1
:10d038005f0c14bf37d9503f585e14bf039f503f51
:10d0480039b014bfaf64503f040215bf3b2a503fac
:10d05800b75315bfa8ef4f3f54a515bff4b44f3fc2
:10d06800d9f615bf1f7a4f3f474816bf2b3f4f3f92
:10d078009f9916bf17044f3fdfea16bfe4c84e3f1b
:10d08800073c17bf908d4e3f188d17bf1c524e3f5f
:10d0980012de17bf89164e3ff52e18bfd5da4d3f61
:10d0a800c07f18bf029f4d3f73d018bf10634d3f1c
:10d0b8000f2119bffd264d3f947119bfcbea4c3f94
:10d0c80000c219bf79ae4c3f55121abf08724c3fc7
:10d0d80093621abf78354c3fb8b21abfc7f84b3fb6
:10d0e800c6021bbff8bb4b3fbb521bbf097f4b3f60
:10d0f80099a21bbffa414b3f5ff21bbfcc044b3fc9
:10d108000c421cbf7fc74a3fa2911cbf138a4a3feb
:10d118001fe11cbf874c4a3f84301dbfdc0e4a3fcd
:10d12800d17f1dbf12d1493f06cf1dbf2993493f6b
:10d13800221e1ebf2155493f266d1ebffa16493fc4
:10d1480012bc1ebfb3d8483fe50a1fbf4e9a483fde
:10d158009f591fbfca5b483f41a81fbf271d483fb3
:10d16800cbf61fbf65de473f3b4520bf849f473f47
:10d17800939320bf8560473fd2e120bf6721473f97
:10d18800f92f21bf2ae2463f067e21bfcea2463fa5
:10d19800fbcb21bf5463463fd71922bfbb23463f71
:10d1a800996722bf03e4453f43b522bf2da4453ffd
:10d1b800d30223bf3964453f4b5023bf2624453f44
:10d1c800a99d23bff5e3443feeea23bfa5a3443f4f
:10d1d8001a3824bf3763443f2c8524bfab22443f11
:10d1e80025d224bf00e2433f041f25bf38a1433f97
:10d1f800cb6b25bf5160433f77b825bf4c1f433fda
:10d208000a0526bf29de423f845126bfe89c423fdb
:10d21800e39d26bf895b423f2aea26bf0b1a423f9d
:10d22800563627bf70d8413f688227bfb796413f1f
:10d2380061ce27bfe154413f401a28bfec12413f5d
:10d24800056628bfdad0403fb0b128bfa98e403f5d
:10d2580041fd28bf5c4c403fb84829bff009403f1a
:10d26800159429bf67c73f3f57df29bfc0843f3f99
:10d27800802a2abffc413f3f8e752abf1bff3e3fd5
:10d2880082c02abf1bbc3e3f5b0b2bbfff783e3fd3
:10d298001b562bbfc5353e3fbfa02bbf6ef23d3f8f
:10d2a8004aeb2bbff9ae3d3fb9352cbf676b3d3f0d
:10d2b8000f802cbfb8273d3f49ca2cbfece33c3f49
:10d2c80069142dbf03a03c3f6f5e2dbffc5b3c3f44
:10d2d80059a82dbfd9173c3f29f22dbf98d33b3f02
:10d2e800de3b2ebf3b8f3b3f78852ebfc14a3b3f7d
:10d2f800f7ce2ebf29063b3f5b182fbf75c13a3fbb
:10d30800a5612fbfa47c3a3fd3aa2fbfb7373a3fb6
:10d31800e6f32fbfacf2393fde3c30bf85ad393f75
:10d32800bb8530bf4268393f7cce30bfe122393ff0
:10d33800221731bf65dd383fad5f31bfcb97383f2e
:10d348001da831bf1652383f71f031bf430c383f2a
:10d35800aa3832bf55c6373fc78032bf4a80373fe9
:10d36800c9c832bf233a373faf1033bfdff3363f68
:10d378007a5833bf7fad363f29a033bf0467363fa5
:10d38800bce733bf6c20363f342f34bfb8d9353fa4
:10d398008f7634bfe792353fcfbd34bffb4b353f67
:10d3a800f30435bff304353ffb4b35bfcfbd343fe6
:10d3b800e79235bf8f76343fb8d935bf342f343f25
:10d3c8006c2036bfbce7333f046736bf29a0333f24
:10d3d8007fad36bf7a58333fdff336bfaf10333fe8
:10d3e800233a37bfc9c8323f4a8037bfc780323f68
:10d3f80055c637bfaa38323f430c38bf71f0313faa
:10d40800165238bf1da8313fcb9738bfad5f313fab
:10d4180065dd38bf2217313fe12239bf7cce303f6e
:10d42800426839bfbb85303f85ad39bfde3c303ff0
:10d43800acf239bfe6f32f3fb7373abfd3aa2f3f35
:10d44800a47c3abfa5612f3f75c13abf5b182f3f37
:10d4580029063bbff7ce2e3fc14a3bbf78852e3ffa
:10d468003b8f3bbfde3b2e3f98d33bbf29f22d3f7e
:10d47800d9173cbf59a82d3ffc5b3cbf6f5e2d3fc1
:10d4880003a03cbf69142d3fece33cbf49ca2c3fc5
:10d49800b8273dbf0f802c3f676b3dbfb9352c3f88
:10d4a800f9ae3dbf4aeb2b3f6ef23dbfbfa02b3f0d
:10d4b800c5353ebf1b562b3fff783ebf5b0b2b3f4e
:10d4c8001bbc3ebf82c02a3f1bff3ebf8e752a3f52
:10d4d800fc413fbf802a2a3fc0843fbf57df293f16
:10d4e80067c73fbf1594293ff00940bfb848293f97
:10d4f8005c4c40bf41fd283fa98e40bfb0b1283fda
:10d50800dad040bf0566283fec1241bf401a283fd9
:10d51800e15441bf61ce273fb79641bf6882273f9c
:10d5280070d841bf5636273f0b1a42bf2aea263f1a
:10d53800895b42bfe39d263fe89c42bf8451263f5a
:10d5480029de42bf0a05263f4c1f43bf77b8253f57
:10d55800516043bfcb6b253f38a143bf041f253f14
:10d5680000e243bf25d2243fab2244bf2c85243f91
:10d57800376344bf1a38243fa5a344bfeeea233fcc
:10d58800f5e344bfa99d233f262445bf4b50233fc5
:10d59800396445bfd302233f2da445bf43b5223f7d
:10d5a80003e445bf9967223fbb2346bfd719223ff3
:10d5b800546346bffbcb213fcea246bf067e213f28
:10d5c8002ae246bff92f213f672147bfd2e1203f1a
:10d5d800856047bf9393203f849f47bf3b45203fcb
:10d5e80065de47bfcbf61f3f271d48bf41a81f3f39
:10d5f800ca5b48bf9f591f3f4e9a48bfe50a1f3f65
:10d60800b3d848bf12bc1e3ffa1649bf266d1e3f4d
:10d61800215549bf221e1e3f299349bf06cf1d3ff2
:10d6280012d149bfd17f1d3fdc0e4abf84301d3f58
:10d63800874c4abf1fe11c3f138a4abfa2911c3f77
:10d648007fc74abf0c421c3fcc044bbf5ff21b3f55
:10d65800fa414bbf99a21b3f097f4bbfbb521b3fef
:10d66800f8bb4bbfc6021b3fc7f84bbfb8b21a3f47
:10d6780078354cbf93621a3f08724cbf55121a3f57
:10d6880079ae4cbf00c2193fcbea4cbf9471193f29
:10d69800fd264dbf0f21193f10634dbf73d0183fb2
:10d6a800029f4dbfc07f183fd5da4dbff52e183ffa
:10d6b80089164ebf12de173f1c524ebf188d173ffa
:10d6c800908d4ebf073c173fe4c84ebfdfea163fb8
:10d6d80017044fbf9f99163f2b3f4fbf4748163f30
:10d6e8001f7a4fbfd9f6153ff4b44fbf54a5153f65
:10d6f800a8ef4fbfb753153f3b2a50bf0402153f51
:10d70800af6450bf39b0143f039f50bf585e143ff9
:10d7180037d950bf5f0c143f4a1351bf50ba133f5b
:10d728003d4d51bf2a68133f108751bfee15133f77
:10d73800c2c051bf9ac3123f54fa51bf3071123f51
:10d74800c63352bfb01e123f186d52bf19cc113fdd
:10d7580049a652bf6b79113f59df52bfa726113f27
:10d76800491853bfcdd3103f185153bfdc80103f29
:10d77800c78953bfd52d103f55c253bfb8da0f3fe5
:10d78800c3fa53bf84870f3f0f3354bf3b340f3f57
:10d798003b6b54bfdbe00e3f47a354bf658d0e3f84
:10d7a80031db54bfda390e3ffb1255bf38e60d3f67
:10d7b800a44a55bf81920d3f2c8255bfb33e0d3f01
:10d7c80093b955bfd0ea0c3fd9f055bfd7960c3f57
:10d7d800fe2756bfc9420c3f025f56bfa5ee0b3f5e
:10d7e800e59556bf6b9a0b3fa7cc56bf1c460b3f1f
:10d7f800480357bfb7f10a3fc73957bf3d9d0a3f96
:10d80800267057bfad480a3f63a657bf09f4093fc2
:10d818007fdc57bf4e9f093f791258bf7f4a093fa7
:10d82800534858bf9bf5083f0b7e58bfa1a0083f3f
:10d83800a1b358bf924b083f17e958bf6ff6073f8f
:10d848006a1e59bf36a1073f9c5359bfe84b073f93
:10d85800ad8859bf86f6063f9cbd59bf0ea1063f4d
:10d868006af259bf824b063f16275abfe2f5053fb9
:10d87800a05b5abf2ca0053f09905abf624a053fda
:10d8880050c45abf84f4043f75f85abf919e043fb0
:10d89800792c5bbf8948043f5a605bbf6df2033f38
:10d8a8001a945bbf3d9c033fb8c75bbff845033f75
:10d8b80034fb5bbf9fef023f8e2e5cbf3299023f65
:10d8c800c7615cbfb142023fdd945cbf1cec013f05
:10d8d800d1c75cbf7395013fa3fa5cbfb53e013f5a
:10d8e800532d5dbfe4e7003fe15f5dbfff90003f60
:10d8f8004d925dbf063a003f97c45dbff3c5ff3e3a
:10d90800bef65dbfb217ff3ec3285ebf4a69fe3e42
:10d91800a65a5ebfbbbafd3e678c5ebf040cfd3ed7
:10d9280005be5ebf275dfc3e81ef5ebf22aefb3ebb
:10d93800db205fbff7fefa3e12525fbfa54ffa3eeb
:10d9480027835fbf2da0f93e19b45fbf8ef0f83e64
:10d95800e9e45fbfc840f83e961560bfdc90f73e2b
:10d96800214660bfcbe0f63e897660bf9330f63e35
:10d97800cfa660bf3580f53ef2d660bfb1cff43e8a
:10d98800f20661bf071ff43ed03661bf386ef33e22
:10d998008a6661bf43bdf23e229661bf290cf23e02
:10d9a80098c561bfea5af13eeaf461bf85a9f03e25
:10d9b8001a2462bffbf7ef3e265362bf4c46ef3e88
:10d9c800108262bf7994ee3ed7b062bf80e2ed3e2e
:10d9d8007bdf62bf6330ed3efc0d63bf217eec3e12
:10d9e8005a3c63bfbbcbeb3e956a63bf3019eb3e35
:10d9f800ac9863bf8166ea3ea1c663bfaeb3e93e99
:10da080073f463bfb700e93e212264bf9c4de83e32
:10da1800ac4f64bf5d9ae73e147d64bffbe6e63e0b
:10da280059aa64bf7533e63e7bd764bfcb7fe53e1a
:10da3800790465bffecbe43e543165bf0e18e43e61
:10da48000b5e65bffa63e33ea08a65bfc4afe23ee2
:10da580010b765bf6afbe13e5ee365bfee46e13e97
:10da6800880f66bf4f92e03e8e3b66bf8ddddf3e7e
:10da7800716766bfa928df3e309366bfa273de3e9a
:10da8800ccbe66bf79bedd3e45ea66bf2e09dd3ee7
:10da9800991567bfc153dc3eca4067bf319edb3e64
:10daa800d86b67bf80e8da3ec19667bfad32da3e11
:10dab80087c167bfb97cd93e2aec67bfa3c6d83ee9
:10dac800a81668bf6b10d83e034168bf135ad73eeb
:10dad800396b68bf99a3d63e4c9568bffdecd53e1f
:10dae8003cbf68bf4136d53e07e968bf647fd43e76
:10daf800ae1269bf67c8d33e323c69bf4811d33ef6
:10db0800916569bf095ad23ecc8e69bfaaa2d13e9f
:10db1800e4b769bf2aebd03ed7e069bf8a33d03e6d
:10db2800a7096abfca7bcf3e52326abfeac3ce3e5c
:10db3800d95a6abfea0bce3e3c836abfca53cd3e70
:10db48007bab6abf8b9bcc3e95d36abf2ce3cb3ea5
:10db58008cfb6abfae2acb3e5e236bbf1072ca3ef7
:10db68000c4b6bbf53b9c93e95726bbf7700c93e6a
:10db7800fb996bbf7c47c83e3bc16bbf628ec73efb
:10db880058e86bbf29d5c63e500f6cbfd21bc63ea6
:10db980024366cbf5c62c53ed45c6cbfc8a8c43e6a
:10dba8005e836cbf15efc33ec5a96cbf4435c33e49
:10dbb80007d06cbf557bc23e24f66cbf48c1c13e3e
:10dbc8001d1c6dbf1e07c13ef2416dbfd54cc03e46
:10dbd800a1676dbf6f92bf3e2d8d6dbfebd7be3e67
:10dbe80093b26dbf4a1dbe3ed5d76dbf8b62bd3e99
:10dbf800f2fc6dbfafa7bc3eeb216ebfb6ecbb3edf
:10dc0800be466ebfa031bb3e6d6b6ebf6e76ba3e30
:10dc1800f88f6ebf1ebbb93e5db46ebfb2ffb83e93
:10dc28009ed86ebf2a44b83ebafc6ebf8488b73e01
:10dc3800b0206fbfc3ccb63e83446fbfe610b63e7c
:10dc480030686fbfec54b53eb88b6fbfd698b43e02
:10dc58001baf6fbfa5dcb33e5ad26fbf5820b33e8f
:10dc680073f56fbfef63b23e671870bf6ba7b13e25
:10dc7800373b70bfcbeab03ee15d70bf102eb03ebf
:10dc8800668070bf3a71af3ec6a270bf49b4ae3e5f
:10dc980002c570bf3cf7ad3e17e770bf153aad3e01
:10dca800080971bfd47cac3ed42a71bf77bfab3ea4
:10dcb8007a4c71bf0102ab3efb6d71bf6f44aa3e47
:10dcc800578f71bfc486a93e8eb071bffec8a83eeb
:10dcd8009fd171bf1f0ba83e8cf271bf254da73e87
:10dce800521372bf128fa63ef43372bfe5d0a53e21
:10dcf800705472bf9f12a53ec77472bf3f54a43eb2
:10dd0800f89472bfc595a33e04b572bf33d7a23e3f
:10dd1800ebd472bf8718a23eacf472bfc259a13ec1
:10dd2800471473bfe59aa03ebe3373bfeedb9f3e38
:10dd38000e5373bfdf1c9f3e397273bfb85d9e3ea2
:10dd48003f9173bf789e9d3e1fb073bf20df9c3efe
:10dd5800d9ce73bfaf1f9c3e6eed73bf27609b3e4d
:10dd6800dd0b74bf86a09a3e272a74bfcee0993e89
:10dd78004b4874bffe20993e496674bf1661983eb1
:10dd8800228474bf17a1973ed5a174bf00e1963ec7
:10dd980062bf74bfd220963ec9dc74bf8d60953ec9
:10dda8000bfa74bf31a0943e271775bfbfdf933eaf
:10ddb8001d3475bf351f933eed5075bf945e923e7e
:10ddc800976d75bfdd9d913e1c8a75bf10dd903e35
:10ddd8007ba675bf2c1c903eb3c275bf325b8f3ecd
:10dde800c6de75bf229a8e3eb3fa75bffcd88d3e4b
:10ddf8007a1676bfc0178d3e1b3276bf6e568c3ea4
:10de0800974d76bf07958b3eec6876bf8ad38a3ede
:10de18001b8476bff8118a3e249f76bf5050893ef6
:10de280007ba76bf938e883ec4d476bfc1cc873eee
:10de38005bef76bfda0a873ecc0977bfdf48863ebc
:10de4800172477bfce86853e3c3e77bfaac4843e62
:10de58003a5877bf7002843e137277bf2240833ee0
:10de6800c58b77bfc07d823e51a577bf4abb813e37
:10de7800b7be77bfc0f8803ef7d777bf2236803e5f
:10de880010f177bfe1e67e3e040a78bf56617d3e19
:10de9800d12278bfa4db7b3e773b78bfcb557a3e57
:10dea800f85378bfcccf783e526c78bfa649773efe
:10deb800868478bf5ac3753e939c78bfe83c743e0d
:10dec8007bb478bf51b6723e3bcc78bf942f713e7d
:10ded800d6e378bfb2a86f3e4afb78bfab216e3e4f
:10dee800981279bf7f9a6c3ebf2979bf2f136b3e7a
:10def800c04079bfba8b693e9a5779bf2204683e01
:10df08004e6e79bf667c663edc8479bf86f4643edb
:10df1800439b79bf836c633e83b179bf5ce4613e08
:10df28009dc779bf135c603e91dd79bfa8d35e3e83
:10df38005ef379bf1a4b5d3e04097abf6ac25b3e45
:10df4800841e7abf97395a3edd337abfa4b0583e53
:10df580010497abf8f27573e1c5e7abf589e553ea0
:10df680002737abf0115543ec1877abf898b523e2e
:10df7800599c7abff101513ecbb07abf38784f3ef9
:10df880016c57abf60ee4d3e3ad97abf67644c3efb
:10df980037ed7abf4fda4a3e0e017bbf1850493e33
:10dfa800be147bbfc2c5473e48287bbf4d3b463e9b
:10dfb800ab3b7bbfb9b0443ee74e7bbf0726433e31
:10dfc800fc617bbf379b413eea747bbf4910403ef2
:10dfd800b2877bbf3e853e3e539a7bbf15fa3c3ed7
:10dfe800cdac7bbfcf6e3b3e20bf7bbf6ce3393ee1
:10dff8004dd17bbfec57383e53e37bbf50cc363e08
:10e0080031f57bbf9840353ee9067cbfc4b4333e4a
:10e018007a187cbfd428323ee5297cbfc99c303ea3
:10e02800283b7cbfa2102f3e444c7cbf61842d3e10
:10e038003a5d7cbf04f82b3e086e7cbf8d6b2a3e90
:10e04800b07e7cbffcde283e318f7cbf5152273e1c
:10e058008a9f7cbf8cc5253ebdaf7cbfad38243eb2
:10e06800c9bf7cbfb6ab223eaecf7cbfa51e213e4a
:10e078006cdf7cbf7b911f3e03ef7cbf38041e3ee4
:10e0880073fe7cbfde761c3ebc0d7dbf6be91a3e7d
:10e09800dd1c7dbfe05b193ed82b7dbf3dce173e12
:10e0a800ac3a7dbf8340163e59497dbfb2b2143e9b
:10e0b800de577dbfca24133e3d667dbfcc96113e18
:10e0c80074747dbfb708103e85827dbf8b7a0e3e83
:10e0d8006e907dbf4aec0c3e309e7dbff35d0b3edb
:10e0e800ccab7dbf86cf093e40b97dbf0541083e18
:10e0f8008cc67dbf6eb2063eb2d37dbfc223053e3d
:10e10800b1e07dbf0295033e88ed7dbf2e06023e3d
:10e1180038fa7dbf4577003ec2067ebf92d0fd3dee
:10e1280024137ebf73b2fa3d5e1f7ebf2c94f73d69
:10e13800722b7ebfc075f43d5e377ebf2e57f13d12
:10e1480023437ebf7638ee3dc14e7ebf9a19eb3d24
:10e15800385a7ebf9afae73d88657ebf76dbe43d94
:10e16800b0707ebf2ebce13db17b7ebfc49cde3d5e
:10e178008b867ebf377ddb3d3d917ebf895dd83d77
:10e18800c99b7ebfb93dd53d2da67ebfc81dd23dda
:10e1980069b07ebfb7fdce3d7fba7ebf86ddcb3d81
:10e1a8006dc47ebf36bdc83d34ce7ebfc69cc53d5e
:10e1b800d4d77ebf397cc23d4ce17ebf8d5bbf3d6d
:10e1c8009dea7ebfc33abc3dc7f37ebfdd19b93daa
:10e1d800c9fc7ebfdaf8b53da4057fbfbbd7b23d09
:10e1e800580e7fbf80b6af3de4167fbf2b95ac3d80
:10e1f800491f7fbfba73a93d87277fbf3052a63d0d
:10e208009d2f7fbf8c30a33d8d377fbfcf0ea03da4
:10e21800543f7fbff9ec9c3df4467fbf0acb993d44
:10e228006d4e7fbf05a9963dbf557fbfe786933ddd
:10e23800e95c7fbfb464903dec637fbf6a428d3d6b
:10e24800c76a7fbf0a208a3d7b717fbf94fd863de8
:10e2580008787fbf0adb833d6d7e7fbf6cb8803d49
:10e26800ab847fbf742b7b3dc28a7fbfe9e5743dd9
:10e27800b1907fbf38a06e3d78967fbf625a683de7
:10e28800189c7fbf6814623d91a17fbf4cce5b3d57
:10e29800e3a67fbf0e88553d0dac7fbfaf414f3d14
:10e2a8000fb17fbf2ffb483deab57fbf91b4423d18
:10e2b8009eba7fbfd56d3c3d2abf7fbffc26363d49
:10e2c8008fc37fbf07e02f3dccc77fbff698293d9e
:10e2d800e2cb7fbfcc51233dd1cf7fbf880a1d3d04
:10e2e80098d37fbf2cc3163d37d77fbfb87b103d6f
:10e2f800afda7fbf2f340a3d00de7fbf90ec033dcd
:10e3080029e17fbfb949fb3c2be47fbf2dbaee3c26
:10e3180005e77fbf7b2ae23cb8e97fbfa69ad53cd8
:10e3280043ec7fbfb00ac93ca7ee7fbf9b7abc3cd9
:10e33800e3f07fbf69eaaf3cf8f27fbf1c5aa33c09
:10e34800e6f47fbfb6c9963cacf67fbf38398a3c45
:10e358004af87fbf4b517b3cc1f97fbf0030623c1c
:10e3680011fb7fbf900e493c39fc7fbf02ed2f3c6b
:10e3780039fd7fbf59cb163c13fe7fbf3053fb3ba3
:10e38800c4fe7fbf890fc93b4eff7fbfc1cb963b01
:10e39800b1ff7fbfc70f493becff7fbfd40fc93a1e
:10e3a800000080bf00000000ecff7fbfd40fc9ba97
:10e3b800b1ff7fbfc70f49bb4eff7fbfc1cb96bb25
:10e3c800c4fe7fbf890fc9bb13fe7fbf3053fbbba1
:10e3d80039fd7fbf59cb16bc39fc7fbf02ed2fbc7e
:10e3e80011fb7fbf900e49bcc1f97fbf003062bcf2
:10e3f8004af87fbf4b517bbcacf67fbf38398abc2b
:10e40800e6f47fbfb6c996bcf8f27fbf1c5aa3bc1e
:10e41800e3f07fbf69eaafbca7ee7fbf9b7abcbcc5
:10e4280043ec7fbfb00ac9bcb8e97fbfa69ad5bc88
:10e4380005e77fbf7b2ae2bc2be47fbf2dbaeebc89
:10e4480029e17fbfb949fbbc00de7fbf90ec03bd6b
:10e45800afda7fbf2f340abd37d77fbfb87b10bd77
:10e4680098d37fbf2cc316bdd1cf7fbf880a1dbdef
:10e47800e2cb7fbfcc5123bdccc77fbff69829bd67
:10e488008fc37fbf07e02fbd2abf7fbffc2636bde5
:10e498009eba7fbfd56d3cbdeab57fbf91b442bd82
:10e4a8000fb17fbf2ffb48bd0dac7fbfaf414fbd44
:10e4b800e3a67fbf0e8855bd91a17fbf4cce5bbd43
:10e4c800189c7fbf681462bd78967fbf625a68bd8a
:10e4d800b1907fbf38a06ebdc28a7fbfe9e574bd29
:10e4e800ab847fbf742b7bbd6d7e7fbf6cb880bd56
:10e4f80008787fbf0adb83bd7b717fbf94fd86bd33
:10e50800c76a7fbf0a208abdec637fbf6a428dbda0
:10e51800e95c7fbfb46490bdbf557fbfe78693bdfc
:10e528006d4e7fbf05a996bdf4467fbf0acb99bd46
:10e53800543f7fbff9ec9cbd8d377fbfcf0ea0bd88
:10e548009d2f7fbf8c30a3bd87277fbf3052a6bdcc
:10e55800491f7fbfba73a9bde4167fbf2b95acbd19
:10e56800580e7fbf80b6afbda4057fbfbbd7b2bd75
:10e57800c9fc7ebfdaf8b5bdc7f37ebfdd19b9bdea
:10e588009dea7ebfc33abcbd4ce17ebf8d5bbfbd7b
:10e59800d4d77ebf397cc2bd34ce7ebfc69cc5bd34
:10e5a8006dc47ebf36bdc8bd7fba7ebf86ddcbbd1c
:10e5b80069b07ebfb7fdcebd2da67ebfc81dd2bd3a
:10e5c800c99b7ebfb93dd5bd3d917ebf895dd8bd94
:10e5d8008b867ebf377ddbbdb17b7ebfc49cdebd35
:10e5e800b0707ebf2ebce1bd88657ebf76dbe4bd22
:10e5f800385a7ebf9afae7bdc14e7ebf9a19ebbd65
:10e6080023437ebf7638eebd5e377ebf2e57f1bd01
:10e61800722b7ebfc075f4bd5e1f7ebf2c94f7bd04
:10e6280024137ebf73b2fabdc2067ebf92d0fdbd71
:10e6380038fa7dbf457700be88ed7dbf2e0602be45
:10e64800b1e07dbf029503beb2d37dbfc22305be34
:10e658008cc67dbf6eb206be40b97dbf054108beff
:10e66800ccab7dbf86cf09be309e7dbff35d0bbeb0
:10e678006e907dbf4aec0cbe85827dbf8b7a0ebe44
:10e6880074747dbfb70810be3d667dbfcc9611bec1
:10e69800de577dbfca2413be59497dbfb2b214be2e
:10e6a800ac3a7dbf834016bed82b7dbf3dce17be8a
:10e6b800dd1c7dbfe05b19bebc0d7dbf6be91abeda
:10e6c80073fe7cbfde761cbe03ef7cbf38041ebe23
:10e6d8006cdf7cbf7b911fbeaecf7cbfa51e21be69
:10e6e800c9bf7cbfb6ab22bebdaf7cbfad3824beb0
:10e6f8008a9f7cbf8cc525be318f7cbf515227bef7
:10e70800b07e7cbffcde28be086e7cbf8d6b2abe47
:10e718003a5d7cbf04f82bbe444c7cbf61842dbe9f
:10e72800283b7cbfa2102fbee5297cbfc99c30be08
:10e738007a187cbfd42832bee9067cbfc4b433be85
:10e7480031f57bbf984035be53e37bbf50cc36be16
:10e758004dd17bbfec5738be20bf7bbf6ce339bec1
:10e76800cdac7bbfcf6e3bbe539a7bbf15fa3cbe88
:10e77800b2877bbf3e853ebeea747bbf491040be70
:10e78800fc617bbf379b41bee74e7bbf072643be7c
:10e79800ab3b7bbfb9b044be48287bbf4d3b46beb0
:10e7a800be147bbfc2c547be0e017bbf185049be11
:10e7b80037ed7abf4fda4abe3ad97abf67644cbea2
:10e7c80016c57abf60ee4dbecbb07abf38784fbe63
:10e7d800599c7abff10151bec1877abf898b52be5d
:10e7e80002737abf011554be1c5e7abf589e55be8f
:10e7f80010497abf8f2757bedd337abfa4b058be01
:10e80800841e7abf97395abe04097abf6ac25bbeb2
:10e818005ef379bf1a4b5dbe91dd79bfa8d35ebeaa
:10e828009dc779bf135c60be83b179bf5ce461beec
:10e83800439b79bf836c63bedc8479bf86f464be76
:10e848004e6e79bf667c66be9a5779bf220468be51
:10e85800c04079bfba8b69bebf2979bf2f136bbe81
:10e86800981279bf7f9a6cbe4afb78bfab216ebe07
:10e87800d6e378bfb2a86fbe3bcc78bf942f71bee9
:10e888007bb478bf51b672be939c78bfe83c74be27
:10e89800868478bf5ac375be526c78bfa64977bec6
:10e8a800f85378bfcccf78be773b78bfcb557abecc
:10e8b800d12278bfa4db7bbe040a78bf56617dbe37
:10e8c80010f177bfe1e67ebef7d777bf223680be6c
:10e8d800b7be77bfc0f880be51a577bf4abb81be1f
:10e8e800c58b77bfc07d82be137277bf224083bebf
:10e8f8003a5877bf700284be3c3e77bfaac484be34
:10e90800172477bfce8685becc0977bfdf4886be81
:10e918005bef76bfda0a87bec4d476bfc1cc87bea8
:10e9280007ba76bf938e88be249f76bf505089bea3
:10e938001b8476bff8118abeec6876bf8ad38abe7c
:10e94800974d76bf07958bbe1b3276bf6e568cbe31
:10e958007a1676bfc0178dbeb3fa75bffcd88dbec8
:10e96800c6de75bf229a8ebeb3c275bf325b8fbe3c
:10e978007ba675bf2c1c90be1c8a75bf10dd90be8f
:10e98800976d75bfdd9d91beed5075bf945e92becb
:10e998001d3475bf351f93be271775bfbfdf93bee4
:10e9a8000bfa74bf31a094bec9dc74bf8d6095beec
:10e9b80062bf74bfd22096bed5a174bf00e196bed7
:10e9c800228474bf17a197be496674bf166198beaa
:10e9d8004b4874bffe2099be272a74bfcee099be6b
:10e9e800dd0b74bf86a09abe6eed73bf27609bbe19
:10e9f800d9ce73bfaf1f9cbe1fb073bf20df9cbeb4
:10ea08003f9173bf789e9dbe397273bfb85d9ebe3d
:10ea18000e5373bfdf1c9fbebe3373bfeedb9fbeba
:10ea2800471473bfe59aa0beacf472bfc259a1be29
:10ea3800ebd472bf8718a2be04b572bf33d7a2be8b
:10ea4800f89472bfc595a3bec77472bf3f54a4bee5
:10ea5800705472bf9f12a5bef43372bfe5d0a5be35
:10ea6800521372bf128fa6be8cf271bf254da7be7e
:10ea78009fd171bf1f0ba8be8eb071bffec8a8bec4
:10ea8800578f71bfc486a9befb6d71bf6f44aabe04
:10ea98007a4c71bf0102abbed42a71bf77bfabbe3f
:10eaa800080971bfd47cacbe17e770bf153aadbe7c
:10eab80002c570bf3cf7adbec6a270bf49b4aebeba
:10eac800668070bf3a71afbee15d70bf102eb0bef8
:10ead800373b70bfcbeab0be671870bf6ba7b1be3b
:10eae80073f56fbfef63b2be5ad26fbf5820b3be83
:10eaf8001baf6fbfa5dcb3beb88b6fbfd698b4bed3
:10eb080030686fbfec54b5be83446fbfe610b6be25
:10eb1800b0206fbfc3ccb6bebafc6ebf8488b7be88
:10eb28009ed86ebf2a44b8be5db46ebfb2ffb8bef1
:10eb3800f88f6ebf1ebbb9be6d6b6ebf6e76babe68
:10eb4800be466ebfa031bbbeeb216ebfb6ecbbbeee
:10eb5800f2fc6dbfafa7bcbed5d76dbf8b62bdbe83
:10eb680093b26dbf4a1dbebe2d8d6dbfebd7bebe25
:10eb7800a1676dbf6f92bfbef2416dbfd54cc0bedd
:10eb88001d1c6dbf1e07c1be24f66cbf48c1c1bea7
:10eb980007d06cbf557bc2bec5a96cbf4435c3be88
:10eba8005e836cbf15efc3bed45c6cbfc8a8c4be7f
:10ebb80024366cbf5c62c5be500f6cbfd21bc6be8c
:10ebc80058e86bbf29d5c6be3bc16bbf628ec7beb6
:10ebd800fb996bbf7c47c8be95726bbf7700c9bef7
:10ebe8000c4b6bbf53b9c9be5e236bbf1072cabe54
:10ebf8008cfb6abfae2acbbe95d36abf2ce3cbbed3
:10ec08007bab6abf8b9bccbe3c836abfca53cdbe6d
:10ec1800d95a6abfea0bcebe52326abfeac3cebe29
:10ec2800a7096abfca7bcfbed7e069bf8a33d0be07
:10ec3800e4b769bf2aebd0becc8e69bfaaa2d1be09
:10ec4800916569bf095ad2be323c69bf4811d3be2b
:10ec5800ae1269bf67c8d3be07e968bf647fd4be78
:10ec68003cbf68bf4136d5be4c9568bffdecd5beec
:10ec7800396b68bf99a3d6be034168bf135ad7be84
:10ec8800a81668bf6b10d8be2aec67bfa3c6d8be4b
:10ec980087c167bfb97cd9bec19667bfad32dabe3e
:10eca800d86b67bf80e8dabeca4067bf319edbbe5b
:10ecb800991567bfc153dcbe45ea66bf2e09ddbea4
:10ecc800ccbe66bf79beddbe309366bfa273debe22
:10ecd800716766bfa928dfbe8e3b66bf8ddddfbecc
:10ece800880f66bf4f92e0be5ee365bfee46e1bea9
:10ecf80010b765bf6afbe1bea08a65bfc4afe2bebc
:10ed08000b5e65bffa63e3be543165bf0e18e4beff
:10ed1800790465bffecbe4be7bd764bfcb7fe5be7d
:10ed280059aa64bf7533e6be147d64bffbe6e6be30
:10ed3800ac4f64bf5d9ae7be212264bf9c4de8be1c
:10ed480073f463bfb700e9bea1c663bfaeb3e9be43
:10ed5800ac9863bf8166eabe956a63bf3019ebbea3
:10ed68005a3c63bfbbcbebbefc0d63bf217eecbe40
:10ed78007bdf62bf6330edbed7b062bf80e2edbe1d
:10ed8800108262bf7994eebe265362bf4c46efbe36
:10ed98001a2462bffbf7efbeeaf461bf85a9f0be93
:10eda80098c561bfea5af1be229661bf290cf2be2e
:10edb8008a6661bf43bdf2bed03661bf386ef3be0e
:10edc800f20661bf071ff4bef2d660bfb1cff4be32
:10edd800cfa660bf3580f5be897660bf9330f6be9a
:10ede800214660bfcbe0f6be961560bfdc90f7be4b
:10edf800e9e45fbfc840f8be19b45fbf8ef0f8be43
:10ee080027835fbf2da0f9be12525fbfa54ffabe80
:10ee1800db205fbff7fefabe81ef5ebf22aefbbe0e
:10ee280005be5ebf275dfcbe678c5ebf040cfdbee1
:10ee3800a65a5ebfbbbafdbec3285ebf4a69febe06
:10ee4800bef65dbfb217ffbe97c45dbff3c5ffbe78
:10ee58004d925dbf063a00bfe15f5dbfff9000bf06
:10ee6800532d5dbfe4e700bfa3fa5cbfb53e01bf09
:10ee7800d1c75cbf739501bfdd945cbf1cec01bfbb
:10ee8800c7615cbfb14202bf8e2e5cbf329902bf20
:10ee980034fb5bbf9fef02bfb8c75bbff84503bf3a
:10eea8001a945bbf3d9c03bf5a605bbf6df203bf02
:10eeb800792c5bbf894804bf75f85abf919e04bf7f
:10eec80050c45abf84f404bf09905abf624a05bfb0
:10eed800a05b5abf2ca005bf16275abfe2f505bf95
:10eee8006af259bf824b06bf9cbd59bf0ea106bf2f
:10eef800ad8859bf86f606bf9c5359bfe84b07bf7c
:10ef08006a1e59bf36a107bf17e958bf6ff607bf7a
:10ef1800a1b358bf924b08bf0b7e58bfa1a008bf32
:10ef2800534858bf9bf508bf791258bf7f4a09bf9d
:10ef38007fdc57bf4e9f09bf63a657bf09f409bfbf
:10ef4800267057bfad480abfc73957bf3d9d0abf96
:10ef5800480357bfb7f10abfa7cc56bf1c460bbf23
:10ef6800e59556bf6b9a0bbf025f56bfa5ee0bbf68
:10ef7800fe2756bfc9420cbfd9f055bfd7960cbf64
:10ef880093b955bfd0ea0cbf2c8255bfb33e0dbf15
:10ef9800a44a55bf81920dbffb1255bf38e60dbf7d
:10efa80031db54bfda390ebf47a354bf658d0ebf9e
:10efb8003b6b54bfdbe00ebf0f3354bf3b340fbf76
:10efc800c3fa53bf84870fbf55c253bfb8da0fbf08
:10efd800c78953bfd52d10bf185153bfdc8010bf50
:10efe800491853bfcdd310bf59df52bfa72611bf51
:10eff80049a652bf6b7911bf186d52bf19cc11bf0a
:10f00800c63352bfb01e12bf54fa51bf307112bf7f
:10f01800c2c051bf9ac312bf108751bfee1513bfac
:10f028003d4d51bf2a6813bf4a1351bf50ba13bf91
:10f0380037d950bf5f0c14bf039f50bf585e14bf31
:10f04800af6450bf39b014bf3b2a50bf040215bf8c
:10f05800a8ef4fbfb75315bff4b44fbf54a515bfa2
:10f068001f7a4fbfd9f615bf2b3f4fbf474816bf72
:10f0780017044fbf9f9916bfe4c84ebfdfea16bffb
:10f08800908d4ebf073c17bf1c524ebf188d17bf3f
:10f0980089164ebf12de17bfd5da4dbff52e18bf41
:10f0a800029f4dbfc07f18bf10634dbf73d018bffc
:10f0b800fd264dbf0f2119bfcbea4cbf947119bf74
:10f0c80079ae4cbf00c219bf08724cbf55121abfa7
:10f0d80078354cbf93621abfc7f84bbfb8b21abf96
:10f0e800f8bb4bbfc6021bbf097f4bbfbb521bbf40
:10f0f800fa414bbf99a21bbfcc044bbf5ff21bbfa9
:10f108007fc74abf0c421cbf138a4abfa2911cbfcb
:10f11800874c4abf1fe11cbfdc0e4abf84301dbfad
:10f1280012d149bfd17f1dbf299349bf06cf1dbf4b
:10f13800215549bf221e1ebffa1649bf266d1ebfa4
:10f14800b3d848bf12bc1ebf4e9a48bfe50a1fbfbe
:10f15800ca5b48bf9f591fbf271d48bf41a81fbf93
:10f1680065de47bfcbf61fbf849f47bf3b4520bf27
:10f17800856047bf939320bf672147bfd2e120bf77
:10f188002ae246bff92f21bfcea246bf067e21bf85
:10f19800546346bffbcb21bfbb2346bfd71922bf51
:10f1a80003e445bf996722bf2da445bf43b522bfdd
:10f1b800396445bfd30223bf262445bf4b5023bf24
:10f1c800f5e344bfa99d23bfa5a344bfeeea23bf2f
:10f1d800376344bf1a3824bfab2244bf2c8524bff1
:10f1e80000e243bf25d224bf38a143bf041f25bf77
:10f1f800516043bfcb6b25bf4c1f43bf77b825bfba
:10f2080029de42bf0a0526bfe89c42bf845126bfbb
:10f21800895b42bfe39d26bf0b1a42bf2aea26bf7d
:10f2280070d841bf563627bfb79641bf688227bfff
:10f23800e15441bf61ce27bfec1241bf401a28bf3d
:10f24800dad040bf056628bfa98e40bfb0b128bf3d
:10f258005c4c40bf41fd28bff00940bfb84829bffa
:10f2680067c73fbf159429bfc0843fbf57df29bf79
:10f27800fc413fbf802a2abf1bff3ebf8e752abfb5
:10f288001bbc3ebf82c02abfff783ebf5b0b2bbfb3
:10f29800c5353ebf1b562bbf6ef23dbfbfa02bbf6f
:10f2a800f9ae3dbf4aeb2bbf676b3dbfb9352cbfed
:10f2b800b8273dbf0f802cbfece33cbf49ca2cbf29
:10f2c80003a03cbf69142dbffc5b3cbf6f5e2dbf24
:10f2d800d9173cbf59a82dbf98d33bbf29f22dbfe2
:10f2e8003b8f3bbfde3b2ebfc14a3bbf78852ebf5d
:10f2f80029063bbff7ce2ebf75c13abf5b182fbf9b
:10f30800a47c3abfa5612fbfb7373abfd3aa2fbf96
:10f31800acf239bfe6f32fbf85ad39bfde3c30bf55
:10f32800426839bfbb8530bfe12239bf7cce30bfd0
:10f3380065dd38bf221731bfcb9738bfad5f31bf0e
:10f34800165238bf1da831bf430c38bf71f031bf0a
:10f3580055c637bfaa3832bf4a8037bfc78032bfc9
:10f36800233a37bfc9c832bfdff336bfaf1033bf48
:10f378007fad36bf7a5833bf046736bf29a033bf85
:10f388006c2036bfbce733bfb8d935bf342f34bf84
:10f39800e79235bf8f7634bffb4b35bfcfbd34bf47
:10f3a800f30435bff30435bfcfbd34bffb4b35bfc6
:10f3b8008f7634bfe79235bf342f34bfb8d935bf05
:10f3c800bce733bf6c2036bf29a033bf046736bf04
:10f3d8007a5833bf7fad36bfaf1033bfdff336bfc8
:10f3e800c9c832bf233a37bfc78032bf4a8037bf48
:10f3f800aa3832bf55c637bf71f031bf430c38bf8a
:10f408001da831bf165238bfad5f31bfcb9738bf8b
:10f41800221731bf65dd38bf7cce30bfe12239bf4e
:10f42800bb8530bf426839bfde3c30bf85ad39bfd0
:10f43800e6f32fbfacf239bfd3aa2fbfb7373abf15
:10f44800a5612fbfa47c3abf5b182fbf75c13abf17
:10f45800f7ce2ebf29063bbf78852ebfc14a3bbfda
:10f46800de3b2ebf3b8f3bbf29f22dbf98d33bbf5e
:10f4780059a82dbfd9173cbf6f5e2dbffc5b3cbfa1
:10f4880069142dbf03a03cbf49ca2cbfece33cbfa5
:10f498000f802cbfb8273dbfb9352cbf676b3dbf68
:10f4a8004aeb2bbff9ae3dbfbfa02bbf6ef23dbfed
:10f4b8001b562bbfc5353ebf5b0b2bbfff783ebf2e
:10f4c80082c02abf1bbc3ebf8e752abf1bff3ebf32
:10f4d800802a2abffc413fbf57df29bfc0843fbff6
:10f4e800159429bf67c73fbfb84829bff00940bf77
:10f4f80041fd28bf5c4c40bfb0b128bfa98e40bfba
:10f50800056628bfdad040bf401a28bfec1241bfb9
:10f5180061ce27bfe15441bf688227bfb79641bf7c
:10f52800563627bf70d841bf2aea26bf0b1a42bffa
:10f53800e39d26bf895b42bf845126bfe89c42bf3a
:10f548000a0526bf29de42bf77b825bf4c1f43bf37
:10f55800cb6b25bf516043bf041f25bf38a143bff4
:10f5680025d224bf00e243bf2c8524bfab2244bf71
:10f578001a3824bf376344bfeeea23bfa5a344bfac
:10f58800a99d23bff5e344bf4b5023bf262445bfa5
:10f59800d30223bf396445bf43b522bf2da445bf5d
:10f5a800996722bf03e445bfd71922bfbb2346bfd3
:10f5b800fbcb21bf546346bf067e21bfcea246bf08
:10f5c800f92f21bf2ae246bfd2e120bf672147bffa
:10f5d800939320bf856047bf3b4520bf849f47bfab
:10f5e800cbf61fbf65de47bf41a81fbf271d48bf19
:10f5f8009f591fbfca5b48bfe50a1fbf4e9a48bf45
:10f6080012bc1ebfb3d848bf266d1ebffa1649bf2d
:10f61800221e1ebf215549bf06cf1dbf299349bfd2
:10f62800d17f1dbf12d149bf84301dbfdc0e4abf38
:10f638001fe11cbf874c4abfa2911cbf138a4abf57
:10f648000c421cbf7fc74abf5ff21bbfcc044bbf35
:10f6580099a21bbffa414bbfbb521bbf097f4bbfcf
:10f66800c6021bbff8bb4bbfb8b21abfc7f84bbf27
:10f6780093621abf78354cbf55121abf08724cbf37
:10f6880000c219bf79ae4cbf947119bfcbea4cbf09
:10f698000f2119bffd264dbf73d018bf10634dbf92
:10f6a800c07f18bf029f4dbff52e18bfd5da4dbfda
:10f6b80012de17bf89164ebf188d17bf1c524ebfda
:10f6c800073c17bf908d4ebfdfea16bfe4c84ebf98
:10f6d8009f9916bf17044fbf474816bf2b3f4fbf10
:10f6e800d9f615bf1f7a4fbf54a515bff4b44fbf45
:10f6f800b75315bfa8ef4fbf040215bf3b2a50bf31
:10f7080039b014bfaf6450bf585e14bf039f50bfd9
:10f718005f0c14bf37d950bf50ba13bf4a1351bf3b
:10f728002a6813bf3d4d51bfee1513bf108751bf57
:10f738009ac312bfc2c051bf307112bf54fa51bf31
:10f74800b01e12bfc63352bf19cc11bf186d52bfbd
:10f758006b7911bf49a652bfa72611bf59df52bf07
:10f76800cdd310bf491853bfdc8010bf185153bf09
:10f77800d52d10bfc78953bfb8da0fbf55c253bfc5
:10f7880084870fbfc3fa53bf3b340fbf0f3354bf37
:10f79800dbe00ebf3b6b54bf658d0ebf47a354bf64
:10f7a800da390ebf31db54bf38e60dbffb1255bf47
:10f7b80081920dbfa44a55bfb33e0dbf2c8255bfe1
:10f7c800d0ea0cbf93b955bfd7960cbfd9f055bf37
:10f7d800c9420cbffe2756bfa5ee0bbf025f56bf3e
:10f7e8006b9a0bbfe59556bf1c460bbfa7cc56bfff
:10f7f800b7f10abf480357bf3d9d0abfc73957bf76
:10f80800ad480abf267057bf09f409bf63a657bfa2
:10f818004e9f09bf7fdc57bf7f4a09bf791258bf87
:10f828009bf508bf534858bfa1a008bf0b7e58bf1f
:10f83800924b08bfa1b358bf6ff607bf17e958bf6f
:10f8480036a107bf6a1e59bfe84b07bf9c5359bf73
:10f8580086f606bfad8859bf0ea106bf9cbd59bf2d
:10f86800824b06bf6af259bfe2f505bf16275abf99
:10f878002ca005bfa05b5abf624a05bf09905abfba
:10f8880084f404bf50c45abf919e04bf75f85abf90
:10f89800894804bf792c5bbf6df203bf5a605bbf18
:10f8a8003d9c03bf1a945bbff84503bfb8c75bbf55
:10f8b8009fef02bf34fb5bbf329902bf8e2e5cbf45
:10f8c800b14202bfc7615cbf1cec01bfdd945cbfe5
:10f8d800739501bfd1c75cbfb53e01bfa3fa5cbf3a
:10f8e800e4e700bf532d5dbfff9000bfe15f5dbf40
:10f8f800063a00bf4d925dbff3c5ffbe97c45dbf1a
:10f90800b217ffbebef65dbf4a69febec3285ebf22
:10f91800bbbafdbea65a5ebf040cfdbe678c5ebfb7
:10f92800275dfcbe05be5ebf22aefbbe81ef5ebf9b
:10f93800f7fefabedb205fbfa54ffabe12525fbfcb
:10f948002da0f9be27835fbf8ef0f8be19b45fbf44
:10f95800c840f8bee9e45fbfdc90f7be961560bf0b
:10f96800cbe0f6be214660bf9330f6be897660bf15
:10f978003580f5becfa660bfb1cff4bef2d660bf6a
:10f98800071ff4bef20661bf386ef3bed03661bf02
:10f9980043bdf2be8a6661bf290cf2be229661bfe2
:10f9a800ea5af1be98c561bf85a9f0beeaf461bf05
:10f9b800fbf7efbe1a2462bf4c46efbe265362bf68
:10f9c8007994eebe108262bf80e2edbed7b062bf0e
:10f9d8006330edbe7bdf62bf217eecbefc0d63bff2
:10f9e800bbcbebbe5a3c63bf3019ebbe956a63bf15
:10f9f8008166eabeac9863bfaeb3e9bea1c663bf79
:10fa0800b700e9be73f463bf9c4de8be212264bf12
:10fa18005d9ae7beac4f64bffbe6e6be147d64bfeb
:10fa28007533e6be59aa64bfcb7fe5be7bd764bffa
:10fa3800fecbe4be790465bf0e18e4be543165bf41
:10fa4800fa63e3be0b5e65bfc4afe2bea08a65bfc2
:10fa58006afbe1be10b765bfee46e1be5ee365bf77
:10fa68004f92e0be880f66bf8ddddfbe8e3b66bf5e
:10fa7800a928dfbe716766bfa273debe309366bf7a
:10fa880079beddbeccbe66bf2e09ddbe45ea66bfc7
:10fa9800c153dcbe991567bf319edbbeca4067bf44
:10faa80080e8dabed86b67bfad32dabec19667bff1
:10fab800b97cd9be87c167bfa3c6d8be2aec67bfc9
:10fac8006b10d8bea81668bf135ad7be034168bfcb
:10fad80099a3d6be396b68bffdecd5be4c9568bfff
:10fae8004136d5be3cbf68bf647fd4be07e968bf56
:10faf80067c8d3beae1269bf4811d3be323c69bfd6
:10fb0800095ad2be916569bfaaa2d1becc8e69bf7f
:10fb18002aebd0bee4b769bf8a33d0bed7e069bf4d
:10fb2800ca7bcfbea7096abfeac3cebe52326abf3c
:10fb3800ea0bcebed95a6abfca53cdbe3c836abf50
:10fb48008b9bccbe7bab6abf2ce3cbbe95d36abf85
:10fb5800ae2acbbe8cfb6abf1072cabe5e236bbfd7
:10fb680053b9c9be0c4b6bbf7700c9be95726bbf4a
:10fb78007c47c8befb996bbf628ec7be3bc16bbfdb
:10fb880029d5c6be58e86bbfd21bc6be500f6cbf86
:10fb98005c62c5be24366cbfc8a8c4bed45c6cbf4a
:10fba80015efc3be5e836cbf4435c3bec5a96cbf29
:10fbb800557bc2be07d06cbf48c1c1be24f66cbf1e
:10fbc8001e07c1be1d1c6dbfd54cc0bef2416dbf26
:10fbd8006f92bfbea1676dbfebd7bebe2d8d6dbf47
:10fbe8004a1dbebe93b26dbf8b62bdbed5d76dbf79
:10fbf800afa7bcbef2fc6dbfb6ecbbbeeb216ebfbf
:10fc0800a031bbbebe466ebf6e76babe6d6b6ebf10
:10fc18001ebbb9bef88f6ebfb2ffb8be5db46ebf73
:10fc28002a44b8be9ed86ebf8488b7bebafc6ebfe1
:10fc3800c3ccb6beb0206fbfe610b6be83446fbf5c
:10fc4800ec54b5be30686fbfd698b4beb88b6fbfe2
:10fc5800a5dcb3be1baf6fbf5820b3be5ad26fbf6f
:10fc6800ef63b2be73f56fbf6ba7b1be671870bf05
:10fc7800cbeab0be373b70bf102eb0bee15d70bf9f
:10fc88003a71afbe668070bf49b4aebec6a270bf3f
:10fc98003cf7adbe02c570bf153aadbe17e770bfe1
:10fca800d47cacbe080971bf77bfabbed42a71bf84
:10fcb8000102abbe7a4c71bf6f44aabefb6d71bf27
:10fcc800c486a9be578f71bffec8a8be8eb071bfcb
:10fcd8001f0ba8be9fd171bf254da7be8cf271bf67
:10fce800128fa6be521372bfe5d0a5bef43372bf01
:10fcf8009f12a5be705472bf3f54a4bec77472bf92
:10fd0800c595a3bef89472bf33d7a2be04b572bf1f
:10fd18008718a2beebd472bfc259a1beacf472bfa1
:10fd2800e59aa0be471473bfeedb9fbebe3373bf18
:10fd3800df1c9fbe0e5373bfb85d9ebe397273bf82
:10fd4800789e9dbe3f9173bf20df9cbe1fb073bfde
:10fd5800af1f9cbed9ce73bf27609bbe6eed73bf2d
:10fd680086a09abedd0b74bfcee099be272a74bf69
:10fd7800fe2099be4b4874bf166198be496674bf91
:10fd880017a197be228474bf00e196bed5a174bfa7
:10fd9800d22096be62bf74bf8d6095bec9dc74bfa9
:10fda80031a094be0bfa74bfbfdf93be271775bf8f
:10fdb800351f93be1d3475bf945e92beed5075bf5e
:10fdc800dd9d91be976d75bf10dd90be1c8a75bf15
:10fdd8002c1c90be7ba675bf325b8fbeb3c275bfad
:10fde800229a8ebec6de75bffcd88dbeb3fa75bf2b
:10fdf800c0178dbe7a1676bf6e568cbe1b3276bf84
:10fe080007958bbe974d76bf8ad38abeec6876bfbe
:10fe1800f8118abe1b8476bf505089be249f76bfd6
:10fe2800938e88be07ba76bfc1cc87bec4d476bfce
:10fe3800da0a87be5bef76bfdf4886becc0977bf9c
:10fe4800ce8685be172477bfaac484be3c3e77bf42
:10fe5800700284be3a5877bf224083be137277bfc0
:10fe6800c07d82bec58b77bf4abb81be51a577bf17
:10fe7800c0f880beb7be77bf223680bef7d777bf3f
:10fe8800e1e67ebe10f177bf56617dbe040a78bff9
:10fe9800a4db7bbed12278bfcb557abe773b78bf37
:10fea800cccf78bef85378bfa64977be526c78bfde
:10feb8005ac375be868478bfe83c74be939c78bfed
:10fec80051b672be7bb478bf942f71be3bcc78bf5d
:10fed800b2a86fbed6e378bfab216ebe4afb78bf2f
:10fee8007f9a6cbe981279bf2f136bbebf2979bf5a
:10fef800ba8b69bec04079bf220468be9a5779bfe1
:10ff0800667c66be4e6e79bf86f464bedc8479bfbb
:10ff1800836c63be439b79bf5ce461be83b179bfe8
:10ff2800135c60be9dc779bfa8d35ebe91dd79bf63
:10ff38001a4b5dbe5ef379bf6ac25bbe04097abf25
:10ff480097395abe841e7abfa4b058bedd337abf33
:10ff58008f2757be10497abf589e55be1c5e7abf80
:10ff6800011554be02737abf898b52bec1877abf0e
:10ff7800f10151be599c7abf38784fbecbb07abfd9
:10ff880060ee4dbe16c57abf67644cbe3ad97abfdb
:10ff98004fda4abe37ed7abf185049be0e017bbf13
:10ffa800c2c547bebe147bbf4d3b46be48287bbf7b
:10ffb800b9b044beab3b7bbf072643bee74e7bbf11
:10ffc800379b41befc617bbf491040beea747bbfd2
:10ffd8003e853ebeb2877bbf15fa3cbe539a7bbfb7
:10ffe800cf6e3bbecdac7bbf6ce339be20bf7bbfc1
:10fff800ec5738be4dd17bbf50cc36be53e37bbfe8
:020000040001f9
:10000800984035be31f57bbfc4b433bee9067cbf2a
:10001800d42832be7a187cbfc99c30bee5297cbf83
:10002800a2102fbe283b7cbf61842dbe444c7cbff0
:1000380004f82bbe3a5d7cbf8d6b2abe086e7cbf70
:10004800fcde28beb07e7cbf515227be318f7cbffc
:100058008cc525be8a9f7cbfad3824bebdaf7cbf92
:10006800b6ab22bec9bf7cbfa51e21beaecf7cbf2a
:100078007b911fbe6cdf7cbf38041ebe03ef7cbfc4
:10008800de761cbe73fe7cbf6be91abebc0d7dbf5d
:10009800e05b19bedd1c7dbf3dce17bed82b7dbff2
:1000a800834016beac3a7dbfb2b214be59497dbf7b
:1000b800ca2413bede577dbfcc9611be3d667dbff8
:1000c800b70810be74747dbf8b7a0ebe85827dbf63
:1000d8004aec0cbe6e907dbff35d0bbe309e7dbfbb
:1000e80086cf09beccab7dbf054108be40b97dbff8
:1000f8006eb206be8cc67dbfc22305beb2d37dbf1d
:10010800029503beb1e07dbf2e0602be88ed7dbf1d
:10011800457700be38fa7dbf92d0fdbdc2067ebfce
:1001280073b2fabd24137ebf2c94f7bd5e1f7ebf49
:10013800c075f4bd722b7ebf2e57f1bd5e377ebff2
:100148007638eebd23437ebf9a19ebbdc14e7ebf04
:100158009afae7bd385a7ebf76dbe4bd88657ebf74
:100168002ebce1bdb0707ebfc49cdebdb17b7ebf3e
:10017800377ddbbd8b867ebf895dd8bd3d917ebf57
:10018800b93dd5bdc99b7ebfc81dd2bd2da67ebfba
:10019800b7fdcebd69b07ebf86ddcbbd7fba7ebf61
:1001a80036bdc8bd6dc47ebfc69cc5bd34ce7ebf3e
:1001b800397cc2bdd4d77ebf8d5bbfbd4ce17ebf4d
:1001c800c33abcbd9dea7ebfdd19b9bdc7f37ebf8a
:1001d800daf8b5bdc9fc7ebfbbd7b2bda4057fbfe9
:1001e80080b6afbd580e7fbf2b95acbde4167fbf60
:1001f800ba73a9bd491f7fbf3052a6bd87277fbfed
:100208008c30a3bd9d2f7fbfcf0ea0bd8d377fbf84
:10021800f9ec9cbd543f7fbf0acb99bdf4467fbf24
:1002280005a996bd6d4e7fbfe78693bdbf557fbfbd
:10023800b46490bde95c7fbf6a428dbdec637fbf4b
:100248000a208abdc76a7fbf94fd86bd7b717fbfc8
:100258000adb83bd08787fbf6cb880bd6d7e7fbf29
:10026800742b7bbdab847fbfe9e574bdc28a7fbfb9
:1002780038a06ebdb1907fbf625a68bd78967fbfc7
:10028800681462bd189c7fbf4cce5bbd91a17fbf37
:100298000e8855bde3a67fbfaf414fbd0dac7fbff4
:1002a8002ffb48bd0fb17fbf91b442bdeab57fbff8
:1002b800d56d3cbd9eba7fbffc2636bd2abf7fbf29
:1002c80007e02fbd8fc37fbff69829bdccc77fbf7e
:1002d800cc5123bde2cb7fbf880a1dbdd1cf7fbfe4
:1002e8002cc316bd98d37fbfb87b10bd37d77fbf4f
:1002f8002f340abdafda7fbf90ec03bd00de7fbfad
:10030800b949fbbc29e17fbf2dbaeebc2be47fbf06
:100318007b2ae2bc05e77fbfa69ad5bcb8e97fbfb8
:10032800b00ac9bc43ec7fbf9b7abcbca7ee7fbfb9
:1003380069eaafbce3f07fbf1c5aa3bcf8f27fbfe9
:10034800b6c996bce6f47fbf38398abcacf67fbf25
:100358004b517bbc4af87fbf003062bcc1f97fbffc
:10036800900e49bc11fb7fbf02ed2fbc39fc7fbf4b
:1003780059cb16bc39fd7fbf3053fbbb13fe7fbf83
:10038800890fc9bbc4fe7fbfc1cb96bb4eff7fbfe1
:10039800c70f49bbb1ff7fbfd40fc9baecff7fbffe
:1003a80000000080000080bfd40fc93aecff7fbf77
:1003b800c70f493bb1ff7fbfc1cb963b4eff7fbf05
:1003c800890fc93bc4fe7fbf3053fb3b13fe7fbf81
:1003d80059cb163c39fd7fbf02ed2f3c39fc7fbf5e
:1003e800900e493c11fb7fbf0030623cc1f97fbfd2
:1003f8004b517b3c4af87fbf38398a3cacf67fbf0b
:10040800b6c9963ce6f47fbf1c5aa33cf8f27fbffe
:1004180069eaaf3ce3f07fbf9b7abc3ca7ee7fbfa5
:10042800b00ac93c43ec7fbfa69ad53cb8e97fbf68
:100438007b2ae23c05e77fbf2dbaee3c2be47fbf69
:10044800b949fb3c29e17fbf90ec033d00de7fbf4b
:100458002f340a3dafda7fbfb87b103d37d77fbf57
:100468002cc3163d98d37fbf880a1d3dd1cf7fbfcf
:10047800cc51233de2cb7fbff698293dccc77fbf47
:1004880007e02f3d8fc37fbffc26363d2abf7fbfc5
:10049800d56d3c3d9eba7fbf91b4423deab57fbf62
:1004a8002ffb483d0fb17fbfaf414f3d0dac7fbf24
:1004b8000e88553de3a67fbf4cce5b3d91a17fbf23
:1004c8006814623d189c7fbf625a683d78967fbf6a
:1004d80038a06e3db1907fbfe9e5743dc28a7fbf09
:1004e800742b7b3dab847fbf6cb8803d6d7e7fbf36
:1004f8000adb833d08787fbf94fd863d7b717fbf13
:100508000a208a3dc76a7fbf6a428d3dec637fbf80
:10051800b464903de95c7fbfe786933dbf557fbfdc
:1005280005a9963d6d4e7fbf0acb993df4467fbf26
:10053800f9ec9c3d543f7fbfcf0ea03d8d377fbf68
:100548008c30a33d9d2f7fbf3052a63d87277fbfac
:10055800ba73a93d491f7fbf2b95ac3de4167fbff9
:1005680080b6af3d580e7fbfbbd7b23da4057fbf55
:10057800daf8b53dc9fc7ebfdd19b93dc7f37ebfca
:10058800c33abc3d9dea7ebf8d5bbf3d4ce17ebf5b
:10059800397cc23dd4d77ebfc69cc53d34ce7ebf14
:1005a80036bdc83d6dc47ebf86ddcb3d7fba7ebffc
:1005b800b7fdce3d69b07ebfc81dd23d2da67ebf1a
:1005c800b93dd53dc99b7ebf895dd83d3d917ebf74
:1005d800377ddb3d8b867ebfc49cde3db17b7ebf15
:1005e8002ebce13db0707ebf76dbe43d88657ebf02
:1005f8009afae73d385a7ebf9a19eb3dc14e7ebf45
:100608007638ee3d23437ebf2e57f13d5e377ebfe1
:10061800c075f43d722b7ebf2c94f73d5e1f7ebfe4
:1006280073b2fa3d24137ebf92d0fd3dc2067ebf51
:100638004577003e38fa7dbf2e06023e88ed7dbf25
:100648000295033eb1e07dbfc223053eb2d37dbf14
:100658006eb2063e8cc67dbf0541083e40b97dbfdf
:1006680086cf093eccab7dbff35d0b3e309e7dbf90
:100678004aec0c3e6e907dbf8b7a0e3e85827dbf24
:10068800b708103e74747dbfcc96113e3d667dbfa1
:10069800ca24133ede577dbfb2b2143e59497dbf0e
:1006a8008340163eac3a7dbf3dce173ed82b7dbf6a
:1006b800e05b193edd1c7dbf6be91a3ebc0d7dbfba
:1006c800de761c3e73fe7cbf38041e3e03ef7cbf03
:1006d8007b911f3e6cdf7cbfa51e213eaecf7cbf49
:1006e800b6ab223ec9bf7cbfad38243ebdaf7cbf90
:1006f8008cc5253e8a9f7cbf5152273e318f7cbfd7
:10070800fcde283eb07e7cbf8d6b2a3e086e7cbf27
:1007180004f82b3e3a5d7cbf61842d3e444c7cbf7f
:10072800a2102f3e283b7cbfc99c303ee5297cbfe8
:10073800d428323e7a187cbfc4b4333ee9067cbf65
:100748009840353e31f57bbf50cc363e53e37bbff6
:10075800ec57383e4dd17bbf6ce3393e20bf7bbfa1
:10076800cf6e3b3ecdac7bbf15fa3c3e539a7bbf68
:100778003e853e3eb2877bbf4910403eea747bbf50
:10078800379b413efc617bbf0726433ee74e7bbf5c
:10079800b9b0443eab3b7bbf4d3b463e48287bbf90
:1007a800c2c5473ebe147bbf1850493e0e017bbff1
:1007b8004fda4a3e37ed7abf67644c3e3ad97abf82
:1007c80060ee4d3e16c57abf38784f3ecbb07abf43
:1007d800f101513e599c7abf898b523ec1877abf3d
:1007e8000115543e02737abf589e553e1c5e7abf6f
:1007f8008f27573e10497abfa4b0583edd337abfe1
:1008080097395a3e841e7abf6ac25b3e04097abf92
:100818001a4b5d3e5ef379bfa8d35e3e91dd79bf8a
:10082800135c603e9dc779bf5ce4613e83b179bfcc
:10083800836c633e439b79bf86f4643edc8479bf56
:10084800667c663e4e6e79bf2204683e9a5779bf31
:10085800ba8b693ec04079bf2f136b3ebf2979bf61
:100868007f9a6c3e981279bfab216e3e4afb78bfe7
:10087800b2a86f3ed6e378bf942f713e3bcc78bfc9
:1008880051b6723e7bb478bfe83c743e939c78bf07
:100898005ac3753e868478bfa649773e526c78bfa6
:1008a800cccf783ef85378bfcb557a3e773b78bfac
:1008b800a4db7b3ed12278bf56617d3e040a78bf17
:1008c800e1e67e3e10f177bf2236803ef7d777bf4c
:1008d800c0f8803eb7be77bf4abb813e51a577bfff
:1008e800c07d823ec58b77bf2240833e137277bf9f
:1008f8007002843e3a5877bfaac4843e3c3e77bf14
:10090800ce86853e172477bfdf48863ecc0977bf61
:10091800da0a873e5bef76bfc1cc873ec4d476bf88
:10092800938e883e07ba76bf5050893e249f76bf83
:10093800f8118a3e1b8476bf8ad38a3eec6876bf5c
:1009480007958b3e974d76bf6e568c3e1b3276bf11
:10095800c0178d3e7a1676bffcd88d3eb3fa75bfa8
:10096800229a8e3ec6de75bf325b8f3eb3c275bf1c
:100978002c1c903e7ba675bf10dd903e1c8a75bf6f
:10098800dd9d913e976d75bf945e923eed5075bfab
:10099800351f933e1d3475bfbfdf933e271775bfc4
:1009a80031a0943e0bfa74bf8d60953ec9dc74bfcc
:1009b800d220963e62bf74bf00e1963ed5a174bfb7
:1009c80017a1973e228474bf1661983e496674bf8a
:1009d800fe20993e4b4874bfcee0993e272a74bf4b
:1009e80086a09a3edd0b74bf27609b3e6eed73bff9
:1009f800af1f9c3ed9ce73bf20df9c3e1fb073bf94
:100a0800789e9d3e3f9173bfb85d9e3e397273bf1d
:100a1800df1c9f3e0e5373bfeedb9f3ebe3373bf9a
:100a2800e59aa03e471473bfc259a13eacf472bf09
:100a38008718a23eebd472bf33d7a23e04b572bf6b
:100a4800c595a33ef89472bf3f54a43ec77472bfc5
:100a58009f12a53e705472bfe5d0a53ef43372bf15
:100a6800128fa63e521372bf254da73e8cf271bf5e
:100a78001f0ba83e9fd171bffec8a83e8eb071bfa4
:100a8800c486a93e578f71bf6f44aa3efb6d71bfe4
:100a98000102ab3e7a4c71bf77bfab3ed42a71bf1f
:100aa800d47cac3e080971bf153aad3e17e770bf5c
:100ab8003cf7ad3e02c570bf49b4ae3ec6a270bf9a
:100ac8003a71af3e668070bf102eb03ee15d70bfd8
:100ad800cbeab03e373b70bf6ba7b13e671870bf1b
:100ae800ef63b23e73f56fbf5820b33e5ad26fbf63
:100af800a5dcb33e1baf6fbfd698b43eb88b6fbfb3
:100b0800ec54b53e30686fbfe610b63e83446fbf05
:100b1800c3ccb63eb0206fbf8488b73ebafc6ebf68
:100b28002a44b83e9ed86ebfb2ffb83e5db46ebfd1
:100b38001ebbb93ef88f6ebf6e76ba3e6d6b6ebf48
:100b4800a031bb3ebe466ebfb6ecbb3eeb216ebfce
:100b5800afa7bc3ef2fc6dbf8b62bd3ed5d76dbf63
:100b68004a1dbe3e93b26dbfebd7be3e2d8d6dbf05
:100b78006f92bf3ea1676dbfd54cc03ef2416dbfbd
:100b88001e07c13e1d1c6dbf48c1c13e24f66cbf87
:100b9800557bc23e07d06cbf4435c33ec5a96cbf68
:100ba80015efc33e5e836cbfc8a8c43ed45c6cbf5f
:100bb8005c62c53e24366cbfd21bc63e500f6cbf6c
:100bc80029d5c63e58e86bbf628ec73e3bc16bbf96
:100bd8007c47c83efb996bbf7700c93e95726bbfd7
:100be80053b9c93e0c4b6bbf1072ca3e5e236bbf34
:100bf800ae2acb3e8cfb6abf2ce3cb3e95d36abfb3
:100c08008b9bcc3e7bab6abfca53cd3e3c836abf4d
:100c1800ea0bce3ed95a6abfeac3ce3e52326abf09
:100c2800ca7bcf3ea7096abf8a33d03ed7e069bfe7
:100c38002aebd03ee4b769bfaaa2d13ecc8e69bfe9
:100c4800095ad23e916569bf4811d33e323c69bf0b
:100c580067c8d33eae1269bf647fd43e07e968bf58
:100c68004136d53e3cbf68bffdecd53e4c9568bfcc
:100c780099a3d63e396b68bf135ad73e034168bf64
:100c88006b10d83ea81668bfa3c6d83e2aec67bf2b
:100c9800b97cd93e87c167bfad32da3ec19667bf1e
:100ca80080e8da3ed86b67bf319edb3eca4067bf3b
:100cb800c153dc3e991567bf2e09dd3e45ea66bf84
:100cc80079bedd3eccbe66bfa273de3e309366bf02
:100cd800a928df3e716766bf8ddddf3e8e3b66bfac
:100ce8004f92e03e880f66bfee46e13e5ee365bf89
:100cf8006afbe13e10b765bfc4afe23ea08a65bf9c
:100d0800fa63e33e0b5e65bf0e18e43e543165bfdf
:100d1800fecbe43e790465bfcb7fe53e7bd764bf5d
:100d28007533e63e59aa64bffbe6e63e147d64bf10
:100d38005d9ae73eac4f64bf9c4de83e212264bffc
:100d4800b700e93e73f463bfaeb3e93ea1c663bf23
:100d58008166ea3eac9863bf3019eb3e956a63bf83
:100d6800bbcbeb3e5a3c63bf217eec3efc0d63bf20
:100d78006330ed3e7bdf62bf80e2ed3ed7b062bffd
:100d88007994ee3e108262bf4c46ef3e265362bf16
:100d9800fbf7ef3e1a2462bf85a9f03eeaf461bf73
:100da800ea5af13e98c561bf290cf23e229661bf0e
:100db80043bdf23e8a6661bf386ef33ed03661bfee
:100dc800071ff43ef20661bfb1cff43ef2d660bf12
:100dd8003580f53ecfa660bf9330f63e897660bf7a
:100de800cbe0f63e214660bfdc90f73e961560bf2b
:100df800c840f83ee9e45fbf8ef0f83e19b45fbf23
:100e08002da0f93e27835fbfa54ffa3e12525fbf60
:100e1800f7fefa3edb205fbf22aefb3e81ef5ebfee
:100e2800275dfc3e05be5ebf040cfd3e678c5ebfc1
:100e3800bbbafd3ea65a5ebf4a69fe3ec3285ebfe6
:100e4800b217ff3ebef65dbff3c5ff3e97c45dbf58
:100e5800063a003f4d925dbfff90003fe15f5dbfe6
:100e6800e4e7003f532d5dbfb53e013fa3fa5cbfe9
:100e78007395013fd1c75cbf1cec013fdd945cbf9b
:100e8800b142023fc7615cbf3299023f8e2e5cbf00
:100e98009fef023f34fb5bbff845033fb8c75bbf1a
:100ea8003d9c033f1a945bbf6df2033f5a605bbfe2
:100eb8008948043f792c5bbf919e043f75f85abf5f
:100ec80084f4043f50c45abf624a053f09905abf90
:100ed8002ca0053fa05b5abfe2f5053f16275abf75
:100ee800824b063f6af259bf0ea1063f9cbd59bf0f
:100ef80086f6063fad8859bfe84b073f9c5359bf5c
:100f080036a1073f6a1e59bf6ff6073f17e958bf5a
:100f1800924b083fa1b358bfa1a0083f0b7e58bf12
:100f28009bf5083f534858bf7f4a093f791258bf7d
:100f38004e9f093f7fdc57bf09f4093f63a657bf9f
:100f4800ad480a3f267057bf3d9d0a3fc73957bf76
:100f5800b7f10a3f480357bf1c460b3fa7cc56bf03
:100f68006b9a0b3fe59556bfa5ee0b3f025f56bf48
:100f7800c9420c3ffe2756bfd7960c3fd9f055bf44
:100f8800d0ea0c3f93b955bfb33e0d3f2c8255bff5
:100f980081920d3fa44a55bf38e60d3ffb1255bf5d
:100fa800da390e3f31db54bf658d0e3f47a354bf7e
:100fb800dbe00e3f3b6b54bf3b340f3f0f3354bf56
:100fc80084870f3fc3fa53bfb8da0f3f55c253bfe8
:100fd800d52d103fc78953bfdc80103f185153bf30
:100fe800cdd3103f491853bfa726113f59df52bf31
:100ff8006b79113f49a652bf19cc113f186d52bfea
:10100800b01e123fc63352bf3071123f54fa51bf5f
:101018009ac3123fc2c051bfee15133f108751bf8c
:101028002a68133f3d4d51bf50ba133f4a1351bf71
:101038005f0c143f37d950bf585e143f039f50bf11
:1010480039b0143faf6450bf0402153f3b2a50bf6c
:10105800b753153fa8ef4fbf54a5153ff4b44fbf82
:10106800d9f6153f1f7a4fbf4748163f2b3f4fbf52
:101078009f99163f17044fbfdfea163fe4c84ebfdb
:10108800073c173f908d4ebf188d173f1c524ebf1f
:1010980012de173f89164ebff52e183fd5da4dbf21
:1010a800c07f183f029f4dbf73d0183f10634dbfdc
:1010b8000f21193ffd264dbf9471193fcbea4cbf54
:1010c80000c2193f79ae4cbf55121a3f08724cbf87
:1010d80093621a3f78354cbfb8b21a3fc7f84bbf76
:1010e800c6021b3ff8bb4bbfbb521b3f097f4bbf20
:1010f80099a21b3ffa414bbf5ff21b3fcc044bbf89
:101108000c421c3f7fc74abfa2911c3f138a4abfab
:101118001fe11c3f874c4abf84301d3fdc0e4abf8d
:10112800d17f1d3f12d149bf06cf1d3f299349bf2b
:10113800221e1e3f215549bf266d1e3ffa1649bf84
:1011480012bc1e3fb3d848bfe50a1f3f4e9a48bf9e
:101158009f591f3fca5b48bf41a81f3f271d48bf73
:10116800cbf61f3f65de47bf3b45203f849f47bf07
:101178009393203f856047bfd2e1203f672147bf57
:10118800f92f213f2ae246bf067e213fcea246bf65
:10119800fbcb213f546346bfd719223fbb2346bf31
:1011a8009967223f03e445bf43b5223f2da445bfbd
:1011b800d302233f396445bf4b50233f262445bf04
:1011c800a99d233ff5e344bfeeea233fa5a344bf0f
:1011d8001a38243f376344bf2c85243fab2244bfd1
:1011e80025d2243f00e243bf041f253f38a143bf57
:1011f800cb6b253f516043bf77b8253f4c1f43bf9a
:101208000a05263f29de42bf8451263fe89c42bf9b
:10121800e39d263f895b42bf2aea263f0b1a42bf5d
:101228005636273f70d841bf6882273fb79641bfdf
:1012380061ce273fe15441bf401a283fec1241bf1d
:101248000566283fdad040bfb0b1283fa98e40bf1d
:1012580041fd283f5c4c40bfb848293ff00940bfda
:101268001594293f67c73fbf57df293fc0843fbf59
:10127800802a2a3ffc413fbf8e752a3f1bff3ebf95
:1012880082c02a3f1bbc3ebf5b0b2b3fff783ebf93
:101298001b562b3fc5353ebfbfa02b3f6ef23dbf4f
:1012a8004aeb2b3ff9ae3dbfb9352c3f676b3dbfcd
:1012b8000f802c3fb8273dbf49ca2c3fece33cbf09
:1012c80069142d3f03a03cbf6f5e2d3ffc5b3cbf04
:1012d80059a82d3fd9173cbf29f22d3f98d33bbfc2
:1012e800de3b2e3f3b8f3bbf78852e3fc14a3bbf3d
:1012f800f7ce2e3f29063bbf5b182f3f75c13abf7b
:10130800a5612f3fa47c3abfd3aa2f3fb7373abf76
:10131800e6f32f3facf239bfde3c303f85ad39bf35
:10132800bb85303f426839bf7cce303fe12239bfb0
:101338002217313f65dd38bfad5f313fcb9738bfee
:101348001da8313f165238bf71f0313f430c38bfea
:10135800aa38323f55c637bfc780323f4a8037bfa9
:10136800c9c8323f233a37bfaf10333fdff336bf28
:101378007a58333f7fad36bf29a0333f046736bf65
:10138800bce7333f6c2036bf342f343fb8d935bf64
:101398008f76343fe79235bfcfbd343ffb4b35bf27
:1013a800f304353ff30435bffb4b353fcfbd34bfa6
:1013b800e792353f8f7634bfb8d9353f342f34bfe5
:1013c8006c20363fbce733bf0467363f29a033bfe4
:1013d8007fad363f7a5833bfdff3363faf1033bfa8
:1013e800233a373fc9c832bf4a80373fc78032bf28
:1013f80055c6373faa3832bf430c383f71f031bf6a
:101408001652383f1da831bfcb97383fad5f31bf6b
:1014180065dd383f221731bfe122393f7cce30bf2e
:101428004268393fbb8530bf85ad393fde3c30bfb0
:10143800acf2393fe6f32fbfb7373a3fd3aa2fbff5
:10144800a47c3a3fa5612fbf75c13a3f5b182fbff7
:1014580029063b3ff7ce2ebfc14a3b3f78852ebfba
:101468003b8f3b3fde3b2ebf98d33b3f29f22dbf3e
:10147800d9173c3f59a82dbffc5b3c3f6f5e2dbf81
:1014880003a03c3f69142dbfece33c3f49ca2cbf85
:10149800b8273d3f0f802cbf676b3d3fb9352cbf48
:1014a800f9ae3d3f4aeb2bbf6ef23d3fbfa02bbfcd
:1014b800c5353e3f1b562bbfff783e3f5b0b2bbf0e
:1014c8001bbc3e3f82c02abf1bff3e3f8e752abf12
:1014d800fc413f3f802a2abfc0843f3f57df29bfd6
:1014e80067c73f3f159429bff009403fb84829bf57
:1014f8005c4c403f41fd28bfa98e403fb0b128bf9a
:10150800dad0403f056628bfec12413f401a28bf99
:10151800e154413f61ce27bfb796413f688227bf5c
:1015280070d8413f563627bf0b1a423f2aea26bfda
:10153800895b423fe39d26bfe89c423f845126bf1a
:1015480029de423f0a0526bf4c1f433f77b825bf17
:101558005160433fcb6b25bf38a1433f041f25bfd4
:1015680000e2433f25d224bfab22443f2c8524bf51
:101578003763443f1a3824bfa5a3443feeea23bf8c
:10158800f5e3443fa99d23bf2624453f4b5023bf85
:101598003964453fd30223bf2da4453f43b522bf3d
:1015a80003e4453f996722bfbb23463fd71922bfb3
:1015b8005463463ffbcb21bfcea2463f067e21bfe8
:1015c8002ae2463ff92f21bf6721473fd2e120bfda
:1015d8008560473f939320bf849f473f3b4520bf8b
:1015e80065de473fcbf61fbf271d483f41a81fbff9
:1015f800ca5b483f9f591fbf4e9a483fe50a1fbf25
:10160800b3d8483f12bc1ebffa16493f266d1ebf0d
:101618002155493f221e1ebf2993493f06cf1dbfb2
:1016280012d1493fd17f1dbfdc0e4a3f84301dbf18
:10163800874c4a3f1fe11cbf138a4a3fa2911cbf37
:101648007fc74a3f0c421cbfcc044b3f5ff21bbf15
:10165800fa414b3f99a21bbf097f4b3fbb521bbfaf
:10166800f8bb4b3fc6021bbfc7f84b3fb8b21abf07
:1016780078354c3f93621abf08724c3f55121abf17
:1016880079ae4c3f00c219bfcbea4c3f947119bfe9
:10169800fd264d3f0f2119bf10634d3f73d018bf72
:1016a800029f4d3fc07f18bfd5da4d3ff52e18bfba
:1016b80089164e3f12de17bf1c524e3f188d17bfba
:1016c800908d4e3f073c17bfe4c84e3fdfea16bf78
:1016d80017044f3f9f9916bf2b3f4f3f474816bff0
:1016e8001f7a4f3fd9f615bff4b44f3f54a515bf25
:1016f800a8ef4f3fb75315bf3b2a503f040215bf11
:10170800af64503f39b014bf039f503f585e14bfb9
:1017180037d9503f5f0c14bf4a13513f50ba13bf1b
:101728003d4d513f2a6813bf1087513fee1513bf37
:10173800c2c0513f9ac312bf54fa513f307112bf11
:10174800c633523fb01e12bf186d523f19cc11bf9d
:1017580049a6523f6b7911bf59df523fa72611bfe7
:101768004918533fcdd310bf1851533fdc8010bfe9
:10177800c789533fd52d10bf55c2533fb8da0fbfa5
:10178800c3fa533f84870fbf0f33543f3b340fbf17
:101798003b6b543fdbe00ebf47a3543f658d0ebf44
:1017a80031db543fda390ebffb12553f38e60dbf27
:1017b800a44a553f81920dbf2c82553fb33e0dbfc1
:1017c80093b9553fd0ea0cbfd9f0553fd7960cbf17
:1017d800fe27563fc9420cbf025f563fa5ee0bbf1e
:1017e800e595563f6b9a0bbfa7cc563f1c460bbfdf
:1017f8004803573fb7f10abfc739573f3d9d0abf56
:101808002670573fad480abf63a6573f09f409bf82
:101818007fdc573f4e9f09bf7912583f7f4a09bf67
:101828005348583f9bf508bf0b7e583fa1a008bfff
:10183800a1b3583f924b08bf17e9583f6ff607bf4f
:101848006a1e593f36a107bf9c53593fe84b07bf53
:10185800ad88593f86f606bf9cbd593f0ea106bf0d
:101868006af2593f824b06bf16275a3fe2f505bf79
:10187800a05b5a3f2ca005bf09905a3f624a05bf9a
:1018880050c45a3f84f404bf75f85a3f919e04bf70
:10189800792c5b3f894804bf5a605b3f6df203bff8
:1018a8001a945b3f3d9c03bfb8c75b3ff84503bf35
:1018b80034fb5b3f9fef02bf8e2e5c3f329902bf25
:1018c800c7615c3fb14202bfdd945c3f1cec01bfc5
:1018d800d1c75c3f739501bfa3fa5c3fb53e01bf1a
:1018e800532d5d3fe4e700bfe15f5d3fff9000bf20
:1018f8004d925d3f063a00bf97c45d3ff3c5ffbefa
:10190800bef65d3fb217ffbec3285e3f4a69febe02
:10191800a65a5e3fbbbafdbe678c5e3f040cfdbe97
:1019280005be5e3f275dfcbe81ef5e3f22aefbbe7b
:10193800db205f3ff7fefabe12525f3fa54ffabeab
:1019480027835f3f2da0f9be19b45f3f8ef0f8be24
:10195800e9e45f3fc840f8be9615603fdc90f7beeb
:101968002146603fcbe0f6be8976603f9330f6bef5
:10197800cfa6603f3580f5bef2d6603fb1cff4be4a
:10198800f206613f071ff4bed036613f386ef3bee2
:101998008a66613f43bdf2be2296613f290cf2bec2
:1019a80098c5613fea5af1beeaf4613f85a9f0bee5
:1019b8001a24623ffbf7efbe2653623f4c46efbe48
:1019c8001082623f7994eebed7b0623f80e2edbeee
:1019d8007bdf623f6330edbefc0d633f217eecbed2
:1019e8005a3c633fbbcbebbe956a633f3019ebbef5
:1019f800ac98633f8166eabea1c6633faeb3e9be59
:101a080073f4633fb700e9be2122643f9c4de8bef2
:101a1800ac4f643f5d9ae7be147d643ffbe6e6becb
:101a280059aa643f7533e6be7bd7643fcb7fe5beda
:101a38007904653ffecbe4be5431653f0e18e4be21
:101a48000b5e653ffa63e3bea08a653fc4afe2bea2
:101a580010b7653f6afbe1be5ee3653fee46e1be57
:101a6800880f663f4f92e0be8e3b663f8ddddfbe3e
:101a78007167663fa928dfbe3093663fa273debe5a
:101a8800ccbe663f79beddbe45ea663f2e09ddbea7
:101a98009915673fc153dcbeca40673f319edbbe24
:101aa800d86b673f80e8dabec196673fad32dabed1
:101ab80087c1673fb97cd9be2aec673fa3c6d8bea9
:101ac800a816683f6b10d8be0341683f135ad7beab
:101ad800396b683f99a3d6be4c95683ffdecd5bedf
:101ae8003cbf683f4136d5be07e9683f647fd4be36
:101af800ae12693f67c8d3be323c693f4811d3beb6
:101b08009165693f095ad2becc8e693faaa2d1be5f
:101b1800e4b7693f2aebd0bed7e0693f8a33d0be2d
:101b2800a7096a3fca7bcfbe52326a3feac3cebe1c
:101b3800d95a6a3fea0bcebe3c836a3fca53cdbe30
:101b48007bab6a3f8b9bccbe95d36a3f2ce3cbbe65
:101b58008cfb6a3fae2acbbe5e236b3f1072cabeb7
:101b68000c4b6b3f53b9c9be95726b3f7700c9be2a
:101b7800fb996b3f7c47c8be3bc16b3f628ec7bebb
:101b880058e86b3f29d5c6be500f6c3fd21bc6be66
:101b980024366c3f5c62c5bed45c6c3fc8a8c4be2a
:101ba8005e836c3f15efc3bec5a96c3f4435c3be09
:101bb80007d06c3f557bc2be24f66c3f48c1c1befe
:101bc8001d1c6d3f1e07c1bef2416d3fd54cc0be06
:101bd800a1676d3f6f92bfbe2d8d6d3febd7bebe27
